:020000040800F2
:1000000000000110F535040839C80308B5050108DA
:10001000F9360408F9360408F9360408000000002F
:1000200000000000000000000000000085CE030872
:1000300081CE0308000000007DCE0308F19F000878
:10004000F9360408F9360408F9360408F9360408C4
:10005000F9360408F93604089D8F0108C990010893
:100060008D9001085190010815900108152704088A
:1000700005270408F5260408E5260408D526040803
:10008000C1260408AD260408F9360408F936040828
:10009000F9360408F9360408F9360408D98F01083E
:1000A0002196000891960008F9360408A1960008E8
:1000B000819600087196000861960008D52704080B
:1000C000DD270408C5270408CD270408F9360408ED
:1000D000F9360408BDA10008F93604081DA100087E
:1000E000638F0108F93604089DCF030811960008B4
:1000F00031960008F936040841960008992604084C
:10010000F9360408F936040851960008F93604084F
:10011000F9360408F936040835460208194602087B
:1001200085260408712604085D260408492604086B
:1001300035260408F9360408F9360408F9360408A7
:10014000F9360408F9360408F93604083DC80308EE
:10015000212604080D260408F92504087DA00008BE
:10016000B5270408BD270408F9360408F936040841
:10017000F9360408F9360408F9360408F936040893
:08018000F9360408F936040801
:080188008C31040001000000AD
:1001900016000800EC290020042A002000000000BE
:1001A000900600081D000100DC2F002068300020B0
:1001B000000000009806000827000400FC2F002023
:1001C0006C300020000000009A06000801010400C5
:1001D000003100204040002000000000000000002E
:1001E00008020900643F0020444000200000000095
:1001F0000988010806020C00DC3F00205040002066
:10020000000000001F8C01080702020000400020CF
:100210005C400020000000009E06000802000C0068
:10022000E83F0020604000200000000000000000C7
:10023000F7010600583F00206C400020000000003D
:10024000A00600082C001000D4450020C445002062
:1002500000000000E50302082B00240008460020EF
:10026000E445002000000000B5030208290050000A
:10027000F04400202C460020000000000000000098
:100280000A020A00A8460020B8460020000000002C
:10029000A606000804020200944B0020D04B002068
:1002A00000000000B006000803123300AB4E00202F
:1002B000784E002000000000B406000825005A0017
:1002C000C44D00201E4E0020000000000000000071
:1002D000F6110C00B84D0020AC4D002000000000CD
:1002E000E806000815007000CC4C00203C4D0020B2
:1002F00000000000000000002A0060000C4C0020FC
:100300006C4C0020000000006D1D03080902010074
:10031000D85100203052002000000000F4060008F0
:100320000C0024006C51002034520020000000001A
:1003300011C301080102050060510020585200203D
:1003400000000000D187020800020500384F00209D
:1003500060520020000000000000000003010A00BD
:10036000C0520020CC52002000000000F606000819
:100370000B201000DC550020645600200000000017
:10038000000700081F000E000454002074560020CF
:10039000000000001007000805020100EC530020D7
:1003A00084560020000000001E07000804008000A2
:1003B0005C670020DC6700200000000000000000F7
:1003C000F90104002C5C00205C68002000000000A3
:1003D00029840008FD012400045C002060680020DE
:1003E00000000000B98300080600160084580020B1
:1003F0008468002000000000F91D0308FB010100D3
:10040000C05700209C6800200000000035800008D4
:10041000FC0109008C560020A068002000000000AC
:10042000018000080A101200E07C0020E484002013
:100430000000000020070008340010000C7C0020A1
:10044000F884002000000000951D030812200C0015
:10045000FC7B002008850020000000003207000817
:1004600011000C008870002014850020000000009E
:1004700079C3010818102C00287000202085002066
:1004800000000000390C02080D00340054700020F8
:100490004C85002000000000FDCF0308FA01020097
:1004A000BC68002080850020000000005D800008FE
:1004B0001E000400848500200C890020000000003C
:1004C0003E07000822000C0024880020108900202C
:1004D0000000000042070008012008001C8F0020D7
:1004E0003C8F0020000000004E0700081A000800A2
:1004F000008F0020448F00200000000056070008F5
:10050000030001000091002008910020000000007D
:100510000000000002020300E4920020EC920020A0
:1005200000000000000000000C020100D492002036
:10053000F0920020000000005E070008FE010900A4
:10054000B8920020F4920020000000003D800008D6
:1005500014000200A0950020A495002000000000D7
:10056000600700081000030090950020A895002067
:10057000000000006207000828001000809500209D
:10058000AC95002000000000B146020823001000D6
:1005900070950020BC95002000000000CD460208A8
:1005A0001900050068950020CC950020000000008F
:1005B00066070008F811010064950020D49500201A
:1005C000000000006C070008000104006095002096
:1005D000D8950020000000006E0700081B00F40002
:1005E000E495002088A4002000000000F901030821
:1005F0000E020200C49700207CA50020000000002D
:10060000720700082F00110072A4002080A50020AE
:10061000000000007407000805100600C0A60020B6
:1006200094A800200000000086070008F5216C0057
:1006300054A600209CA8002000000000B98E0308EA
:1006400026000E0018A9002008A9002000000000C4
:1006500071AA03080E20EA00F8BF002068C100203C
:1006600000000000D91D03081300040028C1002069
:1006700054C20020000000008C07000802010300A3
:10068000E3BF002058C200200000000039C3010869
:10069000C409000019012828000020030000013CC3
:1006A00024010000000000004A01B400D60100004F
:1006B000000000000000000000000000000000003A
:1006C000000000000000000000000000000000002A
:1006D000000000000000000000000000000000001A
:1006E0000000000000000100000000000000000009
:1006F000000000002E00040101006C160000000044
:100700002B21231E64010100000001000A012900C1
:1007100000000000000001000000000500000000D3
:1007200000300100005A0000000090012C01C800B8
:1007300064000000000100054F4246340000000044
:100740000100C800141E010064002C012800E80309
:100750006400040A00017E05EA05B40532000100C8
:1007600003000001050000002801000004009001C2
:100770000000000000000000000000000000000079
:10078000000000000000200001010000080004003B
:1007900001FF000001010000EC88040848BA0408C9
:1007A0000000000000000000FC8804080489040820
:1007B00000000000012000000889040810890408D6
:1007C0000000000001400000148904080C9E040889
:1007D0000000000001200000208904082C89040882
:1007E000000000000400000030890408ECC0040888
:1007F00000000000040000003C89040834B704082D
:100800000000000001000000020100000000803F25
:100810000000803F00000000000000000000000019
:100820000000803F24560408050804000000000072
:1008300004860408F4720408F0850408000000002F
:100840005056040805080A00000000000486040849
:10085000F47204081C86040800000000FFFFFFFF7C
:100860000101D6018DFD010800000000000000001C
:10087000000101010100E001080000002D202D2DE4
:10088000202D2D2D2D202D2D2D2D000000000000C0
:100890000000000000000000000000000000000058
:1008A00001020304010203040607080900FFFF0018
:1008B00000000000AA550501000001AA550B010027
:1008C00000AA5507010000AA550902000000000017
:1008D00001000000C012AA5503009F0001000000A3
:1008E0000000803F00000001000000000000000048
:1008F000000000001DC40308D5C30308C9CE0308C7
:1009000000000000F9BF03083DC20308C5C2030888
:100910009DC103080000000000000000EDBF0308B7
:100920006DBF030869BF030865BF030859BF03080B
:1009300055BF030861BF03085DBF0308E1BF03089B
:10094000D5BF0308ADBF0308C1BF030899BF0308A3
:1009500085BF030871BF03080000803F000000004E
:1009600000000000000000000000803F00000000C8
:100970000000000000000000000000000000000077
:100980000000000000000000000000000000000067
:100990000000803F00000000000000000000000098
:1009A000006002401060024000000000000B0000E8
:1009B0000000200000000000000000000060024075
:1009C0002860024000000000060C0000000020002B
:1009D0000000000000000000006002404060024093
:1009E00000000000100D00000000200000000000CA
:1009F000000000000060024058600240000000005B
:100A0000160E0000000020000000000000000000A2
:100A1000006002407060024000000000200F0000F3
:100A20000000200000000000000000000060024004
:100A30008860024000000000261000000000200036
:100A4000000000000000000000600240A0600240C2
:100A50000000000030110000000020000000000035
:100A60000000000000600240B8600240000000008A
:100A7000362F0000000020000000000000000000F1
:100A800000640240106402400000000000380000D2
:100A90000000400000000000000000000064024070
:100AA00028640240000000000639000000004000F9
:100AB00000000000000000000064024040640240AA
:100AC00000000000103A000000004000000000009C
:100AD0000000000000640240586402400000000072
:100AE000163B000000004000000000000000000075
:100AF000006402407064024000000000203C0000DE
:100B000000004000000000000000000000640240FF
:100B100088640240000000002644000000004000FD
:100B2000000000000000000000640240A0640240D9
:100B30000000000030450000000040000000000000
:100B40000000000000640240B864024000000000A1
:100B500036460000000040000000000000000000D9
:100B60000800000000000101FFFF0000FFFFFFFF81
:100B700001000000D8AD04080000000000000000E3
:100B80004DC30108A0860100040000000000000021
:100B90000000000000000000000000000000000055
:100BA000000000000000000058C80408E8A804087D
:100BB00000000000A53801087D00000006000000CC
:100BC0000000000000000000000000000000000025
:100BD00000000000000000000000000008C1040840
:100BE000000000000000000001FF0008E803000012
:100BF00003000000000000000000000000000000F2
:100C000000000000000000000000000000000000E4
:100C100010C104080000000000000000351F030898
:100C2000102700000300000000000000000000008A
:100C300000000000000000000000000000000000B4
:100C40000000000008B90408000000003D0202088E
:100C5000B1DC0008204E000005000000000000008C
:100C60000000000000000000000000000000000084
:100C7000000000000000000068AF04080000000051
:100C800000000000650601081027000001000000B8
:100C90000000000000000000000000000000000054
:100CA0000000000000000000000000001CC104085B
:100CB00000000000000000007DDC0008E8030000E8
:100CC000050000000000000000000000000000001F
:100CD0000000000000000000000000000000000014
:100CE00028C104080000000000000000ADC5010894
:100CF000204E000003000000000000000000000083
:100D000000000000000000000000000000000000E3
:100D10000000000038C104080000000000000000CE
:100D2000B5C30108204E00000300000000000000D1
:100D300000000000000000000000000000000000B3
:100D4000000000000000000048C10408000000008E
:100D500000000000F1020108400D03000300000044
:100D60000000000000000000000000000000000083
:100D70000000000000000000000000009CAE04081D
:100D800000000000000000001DDA0308102700002A
:100D90000100000000000000000000000000000052
:100DA0000000000000000000000000000000000043
:100DB00004A904080000000000000000C115030899
:100DC00010270000030000000000000000000000E9
:100DD0000000000000000000000000000000000013
:100DE0000000000058C104080000000000000000DE
:100DF000D9060408A08601000100000000000000E0
:100E000000000000000000000000000000000000E2
:100E10000000000000000000F4A80408000000002A
:100E200000000000F905040850C3000001000000A4
:100E300000000000000000000000000000000000B2
:100E4000000000000000000000000000FCA80408F2
:100E50000000000000000000F9AC03087011010060
:100E60000100000000000000000000000000000081
:100E70000000000000000000000000000000000072
:100E800060C1040800000000000000002D000408FC
:100E9000A861000001000000000000000000000048
:100EA0000000000000000000000000000000000042
:100EB000000000006CC104080000000000000000F9
:100EC000A5930208A08601000100000000000000B8
:100ED0000000000000000000000000000000000012
:100EE000000000000000000070AF040800000000D7
:100EF00000000000BD0B0108A00F00000100000071
:100F000000000000000000000000000000000000E1
:100F100000000000000000000000000078C104088C
:100F200000000000000000004193030810270000AB
:100F300001000000000000000000000000000000B0
:100F400000000000000000000000000000000000A1
:100F5000C8AE04080000000000000000B5C701088A
:100F6000A00F0000010000000000000000000000D1
:100F70000000000000000000000000000000000071
:100F800000000000A4AE0408000000000000000003
:100F900075AD03081A4100000100000000000000C8
:100FA0000000000000000000000000000000000041
:100FB0000000000000000000D4AF040800000000A2
:100FC00000000000BDB20208102700000100000070
:100FD0000000000000000000000000000000000011
:100FE00000000000000000000000000040C00408F5
:100FF00000000000000000006DF403081A4100002A
:1010000001000000000000000000000000000000DF
:1010100000000000000000000000000000000000D0
:1010200084C1040800000000000000008DAC01082D
:10103000400D030000000000000000000000000060
:1010400000000000000000000000000000000000A0
:10105000000000008CC10408000000000000000037
:1010600029AC0108400D0300000000000000000052
:101070000000000000000000000000000000000070
:10108000000000000000000094C1040800000000FF
:1010900000000000C51A0308A0860100030000003C
:1010A0000000000000000000000000000000000040
:1010B000000000000000000000000000FFFFFFFF34
:1010C0000403090412010002020200408304405795
:1010D000000201020301000009024300020100C0F6
:1010E000320904000001020201000524001001057C
:1010F00024010001042402020524060001070582E0
:10110000030800FF09040100020A000000070501AE
:10111000024000000705810240000000FF000000BF
:1011200015A90208F1C20308C9A3020841C00308B7
:10113000B1C4030851C003086DC0030831C00308DF
:1011400021C00308000000000000000001010100B0
:1011500089DF030800000000340B00200CC50408E0
:10116000000000000000000000000000000000007F
:1011700048BA04080000000000000000A00B002096
:1011800004000000B8C404080D000000F1E70308E3
:10119000840F002000000000D0C704080D000000EC
:1011A00019E80308780F0020000000002CC504088F
:1011B00008000000000000006C0F00200400000088
:1011C0001CC504080D00000031E00308600F00207A
:1011D00000000000CCC304080300000005F303086E
:1011E000540F00200000000024C504080300000084
:1011F00005F30308480F002000000000D0C30408D6
:1012000001000000000000000000000000000000DD
:10121000000000000E0000000000000000000000C0
:10122000000000000CC504080000000000000000E1
:10123000000000000000000048BA040800000000A0
:1012400000000000A00B00200400000050C40408AF
:101250000300000005E603083C0F00200800000022
:101260001CC504080D00000031E00308600F0020D9
:1012700000000000CCC304080300000005F30308CD
:10128000540F00200000000024C5040803000000E3
:1012900005F30308480F002000000000D0C3040835
:1012A000010000000000000000000000000000003D
:1012B000000000000E000000000000000000000020
:1012C0000000000034C50408000000000000000019
:1012D000000000000000000048BA04080000000000
:1012E00000000000A00B00200400000058C4040807
:1012F0000300000005F30308900F00200000000029
:10130000D0C304080100000000000000000000003D
:1013100000000000000000000E00000000000000BF
:10132000000000000000000020700020702D7200FE
:101330002D202D2D202D2D2D2D202D2D2D0000008B
:10134000000000000000000000000000000000009D
:101350007EBF002088136F170100000080BF0020AF
:1013600088136F1700000000A4C3040800000000E9
:10137000000000000000000000000000B4C30408EA
:101380000800000000000000CC0B0020040000005A
:10139000C0C304080800000000000000C00B0020CB
:1013A00000000000CCC304080400000045E6030868
:1013B0000000000000000000D0C30408010000008D
:1013C000000000000000000000000000000000001D
:1013D0000E000000000000000000000000000000FF
:1013E0007CBF002088136F1701000000E453002029
:1013F00088136F1700000000E9DF030800000000F9
:10140000D80B002024C1002001000000C48504087E
:10141000E653002001000000D0850408DC530020C2
:1014200002000000D885040852BA00200000000025
:101430000000000050BA0020000000000000000082
:101440004EBA002000000000000000004CBA00204E
:1014500000000000000000004ABA00200000000068
:101460000000000048BA002000000000000000005A
:101470004401002000000000000000007BBF0020AD
:1014800002000000E485040808C40408000000000D
:10149000000000000000000000000000B4C30408C9
:1014A00008000000000000005C0C002004000000A8
:1014B000C0C304080800000000000000500C002019
:1014C00000000000CCC3040804000000BDDF0308D6
:1014D0000000000000000000D0C30408010000006C
:1014E00000000000000000000000000000000000FC
:1014F0000E000000000000000000000000000000DE
:1015000018C40408000000000000000000000000F3
:101510000000000028C404080D00000095E703083F
:101520008C0C00200400000034C404080D000000EE
:101530000DE00308800C00200400000040C40408F3
:101540000D00000059E70308740C002000000000A3
:101550004CC404080300000025E60308680C0020C2
:101560000800000058C404080300000005F3030845
:10157000900F002000000000D0C30408010000000C
:10158000000000000000000000000000000000005B
:101590000E0000000000000000000000000000003D
:1015A00060C404080000000000000000000000000B
:1015B0000000000068C404080400000061E603089D
:1015C0000000000000000000D0C30408010000007B
:1015D000000000000000000000000000000000000B
:1015E0000E000000000000000000000000000000ED
:1015F000C0C404080000000000000000000000005B
:101600000000000068B004080D00000000000000A9
:10161000EC0C002004000000D0C404080800000006
:1016200000000000E00C002004000000DCC40408FE
:101630000800000000000000D40C0020040000009E
:10164000E4C404080800000000000000C80C0020EA
:1016500004000000ECC404080800000000000000C2
:10166000BC0C002004000000F4C4040808000000C2
:1016700000000000B00C002004000000FCC40408BE
:101680000800000000000000A40C0020040000007E
:1016900004C504080800000000000000980C0020A9
:1016A00004000000D0C30408010000000000000096
:1016B0000000000000000000000000000E0000001C
:1016C000000000000000000000000000D5DF03085B
:1016D00000000000F80C00200000000000000000E6
:1016E000700D00200000000000000000100E00201F
:1016F000E253002004000000F0850408E0530020BD
:10170000E0150C1700000000DF5300200800000067
:10171000F4720408DE53002005000000048604086B
:101720000000000000000000600E0020000000002B
:1017300000000000D4220020FFFFFFFFFA0000009D
:10174000010000000100000060C5040868C504082D
:1017500060C4040800000000000000000000000059
:101760000000000056C50408040000007FE50308DF
:101770000000000000000000D0C3040801000000C9
:101780000000000000000000000000000000000059
:101790000E0000000000000000000000000000003B
:1017A0000ABA00200100C4090000000008BA0020A5
:1017B0000100C4090000000006BA00200100C409AD
:1017C0000000000004BA00200100C409000000006D
:1017D00000BA00200100C4090000000002BA002085
:1017E0000100C40900000000FEB900200100C40986
:1017F00000000000FCB900200100C4090000000046
:101800008EBF00200100C800010000008CBF002036
:1018100032003075320000008BBF0020055A0500F1
:1018200086BF002000FF01008ABF002001000000E9
:10183000B80F002088BF002002000000508004087C
:1018400085BF002000FF010089BF002001000000CB
:10185000B80F002087BF002002000000508004085D
:101860000000000000000000C00F00209A5200207D
:101870009CFF2C0100000000BC0900200A000000B1
:101880001C86040878BF0020E0150C17000000003B
:10189000BE09002008000000F4720408BD09002001
:1018A00005000000048604087ABF00200200000042
:1018B0003486040818C100200100FF7F01000000E9
:1018C00017C100200200000040860408ECBF002081
:1018D0000300000050860408EBBF00200300000056
:1018E00050860408EAC000200000F4010100000056
:1018F000E8C000200000F40101000000E6C0002064
:101900000000F40101000000E4C000200000F40128
:1019100001000000E2C0002000FF010002C1002021
:10192000E803D0070A00000000C1002000640100A5
:101930000A000000FCC0002000640100FBC0002081
:101940000064010001C10020006401000A000000E1
:10195000FAC00020006401000A000000FFC000205F
:10196000006401000A000000FEC0002000640100C5
:101970000A000000FDC00020006401000A00000011
:10198000F9C0002000FF01000A000000F8C000209C
:1019900000FF01000A000000F4BF00200000F40175
:1019A00001000000F2BF00200000F401010000006F
:1019B000F0BF00200000F40101000000EEBF002095
:1019C0000000F40101000000F4C000201400E8034E
:1019D00001000000F2C00020E803307501000000A3
:1019E000F1C0002000C80100F0C0002000C80100C4
:1019F000EFC0002000C80100EEC00020006401001C
:101A00000A000000EDC0002000FF01000A000000F5
:101A10000DC1002000C801000CC1002000C8010059
:101A20000BC1002000C801000AC1002000C801004D
:101A300009C1002000C8010008C1002000C8010041
:101A400007C1002000C8010006C1002000C8010035
:101A500005C1002000C801008CC50408000000007A
:101A60000000000000000000000000009CC5040809
:101A700009000000000000006410002004000000C5
:101A8000A4C5040809000000000000005810002050
:101A90000400000008CB040809000000000000005A
:101AA0004C100020040000007488040809000000A5
:101AB000000000004010002004000000ACC5040835
:101AC00009000000000000003410002004000000A5
:101AD000B4C5040809000000000000002810002020
:101AE00004000000BCC5040809000000000000005C
:101AF0001C10002004000000C4C5040809000000F8
:101B0000000000001010002004000000D0C30408F2
:101B100001000000000000000000000000000000C4
:101B2000000000000E0000000000000000000000A7
:101B300000000000C4C6040800000000000000000F
:101B400000000000000000008CAD04080700000049
:101B5000000000008810002000000000D4C6040827
:101B600008000000000000007C10002000000000C1
:101B7000E0C604080800000000000000701000200B
:101B800000000000D0C304080100000000000000B5
:101B90000000000000000000000000000E00000037
:101BA000000000000000000000000000E8C604087B
:101BB0000000000000000000000000000000000025
:101BC000F8C604080D00000000000000C41000204A
:101BD0000000000000C704080D0000000000000025
:101BE000B81000200000000008C70408070000002B
:101BF00000000000B01000200000000010C7040822
:101C00000D00000000000000A410002000000000F3
:101C100018C704080D000000000000009810002004
:101C20000000000020C704080700000000000000BA
:101C30009010002000000000D0C304080100000044
:101C40000000000000000000000000000000000094
:101C50000E00000000000000000000000000000076
:101C600028C7040800000000000000000000000079
:101C7000000000008CAD04080C0000000000000013
:101C800090BF0020000000003CC704080C000000CA
:101C90000000000092BF0020000000004CC70408B4
:101CA0000C00000000000000C8BF00200000000081
:101CB0005CC704080C00000000000000BCBF00204E
:101CC0000000000070C704080C00000000000000C5
:101CD00094BF002000000000E4C104080C000000D4
:101CE0000000000096BF0020000000007CC7040830
:101CF0000C0000000000000098BF00200000000061
:101D000090C704080C000000000000009ABF0020EB
:101D10000000000098C704080C000000000000004C
:101D20009CBF002000000000A0C704080C000000B9
:101D300000000000DABF002000000000B8C704085F
:101D40000C000000000000009EBF0020000000000A
:101D5000C4C704080C00000000000000A0BF002061
:101D60000000000000C004080C000000000000009B
:101D7000A2BF002000000000CCC704080C00000037
:101D800000000000A4BF002000000000D8C7040825
:101D90000C00000000000000A6BF002000000000B2
:101DA000E4C704080C00000000000000A8BF0020E9
:101DB00000000000F0C704080C0000000000000054
:101DC000AABF002000000000FCC704080C000000AF
:101DD00000000000ACBF00200000000008C804089C
:101DE0000C00000000000000C0BF00200000000048
:101DF00010C804080C00000000000000BEBF002056
:101E00000000000018C804080C00000000000000DA
:101E1000CCBF00200000000024C804080C00000013
:101E200000000000CEBF00200000000030C8040801
:101E30000C00000000000000D4BF002000000000E3
:101E400060C104080C00000000000000AEBF0020CC
:101E5000000000001CC504080C0000000000000089
:101E6000B6BF0020000000003CC804080C000000C1
:101E700000000000B0BF00200000000048C80408B7
:101E80000C00000000000000B2BF002000000000B5
:101E900054C804080C00000000000000B4BF00207B
:101EA000000000005CC804080C00000000000000F6
:101EB000B8BF002000000000ACAD04080C0000001A
:101EC00000000000C2BF00200000000068C8040835
:101ED0000C00000000000000BABF0020000000005D
:101EE00074C804080C00000000000000CABF0020F5
:101EF0000000000080C804080C0000000000000082
:101F0000C4BF00200000000088C804080C000000C6
:101F100000000000C6BF00200000000090C80408B8
:101F20000C00000000000000D0BF002000000000F6
:101F300098C804080C00000000000000D2BF002078
:101F400000000000D0C304080100000000000000F1
:101F50000000000000000000000000000E00000073
:101F6000000000000000000000000000A0C80408FD
:101F70000000000000000000000000000000000061
:101F8000B0C804080500000000000000EABF0020FF
:101F900000000000D0C304080100000000000000A1
:101FA0000000000000000000000000000E00000023
:101FB000000000000000000000000000B8C8040895
:101FC0000000000000000000000000000000000011
:101FD00048BA04080000000000000000EC000020E7
:101FE00004000000FCB804080D000000E1E503084F
:101FF0001811002000000000B8C404080D00000003
:1020000041DF03080C11002000000000D0C70408C5
:102010000D00000025DF0308001100200000000073
:102020002CC504080800000000000000F410002087
:10203000040000001CC504080D00000071DE030848
:10204000E810002000000000C4C8040809000000D7
:1020500000000000DC10002004000000CCC30408D5
:102060000300000005F30308D0100020000000006A
:10207000D0C30408010000000000000000000000C0
:1020800000000000000000000E0000000000000042
:102090000000000000000000CCC8040800000000A0
:1020A000000000000000000000000000DCC8040880
:1020B0000D000000000000003011002000000000B2
:1020C000E4C804080A000000000000002CC1002041
:1020D00000000000F0C804080A0000000000000032
:1020E00034C1002000000000F8C804080A00000005
:1020F000000000003CC100200000000000C90408EE
:102100000800000000000000241100200000000072
:1021100008C90408040000004DEA0308000000009C
:1021200000000000D0C3040801000000000000000F
:102130000000000000000000000000000E00000091
:1021400000000000000000000000000014C90408A6
:10215000000000000000000000000000000000007F
:1021600028C904080D0000000000000048110020EC
:102170000000000038C904080400000095E80308C6
:10218000000000000000000040C904080D0000002D
:10219000000000003C1100200000000054C90408A9
:1021A0000400000071E803080000000000000000C7
:1021B000D0C304080100000000000000000000007F
:1021C00000000000000000000E0000000000000001
:1021D00000000000000000005CC9040800000000CE
:1021E00000000000000000000000000070C90408AA
:1021F0000700000000000000841100200000000023
:102200007CC90408080000000000000078110020CC
:102210000000000088C90408080000000000000059
:102220006C1100200000000094C9040808000000A0
:10223000000000006011002000000000A0C9040898
:102240000800000000000000541100200000000001
:10225000D0C30408010000000000000000000000DE
:1022600000000000000000000E0000000000000060
:102270000000000000000000ACC9040800000000DD
:10228000000000009B0B002000000000A087040855
:102290000B00000000000000FC1100200000000006
:1022A000B8C904080B00000000000000F011002075
:1022B00000000000C4C904080B000000000000007A
:1022C000E411002000000000D0C904080B00000049
:1022D00000000000D811002000000000DCC9040844
:1022E0000B00000000000000CC11002000000000E6
:1022F000A88704080B00000000000000C0110020A7
:1023000000000000E8C904080B0000000000000005
:10231000B411002000000000F4C904080700000008
:1023200000000000AC11002000000000FCC90408FF
:102330000700000000000000A411002000000000C1
:1023400008CA04080B0000000000000098110020DB
:102350000000000014CA040808000000000000008B
:102360008C11002000000000D0C304080100000010
:10237000000000000000000000000000000000005D
:102380000E0000000000000000000000000000003F
:1023900020CA040800000000000000000000000047
:1023A0000000000034CA040808000000000000001B
:1023B0002C1200200000000040CA040808000000A1
:1023C0000000000020120020000000004CCA040899
:1023D00008000000000000001412002000000000AF
:1023E00058CA04080800000000000000081200207D
:1023F00000000000D0C3040801000000000000003D
:102400000000000000000000000000000E000000BE
:1024100000000000000000000000000060CA040886
:102420000000000000000000980B002000000000E9
:1024300070CA04080B0000000000000074120020A5
:10244000000000007CCA04080B000000000000002F
:10245000681200200000000088CA0408070000007D
:1024600000000000601200200000000094CA040870
:1024700007000000000000005812002000000000CB
:10248000A0CA04080700000000000000501200204D
:1024900000000000ACCA04080800000000000000B2
:1024A0004412002000000000B4CA04080800000024
:1024B000000000003812002000000000D0C3040813
:1024C000010000000000000000000000000000000B
:1024D000000000000E0000000000000000000000EE
:1024E00000000000BCCA040800000000000000005A
:1024F000980B002000000000C8CA04080700000074
:1025000000000000C012002000000000D0CA040833
:102510000700000000000000B812002000000000CA
:10252000D8CA04080700000000000000B012002014
:10253000000000003C8804080700000000000000C4
:10254000A8120020000000004488040807000000D2
:1025500000000000A0120020000000004C880408C9
:10256000070000000000000098120020000000009A
:10257000E0CA0408070000000000000090120020DC
:1025800000000000E8CA0408070000000000000086
:102590008812002000000000F0CA040807000000B4
:1025A000000000008012002000000000D0C30408DA
:1025B000010000000000000000000000000000001A
:1025C000000000000E0000000000000000000000FD
:1025D000000000000000000005E20308C81200200F
:1025E000E8BF00201B00000060860408E7BF002051
:1025F0000A320100E6BF002001FA0100E2BF00201C
:1026000000C80100E0BF0020E803D007010000007F
:102610004F4D4E49425553463400000084BF0020C0
:102620000003010083BF00200003010029E103082B
:1026300005E10308A4130020CDE003088DE00308A2
:102640001C14002065E103084DE10308D0140020AC
:102650001BE2030841E80308DC170020ADDE030895
:10266000000000002C18002029EA03088DE403086C
:102670000819002041E2030800000000BC190020F6
:10268000E5E20308B5E20308481A002071E30308F5
:10269000B9E30308E81A0020F6C000200103010096
:1026A00081E2030855E20308001C002015E303083B
:1026B000B9E803088C1C0020E9E3030815E90308C6
:1026C000541D0020ECC0002001030100F8CA0408DA
:1026D00000000000000000000000000000000000FA
:1026E00004CB04080800000000000000741E002055
:1026F000000000000CCB04080700000000000000F0
:102700006C1E0020000000001CCB04080700000025
:1027100000000000641E00200000000028CB040818
:1027200007000000000000005C1E00200000000008
:1027300034CB04080D00000000000000501E0020F3
:102740000000000040CB04080300000005F303086C
:10275000441E002000000000D0C304080100000057
:102760000000000000000000000000000000000069
:102770000E0000000000000000000000000000004B
:1027800048CB04080000000000000000000000002A
:102790000000000058CB04080A0000000000000000
:1027A000008704080000000060CB04080A00000055
:1027B00000000000CC8804080000000068CB04087A
:1027C0000A000000000000000EC100200000000010
:1027D00070CB04080A00000000000000801E0020EA
:1027E00000000000D0C30408010000000000000049
:1027F0000000000000000000000000000E000000CB
:1028000000000000000000000000000078CB040879
:1028100000000000000000000000000000000000B8
:1028200084CB04080300000005F30308B41E002055
:102830000000000090CB04080300000005F303082B
:10284000A81E00200000000098CB04080300000030
:1028500005F303089C1E002000000000A0CB040824
:10286000050000000000000082BF00200000000002
:10287000A8CB04080700000000000000941E002000
:1028800000000000B4CB04080700000000000000B6
:102890008C1E002000000000D0C3040801000000CE
:1028A0000000000000000000000000000000000028
:1028B0000E0000000000000000000000000000000A
:1028C000C0CB040800000000000000000000000071
:1028D0000000000098C204080300000005F303088C
:1028E000D81E002000000000D4CB04080300000024
:1028F00005F30308C009002000000000DCCB040839
:102900000300000005F30308CC1E002000000000B7
:10291000E4CB04080300000005F30308C01E0020F8
:1029200000000000D0C30408010000000000000007
:102930000000000000000000000000000E00000089
:10294000000000000000000000000000F0CB0408C0
:102950000000000000000000000000000000000077
:10296000FCCB04080700000061E90308341F0020C5
:102970000000000058C804080300000005F3030825
:10298000281F00200000000008CC040803000000FD
:1029900005F303081C1F00200000000010CC0408F1
:1029A0000300000005F30308101F002000000000D2
:1029B00018CC04080700000045E90308081F0020A0
:1029C00000000000D08704080300000005F303089E
:1029D000FC1E00200000000024CC040803000000BE
:1029E00005F30308F01E00200000000030CC0408AE
:1029F0000300000005F30308E41E002000000000AF
:102A0000D0C3040801000000000000000000000026
:102A100000000000000000000E00000000000000A8
:102A20000000000000000000C1E103087DE1030890
:102A30003C1F002059E4030800000000F01F0020A4
:102A400071E0030855E003087C200020000000002E
:102A5000000000003021002031E403087DE9030874
:102A6000BC2100203CCC0408000000000000000055
:102A7000000000000000000000B90408030000008E
:102A800005F30308C82200200000000048CC040819
:102A90000300000005F30308BC2200200000000032
:102AA000A4AE04080300000005F30308B0220020D0
:102AB0000000000054CC04080300000005F30308E4
:102AC000A42200200000000060CC040803000000E5
:102AD00005F30308982200200000000068CC0408D9
:102AE000020000001DF203080000000000000000CA
:102AF00070CC0408020000001DF203080100000071
:102B0000000000007CCC0408020000001DF2030855
:102B10000200000000000000000000000E000000A5
:102B2000000000000000000000000000685E0C00D3
:102B3000010000005001000007000000020000003A
:102B4000B42300200000000000000000000000008E
:102B50000000000000000000000000000000000075
:102B60000000000000000000000000000000000065
:102B70000000000000000000000000000000000055
:102B80000000000000000000000000000000000045
:102B90000000000000000000000000000000000035
:102BA00000000000430000000000000000000000E2
:102BB0000000000000000000000000000000000015
:102BC00000000000430000000000000000000000C2
:102BD00000000000000000000000000000000000F5
:102BE00000000000430000000000000000000000A2
:102BF00000000000000000000000000000000000D5
:102C00000000000043000000000000000000000081
:102C100000000000000000000000000000000000B4
:102C20000000000043000000000000000000000061
:102C30000000000000000000000000000000000094
:102C40000000000043000000000000000000000041
:102C50000000000000000000000000000000000074
:102C60000000000043000000000000000000000021
:102C70000000000000000000000000000000000054
:102C8000000000003B390408173904080000000068
:102C90008ECC040852C50408228E0408228E040833
:102CA000228E0408228E0408228E0408228E040834
:102CB000228E0408228E0408228E0408FFFFFFFFE4
:102CC000FFFFFFFFFFFFFFFFFFFF00000100415379
:102CD000434949000000000000000000000000001F
:102CE0000000000000000000000000000000415350
:102CF00043494900000000000000000000000000FF
:102D000000000000000000000000000000000000C3
:042D100001000000BE
:108000000B4B002210B4027203F59C74032102E0B2
:10801000072A09DC9979890702D519798154013237
:108020009C4203F11803F3D15DF8044B704700BF85
:10803000F47D04082E230370704700BF30B4012381
:108040000225322431211022057244704171C27020
:1080500003700371837030BC704700BF2322032379
:1080600002704370704700BF2DE9F0410B78047B2C
:10807000DB43DEB200F1100200F1380342F8044F96
:108080009342FBD1DFF89CC000F16001002243F86D
:10809000042F8B42FBD14FF0140E0521002546FA28
:1080A00001F303F00103002B1D4414BF4FF0190826
:1080B0004FF00A0811F0010FEDB214BF2746002758
:1080C00000220EEB02039BB200EB83030132424518
:1080D0005F61F6D1013A92B2013201390EEB02032F
:1080E0004A1C9BB201D09E46D9E715F0010F14BF80
:1080F00019250A2500215A1892B200EB820201319B
:10810000A9425461F7D10B449BB21A1D00EB8202C5
:10811000013300219BB25160ACF800300361BDE82F
:10812000F08100BF88250020254B5B880B332DE9AB
:10813000F04F8A4601F1060B1FFA83F94FF0010850
:10814000002100271AF801EB3E464C460122A4F11B
:108150000B039BB207E001339BB2B0F80CC0C5F82B
:1081600014C09C420AD000EB8305002AF3D100EB37
:10817000830501339BB29C426A61F4D1231D00EB5D
:1081800083030136092FF6B259600CD0092E14D0A2
:1081900008FA07F313EA0E0F14BF012200220C3471
:1081A000A4B20137D3E709F17809DA451FFA89F952
:1081B000C7D1034B5980BDE8F08F0022EFE700BF25
:1081C000882500202DE9F047DFF85C80B8F80430FE
:1081D00004338A461FFA83FC01F109094FF0010EAE
:1081E0001AF8017B64460026231F0EFA06F29BB2A2
:1081F0003A40BAB1818900EB830501339BB29C42BE
:108200006961F6D101360434082EA4B2ECD10CF128
:10821000200CCA451FFA8CFCE2D10023A8F80430D8
:10822000BDE8F0871146E6E78825002010B5027BFF
:1082300001681F2A4FF020030ED94C68203A934062
:108240001C4216D00B4A406800241470026822F0C9
:1082500001020260CB6010BD0C6893401C4208D044
:10826000044A406800241470026822F0010202608F
:108270008B6010BD71310020436A8269D154436A1A
:108280000169826B01338B4228BF00234362002ABD
:108290002FD0EFF31182502383F31288836B196878
:1082A000C9072CD470B45E686EB9456A816A8D4284
:1082B00017D084690C44DC600ED9691A5960856254
:1082C000002180F85C10196841F00101D2B21960F8
:1082D00082F3118870BC70470469611A5960866224
:1082E000EEE7012380F85C30D2B282F3118870BCD3
:1082F0007047826DD36843F08003D3607047D2B279
:1083000082F31188704700BF426B10B462B1C36C36
:10831000C2684469D11A013B615C5DF8044B08BF37
:108320001346C364C8B27047016A4369C4685B5CA2
:108330000131A14228BF114601625DF8044BD8B259
:10834000704700BF836B13B190F85C007047836A7D
:10835000406A181AB0FA80F040097047416A836A8F
:1083600099420AD3CB1A816B026961B14968501EE8
:108370000B4483420AD2C01A704702691144CB1AD7
:10838000816B0029F2D1501EC01A7047002070473F
:10839000436B43B1C26C5B6893422FBF981AC068AD
:1083A0009B1AC0187047C269036A9A422FBFD01A3D
:1083B000C0688018C01A70470A4B30B503F1140426
:1083C00093F900205D78072AC8BF143A8118043356
:1083D0000D7313F8025C855413F8012C0A76A3423E
:1083E000EED130BD784B040803682DE9F041DF6918
:1083F0001FB13B46BDE8F0411847002A164611DD83
:1084000004460D460E4400E023689B6820469847CA
:108410000028F9D0236815F8011B1B6820469847EF
:10842000AE42F1D1BDE8F0810023252202704370F5
:108430008370C370704700BF038A2DE9F0478589B8
:10844000ADB21D4029D00F4606464FF000484FF010
:108450000009B5FA85F328FA03F2D24391B21B3B27
:1084600015403182042B16D8DFE803F03129211999
:1084700003007B6A002B32D003F1FF3A1FFA8AFA1D
:10848000C7F824903C6A34B1236820465146984787
:108490006468002CF8D1002DDBD1BDE8F087386886
:1084A000716B036889B29847002DD2D1F5E77868DF
:1084B000B16B036889B29847002DCAD1EDE7B8685F
:1084C000F16B036889B29847002DC2D1E5E7F868DF
:1084D000316C036889B29847002DBAD1DDE7F36AA1
:1084E0001FFA83FACEE700BF30B50446806D617194
:1084F0008389A26823F400531B041B0C838185B07D
:10850000A379009213F0040230D04FF4805213F09C
:108510000203ADF8042056D1ADF806304FF4806365
:108520000022ADF8083011F00103ADF80C2028D17D
:10853000ADF80A3008238D07694648BFADF80A3008
:1085400022F044FBA279A36DD10724D412F0080FC6
:108550009A8A1BD122F008021204120C9A829A897C
:1085600092B242F400529A8105B030BD13F002037A
:10857000ADF8042024D04FF400551346ADF8065052
:10858000CEE70423ADF80A300C23D4E792B242F0D0
:1085900008029A82E3E70D498B420FD0A1F54841CA
:1085A0008B4209D00A498B42D0D10520012139F0F4
:1085B000B1FFA279A36DC9E70220F7E70020F5E734
:1085C000ADF80630ACE74FF40053A5E700100140CA
:1085D0000014014010B50446806DA160838923F426
:1085E00000531B041B0C8381A37984B013F0040295
:1085F000009135D04FF4805213F00203ADF80420FF
:1086000056D1ADF806304FF480636279ADF808308A
:10861000D1074FF00003ADF80A30ADF80C3045BF7C
:108620000423ADF80A3008230C236946920748BF9B
:10863000ADF80A3022F0CAFAA279A36DD1071FD48F
:1086400012F0080F9A8A16D122F008021204120CB6
:108650009A829A8992B242F400529A8104B010BD73
:1086600013F00203ADF804201FD04FF4005113465D
:10867000ADF80610C9E792B242F008029A82E8E724
:108680000D498B420FD0A1F548418B4209D00B49CF
:108690008B42D5D10520012139F03CFFA279A36D91
:1086A000CEE70220F7E70020F5E7ADF80630ACE7AB
:1086B0004FF40053A5E700BF001001400014014033
:1086C0002DE98048013085B0C3B203938B4D8C4FA8
:1086D0008C4C8D4E0A2302933220DFF830922DF01D
:1086E0002DFE4FF4FA7A4FF0100C4FF47A70D9F84F
:1086F0000430C3F30803002B40F0C180EFF3118373
:10870000002B40F0BC802968A26800BF2B6899420A
:10871000F9D1D7F800E000FB0EF39B1AB3FBFEF390
:1087200000FB01314FF0010E0191D9F80430C3F381
:108730000803002B40F08780EFF31183002B40F0FB
:1087400082802B68A16800BF2A689342F9D1D7F8CC
:1087500000B000FB0BF2521AB2FBFBF200FB03234A
:10876000019A9B1AB3F57A7FDFD3BAF1010ABED121
:10877000039B002B40F0BD804FF47A7ADFF88C9198
:1087800050464FF0100CD9F80430C3F30803002B07
:1087900040F09280EFF31183002B40F08D80296828
:1087A000A26800BF2B689942F9D1D7F800E000FB1E
:1087B0000EF39B1AB3FBFEF300FB01314FF0010EE9
:1087C0000191D9F80430C3F3080303BBEFF311831D
:1087D000EBB92B68A16800BF2A689342F9D1D7F89A
:1087E00000B000FB0BF2521AB2FBFBF200FB0323BA
:1087F000019A9B1AB3F57A7FE3D3BAF1010AC2D189
:10880000029B013B02937FF467AF39F0CDFEEFF39B
:1088100011888CF31288A1682368DB0344BFC6F873
:1088200000E0A1682B6832685FFA88F888F3118845
:10883000D7F800801A4400FB08F35B1AB3FBF8F387
:1088400000FB0233D4E7EFF311888CF31288A168A0
:108850002368DB0344BFC6F800E0A1682B683268D8
:108860005FFA88F888F31188D7F800801A4400FB73
:1088700008F35B1AB3FBF8F300FB023370E7EFF386
:1088800011828CF31288D4F808E02368D90303D549
:1088900001233360D4F808E02B683168D2B282F348
:1088A00011883A68194400FB02F3A3EB0E03B3FBF3
:1088B000F2F300FB013135E7EFF311828CF31288FC
:1088C000D4F808E02368D90303D501233360D4F832
:1088D00008E02B683168D2B282F311883A681944F3
:1088E00000FB02F3A3EB0E03B3FBF2F300FB013139
:1088F00064E718462DF084FB3EE700BF9C92002001
:10890000A092002010E000E09892002000ED00E02E
:1089100038B5484B5A899989914224BF00225A811F
:10892000198ADA89914224BF0022DA81DA78CAB141
:10893000072A41496AD091F85300404D0124002193
:108940000A282C709C70D9715DD00C2807D0002AA1
:108950006CD0DFED3B7A072A0ED00A2862D0DFED1B
:10896000397A09E0344A92F853000A2856D00C2884
:108970005BD1D979DFED347A344C9FED350AA2789A
:10898000002918BFF0EE407A062A04D8314901EBDD
:10899000820191ED050A217979B1013A032A0BD8B8
:1089A000F7EE007A87EE800A3BF0BAF82388984207
:1089B00028BF1846208038BD38BD9B781F4A07EE77
:1089C000103A1178B8EEC77A67EE277A07EE101AD8
:1089D000B8EEC77A27EE277AB4EEC70AF1EE10FA9E
:1089E000EADD80EE277AFDEEC77A17EE903A102B7B
:1089F000A8BF1023012BB8BF0123DBB28B4238BFC5
:108A00000B46137038BDDFED147AA4E791F85300DC
:108A10000A2803D00C28ACD0D9799AE7D979DFEDB0
:108A20000E7AA9E7DFED0D7AA6E7D979DFED047AB2
:108A3000A2E700BFE07C0020F47C002064950020C9
:108A40006F1203396F12833A0AD7A3398458002072
:108A50006F120338784B04085304E9380F506E3A0C
:108A60002DE9F047A64FA74E18F022FBBE421ED2BA
:108A7000DFF81483DFF814934446258862197DB12A
:108A80004A450DD2052D0BD933886188C3F30B03FA
:108A9000994200F0D880144625886219002DEFD144
:108AA00071683046143610F0FDFDBE42E4D3964A9C
:108AB0001378A3F1170102290FD9944911F8330053
:108AC000002840F0EF80D8000144497829B190494E
:108AD00011F833300BB9182313708E4B5A78022AD1
:108AE00000F2D1808C498D4802EB420201EB8201F9
:108AF0001A780160022A00F2CF8002EB8201884BD3
:108B0000C2EBC10203EB4203998C5A8C854C914213
:108B1000236001D300225A84834B9A78042A00F000
:108B2000E28032B91A88B2F5F07F84BF4FF4F07258
:108B30001A807E4DFFF7ECFE2B687D4A1A40002A12
:108B400000F0DA80D80700F1C980590400F1C18033
:108B50001A0700F1B0809B0400F1B48026F032F8CF
:108B600010B9744834F04AFA4FF0007010F0D0FD9C
:108B70004FF0806010F0CCFD2BF090FB00213022F4
:108B80006D483BF08AFF20682AF0D8FA6B4B2568C5
:108B900003F1500103E00433994200F081801A7818
:108BA000002AF8D19C78D8788442F4D26449654B85
:108BB0000A7028461D6020F0E3FD634A634910797E
:108BC000634A644B1160C822642111FB002100221A
:108BD00059609A60DA601A615A619A61DA6183F8C1
:108BE000202083F821201DF02DF95B4B9FED5B5A6F
:108BF0001B885B4A9FED5B6A55795B4C5B495C481F
:108C0000086006EE903AF8EEE66A1388C5EE265A3A
:108C100007EE103A53881279C4ED005A07EE903AE5
:108C2000B8EEC77A534BF8EEE77A1D725A7227EE08
:108C3000067A67EE867ABDE8F04783ED017AC3EDE8
:108C4000007A18F01DBA63799B077FF424AF71682E
:108C500094F804A0304610F025FD3388BAEB133F9A
:108C600004D01436BE42FFF407AF20E77388706863
:108C7000AA1FC3F30B039A4204F10601A8BF1A46C8
:108C80003AF078FDEDE700225A701A78234822491D
:108C90000160022A7FF631AF00221A70204B33E7C1
:108CA000012283E7D8000C186468002C7FF40CAF15
:108CB0001724147008E7304810F02AFD2B689B0435
:108CC0007FF54CAF2D4810F023FD402010F020FD23
:108CD00044E72B4810F01CFD2B6839E7294810F0B9
:108CE00017FD2B6831E79A8AB2F57A7FBFF421AF7E
:108CF0004FF47A729A821CE743F008032B6021E755
:108D00009006000890010008A09500200C7404084B
:108D1000E07B0408FC7B00206C5100205C560020A6
:108D2000F8BF0020585600208458002028C1002099
:108D30000960000254700020AC2A0020F04400209A
:108D4000A0230020E02A00201C8F00207695002020
:108D5000E82A002098970020FC2F0020C0C9FB487B
:108D6000EC29002017B7D138003000208889002076
:108D70003661023D64890020016000020940000262
:108D8000092000020860000202400008008000087C
:108D900038B50E4C0E4DAC4206D2616820461434F4
:108DA00010F080FCAC42F8D30A4A0B4B0B4C0C4D34
:108DB0001560022500220B4925701A705A700A4866
:108DC0000860BDE8384027F05FBF00BF9001000891
:108DD0009006000858560020FC7B0020D49200200A
:108DE000F8BF00205C5600206C510020054B10B5E8
:108DF0009A68054C2178501C09B99A6010BD02464A
:108E0000F8E700BF8825002071310020F0B50C295B
:108E100034D8DFE801F0893333335E33333334330E
:108E200033330700048C9689B2F802E01788734D3B
:108E300024F480542404240C0484038C8488818BBF
:108E400023F4005321F4E6411B0409041B0C46EAF9
:108E50000E06090C43EA063341EA0721A8429BB2F9
:108E6000A4B289B200F09E8005F58065A84200F0AA
:108E7000998092688480818302640384F0BD048CAD
:108E80009589B2F802C0B2F800E05C4F24F4807417
:108E90002404240C0484038C8688818B23F40073BF
:108EA0001B0421F073011B0C45EA0C04090443EA7E
:108EB0000423090CB8429BB2B6B241EA0E015CD061
:108EC0004F4CA04259D0926886808183C26303844C
:108ED000F0BD048C9589B2F802C0B2F800E0474EAC
:108EE00024F010042404240C0484038C8788018B50
:108EF00023F0200321F4E6411B0409041B0C45EA7E
:108F00000C04090C43EA041341EA0E21B0429BB25F
:108F1000BFB289B25DD03A4CA0425AD092688780E5
:108F2000018382630384F0BD048C9789B2F802E068
:108F30001688324D24F001042404240C0484038C8C
:108F40008488018B23F002031B0421F073011B0CA6
:108F500047EA0E0709043B43090CA8429BB2A4B29E
:108F600041EA060125D005F58065A84221D0926826
:108F70008480018342630384F0BDD589148A578AB3
:108F800023F4006343EA05254FF6FF332B40958811
:108F900026F440563C4343EA052346EA04169BB2B6
:108FA000B6B290E7158A24F4804444EA8514A4B24A
:108FB0005FE7D689158A578A23F00803334324F4E0
:108FC000407496883D4323F004032C433343A4B2FA
:108FD000CDE7D489158A568A23F0800343EA041327
:108FE0004FF6BF741C40938827F44067354344EA2A
:108FF000031347EA85079BB2BFB28FE70000014029
:10900000000401402DE9F84F4FF4A072002191486F
:10901000914CDFF86892914D914E924FDFF860824B
:109020003BF03BFD90489149DFF858E2DFF858C229
:1090300000221359834200F0E980B3F1804F00F021
:10904000E780AB4200F0F280B34200F0F180BB4217
:1090500000F0F080734500F0EF80634500F0EE8093
:10906000434500F0ED80DFF824A2534500F0EA808C
:109070000AF5806A534500F0E7800AF5806A534597
:1090800000F0E480AAF5983A534500F0E1800AF533
:10909000806A534500F097800AF5806A534508BFFF
:1090A0000D2300F091801832B2F5A87FC1D16A4E2D
:1090B000DFF8DCA106F5A8774FF003094FF00208AE
:1090C00003E01836B74200F09F80B379002BF8D048
:1090D00033791C09013C032C03F00F03F1D8644AD7
:1090E00032F8140040FA03F2D207EAD5012505FA56
:1090F00003F3013B18403AF0F9F85E4B1B5D18444E
:109100001AEBC002DDD05AF830305B4C317A03F1F3
:109110003F4000F57E00800A205C00F01F044009FB
:10912000032805FA04F57BD0042873D0022804D163
:109130004E48406C05434D484564B2F804E0BEFA21
:109140008EF2C2F11F0292B2D00803EB800002F04F
:109150000702046A92000F25954024EA0504046280
:10916000046A01FA02F22243002502624FF0010C68
:109170002A4603E0102A05F10205A2D00CFA02F0FB
:1091800030EA0E0102F10102F4D11C6809FA05F17E
:10919000C9430C401C60D3F800B008FA05F444EA57
:1091A0000B041C609C680C409C609C689C605C6824
:1091B00024EA0000586058685860D8680140D960B7
:1091C000D968D960D6E70C2309EBC3034FF0010A35
:1091D0001B7903F01F0B5B09032B0AFA0BFA09D06A
:1091E000042B0CD0022B7FF45EAF4B6C4AEA0303D6
:1091F0004B6458E70B6C4AEA03030B6453E70B6BB1
:109200004AEA03030B634EE7BDE8F88F0023DBE770
:109210000123D9E71548006B0543144805638CE723
:109220001248006C05431148056486E70223CBE72A
:109230000323C9E70423C7E70523C5E70623C3E7DC
:109240000723C1E70823BFE70923BDE70A23BBE7DC
:109250000B23B9E7F4680020F47D04080004004003
:1092600000080040000C00400000014000380240AF
:10927000487F0408447F0408BC7D04089C730408EC
:109280000004014000100040001400400040014074
:109290000C91002000286AD003682DE9F04F03F1FB
:1092A0003F4404F57E045F4EA40A0125345D04F0BA
:1092B0001F066409032C05FA06F559D0042C00F0AA
:1092C000AC80022C59D08588B5FA85F0C0F11F001A
:1092D00080B2C40803EB840400F00700266A800013
:1092E0000F27874026EA07062662276A01F0030651
:1092F0008240701E3A430128C1F3810CC1F300186B
:109300002262C1F341113DD90024224601274FF0CA
:10931000030E03E0102A04F1020426D007FA02F03B
:10932000A84302F10102F5D1D3F800C00EFA04F00F
:10933000C04300EA0C0CC3F800C0D3F8008006FA62
:1093400004FC4CEA080CC3F800C0D3F80CC000EAD7
:109350000C00D860D3F80CC001FA04F040EA0C000D
:10936000102AD86004F10204D8D1BDE8F08F70470C
:109370002D4C266C35432564A5E72B4C666C354394
:109380006564A0E7002002464FF0010E4FF003098C
:1093900004E00132102A00F102003CD00EFA02F77C
:1093A00037EA0504F5D1D3F800A009FA00F4E44344
:1093B0000AEA040AC3F800A0D3F800B006FA00FADB
:1093C0004AEA0B0AC3F800A0D3F808A004EA0A0A84
:1093D000C3F808A0D3F808B00CFA00FA4AEA0B0A5E
:1093E000C3F808A0D3F804A02AEA07075F60D3F8FF
:1093F00004A008FA02F747EA0A075F60DF683C400A
:10940000DC60DF6801FA00F401323C43102ADC60C2
:1094100000F10200C2D1BDE8F08F034C266B35434A
:10942000256350E7BC7D04080038024003682DE93D
:10943000F04F03F13F4404F57E04604EA40A012579
:10944000345D04F01F066409032C05FA06F500F0EC
:10945000AF80042C00F0A780022C54D08588B5FA88
:1094600085F0C0F11F0080B2C40803EB840400F053
:109470000700266A80000F27874026EA0706266233
:10948000276A01F0030602FA00F0721E3843012A2F
:10949000C1F3810CC1F300182062C1F3411137D927
:1094A0000024224601274FF0030E03E0102A04F1A6
:1094B000020426D007FA02F0A84302F10102F5D116
:1094C000D3F800C00EFA04F0C04300EA0C0CC3F855
:1094D00000C0D3F8008006FA04FC4CEA080CC3F87C
:1094E00000C0D3F80CC000EA0C00D860D3F80CC060
:1094F00001FA04F040EA0C00102AD86004F10204DA
:10950000D8D1BDE8F08F2E4C666C35436564A5E775
:10951000002002464FF0010E4FF0030904E0013233
:10952000102A00F102003CD00EFA02F737EA0504D7
:10953000F5D1D3F800A009FA00F4E4430AEA040ADA
:10954000C3F800A0D3F800B006FA00FA4AEA0B0A02
:10955000C3F800A0D3F808A004EA0A0AC3F808A0D8
:10956000D3F808B00CFA00FA4AEA0B0AC3F808A0CC
:10957000D3F804A02AEA07075F60D3F804A008FA2A
:1095800002F747EA0A075F60DF683C40DC60DF689B
:1095900001FA00F401323C43102ADC6000F10200C1
:1095A000C2D1BDE8F08F064C266B3543256355E7E5
:1095B000034C266C3543256450E700BFBC7D04088E
:1095C0000038024010B50409013C032C17D80D4B9C
:1095D00033F8142000F00F0042FA00F313F00103F7
:1095E0000DD0012303FA00F00138104039F07EFE5F
:1095F000054A064B125D104403EBC00010BD00206D
:1096000010BD00BF487F0408447F04080C9100206F
:1096100001490248FEF710BF0C6A00200018004004
:1096200001490248FEF708BFE469002000400140FC
:1096300001490248FEF700BFBC6900200004014058
:1096400001490248FEF7F8BEBC6900200004014051
:1096500001490248FEF7F0BE94690020000C00406A
:1096600001490248FEF7E8BE6C690020000800408E
:1096700001490248FEF7E0BE4469002000040040B2
:1096800002494FF08040FEF7D7BE00BF1C690020A2
:1096900001490248FEF7D0BEF468002000000140F6
:1096A00001490248FEF7C8BEF468002000000140EE
:1096B000F0B50468A30AA3F58013502B2AD8DFE87D
:1096C00003F02A7A8E9229297E29292929292929F4
:1096D00029292929292929292929292929292929FA
:1096E00029292929292929292929292929292929EA
:1096F00029292929292929292929292929292929DA
:109700002929828629292929292929292929292913
:1097100029298A00F0BD4FF0480E01264779B00094
:109720004FEA970C00296BD063460227A5899F401A
:1097300083190CEB43032F4303F1040C3A4DBFB2E2
:1097400045F8231045F82C20A781EFF31181502212
:1097500082F31288821905EBC2021369002B46D0EE
:1097600013620433821905EBC202576917B11F60F7
:1097700053690433821905EBC202976917B11F6060
:1097800093690433821905EBC202D76917B11F60D0
:10979000D36904330027CAB21F6082F311883044B2
:1097A00005EBC000036A2BBBA38923F001031B0454
:1097B0001B0CA381F0BD4FF0700E0226AEE74FF4F4
:1097C0009C7E0726AAE74FF0200E0026A6E74FF062
:1097D000E80E0526A2E74FF4887E06269EE74FF0A6
:1097E000980E03269AE74FF0C00E042696E705EB85
:1097F0000E03B7E7A3899BB243F00103A381F0BD39
:109800000223BF0803FA07F7A389074D9BB223EA97
:10981000070387190CEB470CA3810CF1040345F8EF
:109820002C1045F8232090E7F468002010B5036859
:1098300082480139834282B089B200F0CA80A0F523
:109840008060834200F0C58000F58040834200F0D4
:10985000B78000F58060834200F0B28000F5806040
:10986000834200F0AD80764C188824686408B4FB0D
:10987000F2F4013CA4B282B2B3F1804F0AD0714835
:10988000834207D000F58060834203D000F58060FA
:10989000834202D122F0700292B26B48834200F000
:1098A000A18000F58060834200F0A68022F440721F
:1098B00000F56C4092B283421A80D9621C854FD069
:1098C0005E4A93424CD001229A821A8892B242F0A8
:1098D00001021A80B3F1804F00F09880594A9342F8
:1098E00000F0968002F58062934200F0938002F5CA
:1098F0008062934200F0908002F58062934200F013
:109900008D8002F58062934200F08A8002F57042F9
:10991000934200F0878002F57052934200F08480F9
:1099200002F58062934200F0818002F580629342EA
:109930007ED0A2F5983293427CD002F580629342A9
:109940007AD002F58062934208BF0D2215D002A89A
:109950004FF0012340F8043D21F0A2F802B010BD01
:109960000122002119869A821A88384892B242F060
:10997000010283421A80ADD10A46354B03EBC20384
:1099800001A85C798DF80440012300228DF8053090
:109990008DF807308DF8062021F082F81B2C08D0B6
:1099A0002E2CDBD12B4B019301A821F079F802B0CA
:1099B00010BD294B019301A821F072F802B010BD2F
:1099C0001F4C18882468B4FBF2F4013CA4B282B2A4
:1099D00052E71B4C18882468B4FBF2F4013CA4B293
:1099E00082B257E701201A80D9621C8598821A88B2
:1099F00092B202431A8071E701201A80D9621C8555
:109A000098821A8892B202431A8063E70122B4E76F
:109A10000222B2E70322B0E70422AEE70522ACE758
:109A20000622AAE70722A8E70822A6E70922A4E758
:109A30000A22A2E70B22A0E70C229EE700040140C5
:109A4000DC7C0020000400400010004000000140C9
:109A50009C7304082C010001190100012B4B984252
:109A60003CD0B0F1804F3BD0A3F57C43984239D035
:109A700003F58063984237D003F58063984235D070
:109A800003F58063984233D003F58063984231D068
:109A900003F5704398422FD003F5705398422DD0B0
:109AA00003F5806398422BD003F58063984229D058
:109AB000A3F59833984227D003F58063984207D0E6
:109AC00003F58063984208BF0D2202D00020704742
:109AD0000C220F4B03EBC203187970470022F8E702
:109AE0000122F6E70222F4E70322F2E70422F0E77C
:109AF0000522EEE70622ECE70722EAE70822E8E77C
:109B00000922E6E70A22E4E70B22E2E7000001402F
:109B10009C7304082DE9F04F013085B0C3B2039364
:109B20000B4602918B4C8C4E002B00F09A80322019
:109B30008A4D8B4FDFF82C922CF000FC4FF4FA7A10
:109B40004FF0100C4FF47A70D9F80430C3F30803C7
:109B5000002B40F0DE80EFF31183002B40F0D98022
:109B60002968A26800BF2B689942F9D1D7F800E0B4
:109B700000FB0EF39B1AB3FBFEF300FB01314FF029
:109B8000010E0191D9F80430C3F30803002B40F013
:109B90008780EFF31183002B40F082802B68A1684F
:109BA00000BF2A689342F9D1D7F800B000FB0BF24E
:109BB000521AB2FBFBF200FB0323019A9B1AB3F586
:109BC0007A7FDFD3BAF1010ABED1039B002B40F0AC
:109BD000BD804FF47A7ADFF88C9150464FF0100C2C
:109BE000D9F80430C3F30803002B75D1EFF31183C8
:109BF000002B71D12968A26800BF2B689942F9D166
:109C0000D7F800E000FB0EF39B1AB3FBFEF300FB5A
:109C100001314FF0010E0191D9F80430C3F308036C
:109C200013BBEFF31183FBB92B68A16800BF2A684F
:109C30009342F9D1D7F800B000FB0BF2521AB2FBF5
:109C4000FBF200FB0323019A9B1AB3F57A7FE3D35F
:109C5000BAF1010AC4D1029B013B0293002B7FF4AD
:109C600066AF05B0BDE8F08FEFF311888CF3128872
:109C7000A1682368DB0344BFC6F800E0A1682B6835
:109C800032685FFA88F888F31188D7F800801A44A0
:109C900000FB08F35B1AB3FBF8F300FB0233D2E7D7
:109CA000EFF311888CF31288A1682368DB0344BFAB
:109CB000C6F800E0A1682B6832685FFA88F888F37C
:109CC0001188D7F800801A4400FB08F35B1AB3FB35
:109CD000F8F300FB023370E7EFF311828CF3128884
:109CE000D4F808E02368D90303D501233360D4F8FE
:109CF00008E02B683168D2B282F311883A681944BF
:109D000000FB02F3A3EB0E03B3FBF2F300FB013104
:109D10007FE7EFF311828CF31288D4F808E0236810
:109D2000D90303D501233360D4F808E02B683168E8
:109D3000D2B282F311883A68194400FB02F3A3EB14
:109D40000E03B3FBF2F300FB013118E718462CF0C9
:109D500057F93EE710E000E0989200209C92002026
:109D6000A092002000ED00E0204B5B68C3F30803E5
:109D700030B4BBB9EFF31183A3B91D4B1D4C186868
:109D8000A16800BF1A689042F9D11B4B1C684FF4C0
:109D90007A7202FB04F3591AB1FBF4F130BC02FBF6
:109DA00000107047EFF31182102383F312881149DA
:109DB0008C680B6813F4803F104B02D001201860B0
:109DC0008C680B49D2B20D68186882F311880A4B6F
:109DD00019684FF47A72284402FB01F31B1B30BC54
:109DE000B3FBF1F302FB0030704700BF00ED00E071
:109DF0009C92002010E000E0A092002098920020A9
:109E00002DE9F84F8046FFF7AFFF254E2549DFF8D3
:109E1000A0E0254A254D844610274FF47A7401208E
:109E2000DEF80430C3F30803D3B9EFF31183BBB9F1
:109E30000B68D2F808A000BFD1F800904B45F7D1CD
:109E4000D6F800B004FB0BF9A9EB0A09B9FBFBF942
:109E500004FB0393A3EB0C034345E1D3BDE8F88F68
:109E6000EFF3118A87F31288D2F808B01368DB0386
:109E700044BF2860D2F808B00B68D5F800905FFAAC
:109E80008AFA8AF31188D6F800A0994404FB0AF3F1
:109E9000A3EB0B03B3FBFAF304FB0933DAE700BFD0
:109EA000A09200209C92002010E000E098920020F8
:109EB00000ED00E02DE9F04FDFF830C1474A484996
:109EC000484E494D8046102718F1FF38C0F0848075
:109ED000DCF80430C3F30803002B5CD1EFF31183EB
:109EE000002B58D10B68946800BF08688342F9D1F1
:109EF000D6F800904FF47A7000FB09FEAEEB040E2A
:109F0000BEFBF9FE00FB03EEDCF80430C3F30803EC
:109F10004FF47A740120FBB9EFF31183E3B90B68B6
:109F2000D2F808A000BFD1F800904B45F7D1D6F881
:109F300000B004FB0BF9A9EB0A09B9FBFBF904FB20
:109F40000393A3EB0E03B3F57A7FBDD2DCF80430A4
:109F5000C3F30803002BDFD0EFF3118A87F31288D5
:109F6000D2F808B01368DB0344BF2860D2F808B009
:109F70000B68D5F800905FFA8AFA8AF31188D6F850
:109F800000A0994404FB0AF3A3EB0B03B3FBFAF321
:109F900004FB0933D5E7EFF3118487F31288D2F875
:109FA00008901368D80303D501232B60D2F80890DA
:109FB0000B682868E4B284F31188D6F800A04FF447
:109FC0007A7400EB030E04FB0AF3A3EB0903B3FB63
:109FD000FAF304FB0E3E97E7BDE8F08F10E000E0D7
:109FE0009C920020A09200209892002000ED00E0BA
:109FF00030B4EFF31183102282F312880649074C24
:10A000000A680748013200250A602560DBB2026851
:10A0100083F3118830BC70479C92002098920020F6
:10A0200010E000E00F4B1B88014643B90E4B0F4A6E
:10A030001B7810680BB981F001010EF081BF0C4B49
:10A040005A691AB118B91A68106058747047094AE9
:10A0500018681188084A92FBF1F2012102605974D4
:10A06000704700BF74920020769200207892002002
:10A070007C9200209492002020A1070038B5264B46
:10A080005C69636B73B1A36DA26BD2B1998A1A88B4
:10A09000C90592B201D5D20700D438BD4FF6F77288
:10A0A0001A8038BDA36D99891A88890692B2EBD5BA
:10A0B0009206E9D5E26AD2B19888216B80B29047C6
:10A0C000E1E799891A880D0692B2DFD51006DDD531
:10A0D000A26A616A8A4219D0A1692569885C988060
:10A0E0000132B2FBF5F105FB1122A262CEE79B889B
:10A0F000E2696169DBB28B54E269E068A36D013209
:10A10000B2FBF0F100FB1122E261BDE7DA6822F058
:10A110008002DA60BAE700BF403F002038B5264B26
:10A120009C68636B73B1A36DA26BD2B1998A1A88D4
:10A13000C90592B201D5D20700D438BD4FF6F772E7
:10A140001A8038BDA36D99891A88890692B2EBD519
:10A150009206E9D5E26AD2B19888216B80B2904725
:10A16000E1E799891A880D0692B2DFD51006DDD590
:10A17000A26A616A8A4219D0A1692569885C9880BF
:10A180000132B2FBF5F105FB1122A262CEE79B88FA
:10A19000E2696169DBB28B54E269E068A36D013268
:10A1A000B2FBF0F100FB1122E261BDE7DA6822F0B8
:10A1B0008002DA60BAE700BF403F002038B5264B86
:10A1C0001C68636B73B1A36DA26BD2B1998A1A88B4
:10A1D000C90592B201D5D20700D438BD4FF6F77247
:10A1E0001A8038BDA36D99891A88890692B2EBD579
:10A1F0009206E9D5E26AD2B19888216B80B2904785
:10A20000E1E799891A880D0692B2DFD51006DDD5EF
:10A21000A26A616A8A4219D0A1692569885C98801E
:10A220000132B2FBF5F105FB1122A262CEE79B8859
:10A23000E2696169DBB28B54E269E068A36D0132C7
:10A24000B2FBF0F100FB1122E261BDE7DA6822F017
:10A250008002DA60BAE700BF403F002070B4EFF33D
:10A260001186502383F31288836B1A68D20720D497
:10A270005D686DB9446A826A944217D0816911445D
:10A28000D9600ED9A21A5A608462002280F85C203C
:10A290001A6842F00102F1B21A6081F3118870BCB1
:10A2A000704701698A1A5A608562EEE7012380F8D7
:10A2B0005C30F3B283F3118870BC704703685B6A4B
:10A2C00003B11847704700BF03681B6A03B1184702
:10A2D000704700BF03682DE9F041DF691FB13B46BD
:10A2E000BDE8F0411847002A164611DD04460D4628
:10A2F0000E4400E023689B68204698470028F9D068
:10A30000236815F8011B1B6820469847AE42F1D11F
:10A31000BDE8F08103689B69184700BF03685B696B
:10A32000184700BF03681B69184700BF0368DB6854
:10A33000184700BF03689B68184700BF03685B6845
:10A34000184700BF03681B68184700BF38B50C46A4
:10A35000097849B1054601342B6828461B6898479F
:10A3600014F8011B0029F7D138BD00BF10B40B4B06
:10A370000B4A1C7801238340234052F8200031B956
:10A38000B3FA83F149095DF8044B0EF0D9BD191CED
:10A3900018BF01215DF8044B0EF0D2BD649200207D
:10A3A00068920020064B53F820302BB11A689B8826
:10A3B00051690B4201D1138370475383704700BF2B
:10A3C00068920020026802F13F4303F57E032DE905
:10A3D000F04F9B0A544DEB5C03F01F055B09012411
:10A3E000032B04FA05F400F09980042B00F091800F
:10A3F000022B3ED001F00306731E012BC1F3810C2A
:10A40000C1F300188588C1F3411137D900242346D0
:10A4100001274FF0030E03E0102B04F1020426D0B5
:10A4200007FA03F0A84303F10103F5D1D2F800C005
:10A430000EFA04F0C04300EA0C0CC2F800C0D2F8D7
:10A44000008006FA04FC4CEA080CC2F800C0D2F8FE
:10A450000CC000EA0C00D060D2F80CC001FA04F085
:10A4600040EA0C00102BD06004F10204D8D1BDE802
:10A47000F08F2E4B5D6C2C435C64BBE700200346E1
:10A480004FF0010E4FF0030904E00133102B00F1EF
:10A4900002003CD00EFA03F737EA0504F5D1D2F8F2
:10A4A00000A009FA00F4E4430AEA040AC2F800A092
:10A4B000D2F800B006FA00FA4AEA0B0AC2F800A085
:10A4C000D2F808A004EA0A0AC2F808A0D2F808B034
:10A4D0000CFA00FA4AEA0B0AC2F808A0D2F804A063
:10A4E0002AEA07075760D2F804A008FA03F747EAF8
:10A4F0000A075760D7683C40D460D76801FA00F477
:10A5000001333C43102BD46000F10200C2D1BDE8FE
:10A51000F08F064B1D6B2C431C636BE7034B1D6CCC
:10A520002C431C6466E700BFBC7D04080038024071
:10A530002DE9F04F4A484B494B4B4C4C4FF0010A28
:10A540004FF002094FF004084FF0080C4FF0100EC6
:10A5500020274026802530F8022B12F0010F03D06F
:10A560001960A3F804A0083312F0020F03D0196099
:10A57000A3F80490083312F0040F03D01960A3F875
:10A580000480083312F0080F03D01960A3F804C048
:10A59000083312F0100F03D01960A3F804E0083359
:10A5A00012F0200F02D019609F80083312F0400F84
:10A5B00002D019609E80083312F0800F02D019601B
:10A5C0009D80083312F4807F05D04FF4807B1960A2
:10A5D000A3F804B0083312F4007F05D04FF4007BD9
:10A5E0001960A3F804B0083312F4806F05D04FF45B
:10A5F000806B1960A3F804B0083312F4006F05D023
:10A600004FF4006B1960A3F804B0083312F4805FB4
:10A6100005D04FF4805B1960A3F804B0083312F43E
:10A62000005F05D04FF4005B1960A3F804B0083355
:10A6300012F4804F05D04FF4804B1960A3F804B09A
:10A640000833D20B04D04FF4004219609A800833CB
:10A6500001F58061A1427FF47EAFBDE8F08F00BFBD
:10A66000487F0408000002400C91002000100240C6
:10A670002DE9F04F4FF4807385B043838383C38308
:10A6800000F10C0504463220FFF714FC11220021D2
:10A6900028460EF00FFF6022012128460EF00AFF27
:10A6A0006420FFF707FC02A92046002737F038FE98
:10A6B0000123B946B8463E460193012E14BF11222C
:10A6C0001222002128460EF0F5FE002E0CBF4FF09E
:10A6D000010B4FF0FF3B4FF00A0A012202212846EE
:10A6E0000EF0E8FE1420FFF7E5FB02A9204637F044
:10A6F00017FEBDF90A20BDF90C00BDF90810234B67
:10A7000082420BFB0299A8BF02468A42A8BF0A46B2
:10A710009A4201FB0B880BFB007733DB0120FFF72C
:10A7200041FEBAF1010AD8D10136022EC5D1184B2B
:10A7300093FBF8F893FBF9F97022A3F58423002129
:10A7400093FBF7F7A4F81A80A4F81C90E783284637
:10A750000EF0B0FE2022012128460EF0ABFE0022B2
:10A76000314628460EF0A6FE6420FFF7A3FB019BAE
:10A7700023B94FF480736383A383E383012005B07F
:10A78000BDE8F08F00230193CEE700BF01F0FFFF8B
:10A7900000D03B0038B504460D4600BF80680EF07F
:10A7A000C5FB2946606837F0CFFBA0680EF0C3FBFD
:10A7B00000BF38BDF0B55FEA930E33D000F110064C
:10A7C00001F1100502F11004774616ED046A55ED0B
:10A7D000044A56ED026A15ED025A16ED037A55ED5C
:10A7E000035A56ED017A26EE246A66EE856A04ED78
:10A7F000046A15ED016A44ED026A27EE257A67EED8
:10A80000867A013F04ED037A44ED017A06F11006E1
:10A8100005F1100504F11004D7D14FEA0E142044BD
:10A820002144224413F003030BD000EB8303F0EC2C
:10A83000017AB1EC017A67EE877A8342E2EC017A21
:10A84000F5D1F0BDA849A948A94A2DE9F84F01233F
:10A8500003700B88128823F040031B041B0C0B8031
:10A860000B8823F038031B0452084FEA13430BD024
:10A8700042F48072002A92FAA2F1B1FA81F208BF82
:10A880004FF0FF32013AD2001343974A9BB2138034
:10A8900013889BB243F040031380964B1B6813B19F
:10A8A0001A689B885383904940F2E93302E0002BF9
:10A8B00000F09E810A89013B12F0020F9BB2F6D094
:10A8C00005238B8140F2E933874902E0002B00F039
:10A8D0008F810A89013B12F0010F9BB2F6D08B8960
:10A8E000814940F2E93302E0002B00F0A5810A899A
:10A8F000013B12F0020F9BB2F6D000238B8140F295
:10A90000E933794902E0002B00F096810A89013B86
:10A9100012F0010F9BB2F6D08B89734940F2E933F4
:10A9200002E0002B00F084810A89013B12F0020F43
:10A930009BB2F6D006238B8140F2E9336A4902E0EC
:10A94000002B00F075810A89013B12F0010F9BB2C8
:10A95000F6D08B89644940F2E93302E0002B00F025
:10A9600063810A89013B12F0020F9BB2F6D00023EB
:10A970008B8140F2E9335C4902E0002B00F0548106
:10A980000A89013B12F0010F9BB2F6D08B89DFF8E8
:10A990006CA155499AF8004040F2E93344F00104B3
:10A9A00002E0002B00F03C810A89013B12F0020F0B
:10A9B0009BB2F6D004238B8140F2E9334A4902E08E
:10A9C000002B00F02D810A89013B12F0010F9BB290
:10A9D000F6D08B89444940F2E93302E0002B00F0C5
:10A9E0001B810A89013B12F0020F9BB2F6D0A4B280
:10A9F0008C8140F2E9333C4902E0002B00F00C81ED
:10AA00000A89013B12F0010F9BB2F6D08B893A4FB5
:10AA10003B88002B47D0DFF8E890DFF8E880324C25
:10AA20004FF0000B072699F8015040F2E93302E09D
:10AA3000002B00F0D5802089013B10F0020F9BB263
:10AA4000F6D0A68140F2E93302E0002B00F0C88086
:10AA50002089013B10F0010F9BB2F6D0A38940F290
:10AA6000E93302E0002B00F0BF802089013B10F0A9
:10AA7000020F9BB2F6D0ADB2A58140F2E93302E0FD
:10AA8000002B00F0B1802089013B10F0010F9BB238
:10AA9000F6D0A3893B8819F8010F08F8010F0BF1D4
:10AAA000010B9B45BFDB104840F2E93302E0002B6D
:10AAB00000F0AE800289013B12F0020F9BB2F6D08B
:10AAC00007238381084940F2E93302E0002B00F0BC
:10AAD0009F800A89013B12F0010F9BB2F6D08B894F
:10AAE000014840F2E93311E0003C00405F51002092
:10AAF000D0030020CC920020E60000209425002006
:10AB00003F4F002097250020002B7DD00289013B7C
:10AB100012F0020F9BB2F7D0FF238381484940F225
:10AB2000E93301E0002B6FD00A89013B12F0010FDD
:10AB30009BB2F7D08B899AF80040414840F2E93344
:10AB400001E0002B5CD00289013B12F0020F9BB2A6
:10AB5000F7D0042383813A4940F2E93301E0002B26
:10AB60004ED00A89013B12F0010F9BB2F7D08B89BE
:10AB7000334840F2E93301E0002B3DD00289013B2C
:10AB800012F0020F9BB2F7D0A4B22D49848140F29B
:10AB9000E93301E0002B2FD00A89013B12F0010FAD
:10ABA0009BB2F7D08B89274B1B6813B11A689B881F
:10ABB0001383234A138823F040031B041B0C1380C8
:10ABC000138823F038031B041B0C138013889BB2DB
:10ABD00043F0400313801C4B00211970BDE8F88F2F
:10ABE00020460EF083FB3AE720460EF07FFB51E74C
:10ABF00013480EF07BFB73E611480EF077FBD2E7AB
:10AC00000F480EF073FBB3E70D480EF06FFB92E7B1
:10AC10000B480EF06BFB63E709480EF067FBF6E6A6
:10AC200007480EF063FBD5E605480EF05FFBAEE685
:10AC300003480EF05BFB8DE601480EF057FB6CE617
:10AC4000003C0040CC9200205F510020AA490A88B5
:10AC500022F040022DE9F0471204A84F120C3B8865
:10AC60000A800A8822F0380212045B084FEA124276
:10AC700000F00D8243F4807090FAA0F10028B1FA40
:10AC800081F108BF4FF0FF310139C9000A439A49E9
:10AC90009B4D92B20A800A8892B242F040020A802A
:10ACA000296811B10A6888885083964A1278012A67
:10ACB00000F05482C0F00D82022A40F0D481924EFE
:10ACC000082232704FF4C372DFF844828A48A8F831
:10ACD0000020028822F040021204120C0280028836
:10ACE00022F038021204120C5BB143F4807090FA27
:10ACF000A0F30028B3FA83F308BF4FF0FF33013B02
:10AD0000DB0013437C4A9BB2138013889BB243F051
:10AD10004003138011B10B688A885A83764C4FF038
:10AD200010094FF0010A40F2E93302E0002B00F075
:10AD3000A4812289013B12F0020F9BB2F6D01FFAC8
:10AD400089F3A38140F2E93302E0002B00F0958102
:10AD50002289013B12F0010F9BB2F6D0A38940F289
:10AD6000E93302E0002B00F08C812289013B12F0D4
:10AD7000020F9BB2F6D0A4F80CA040F2E93302E037
:10AD8000002B00F07E812289013B12F0010F9BB263
:10AD9000F6D0A38909F10109B9F1200FC3D12968BF
:10ADA00011B10B688A881A83534B1A8822F040022B
:10ADB0001204120C1A801A8822F038021204120CA3
:10ADC0001A801A8892B242F040021A8018883A8893
:10ADD00020F040000004000C18801B8823F038038A
:10ADE0001B0452084FEA13430BD042F48072002A2E
:10ADF00092FAA2F0B0FA80F208BF4FF0FF32013AA7
:10AE0000D20013433C4A9BB2138013889BB243F099
:10AE10004003138011B10B688A885A83347836490D
:10AE200040F2E93302E0002B00F04B810A89013B3C
:10AE300012F0020F9BB2F6D000238B8140F2E9336F
:10AE40002D4902E0002B00F03C810A89013B12F001
:10AE5000010F9BB2F6D08B89274940F2E93302E01B
:10AE6000002B00F032810A89013B12F0020F9BB2E5
:10AE7000F6D0A4B28C8140F2E9331F4902E0002BE6
:10AE800000F023810A89013B12F0010F9BB2F6D03A
:10AE90008B891E4B18491C7840F2E93302E0002BE5
:10AEA00000F0F7800A89013B12F0020F9BB2F6D046
:10AEB00002238B8140F2E9330F4902E0002B00F0BE
:10AEC000E8800A89013B12F0010F9BB2F6D08B8912
:10AED000094940F2E93302E0002B00F0DE800A89E4
:10AEE000013B12F0020F9BB2F6D0A4B28C8140F26B
:10AEF000E933014911E000BF003C0040D0030020CD
:10AF0000CC920020E0920020E8000020E792002090
:10AF1000E6000020002B00F0C0800A89013B12F0FF
:10AF2000010F9BB2F6D08B899A4B9B481C7840F25C
:10AF3000E93302E0002B00F0B4800289013B12F0FB
:10AF4000020F9BB2F6D003238381934940F2E93389
:10AF500002E0002B00F0A5800A89013B12F0010FEE
:10AF60009BB2F6D08B898C4840F2E93302E0002B8B
:10AF700000F09B800289013B12F0020F9BB2F6D0D9
:10AF8000A4B28549848140F2E93302E0002B00F04D
:10AF90008C800A89013B12F0010F9BB2F6D08B899D
:10AFA0007E4B7D481C7840F2E93344F0040401E014
:10AFB000002B7ED00289013B12F0020F9BB2F7D02A
:10AFC00004238381744940F2E93301E0002B70D0FF
:10AFD0000A89013B12F0010F9BB2F7D08B896E48B2
:10AFE00040F2E93301E0002B67D00289013B12F007
:10AFF000020F9BB2F7D0A4B26749848140F2E933D3
:10B0000001E0002B59D00A89013B12F0010F9BB2DD
:10B01000F7D08B892B6813B11A689B8813835E4A1B
:10B020005F4C13885F4823F040031B041B0C138004
:10B03000138823F038031B041B0C138013889BB266
:10B0400043F040031380B8F80020002139F025FDBB
:10B050002378D3B1544B1B78002B00F0858000235C
:10B060002370BDE8F087514E327812F0400F0CBFCC
:10B070004FF4C3724FF4F07226E620460EF036F914
:10B080006DE620460EF032F984E6BDE8F0871946F9
:10B09000FCE541480EF02AF91AE73F480EF026F980
:10B0A00042E73D480EF022F95DE73B480EF01EF9FD
:10B0B00076E739480EF01AF991E737480EF016F99D
:10B0C000A8E735480EF012F9C6E633480EF00EF93F
:10B0D000DFE6314940F2E93301E0002B55D00A891F
:10B0E000013B12F0020F9BB2F7D0A0238B8140F2FC
:10B0F000E933294901E0002B47D00A89013B12F0CE
:10B10000010F9BB2F7D08B89234940F2E93301E06C
:10B11000002B35D00A89013B12F0020F9BB2F7D009
:10B1200000238B8140F2E9331B4900E043B30A89D5
:10B13000013B12F0010F9BB2F8D08B89D8B200F01E
:10B140000603022B194E03D000F00503012B11D08A
:10B150003B882968082232705B08B3E5134E482209
:10B1600032704FF4F072AFE5FFF76CFB00232370F1
:10B17000BDE8F0873B882968482232705B08F0E719
:10B1800005480EF0B3F8C0B2D9E703480EF0AEF8A8
:10B19000BAE700BFE8920020003C00409425002060
:10B1A00000000020982500205F510020E8000020CA
:10B1B000AE49AF4A2DE9F84F012313700B88AD4A11
:10B1C00023F040031B041B0C12880B800B8823F018
:10B1D00038031B0452084FEA13430BD042F4807229
:10B1E000002A92FAA2F1B1FA81F208BF4FF0FF32C1
:10B1F000013AD20013439D4A9BB2138013889BB23D
:10B2000043F0400313809C4B1B6813B11A689B8862
:10B210005383964940F2E93302E0002B00F071813C
:10B220000A89013B12F0020F9BB2F6D080238B817A
:10B2300040F2E9338D4902E0002B00F062810A8977
:10B24000013B12F0010F9BB2F6D08B89874940F287
:10B25000E93302E0002B00F058810A89013B12F02B
:10B26000020F9BB2F6D000238B8140F2E9337F4975
:10B2700002E0002B00F049810A89013B12F0010F26
:10B280009BB2F6D08889C0B27B4B1B6813B11A6899
:10B290009B881383754A794C1388794D23F04003BA
:10B2A0001B041B0C1380138823F038031B041B0C96
:10B2B000138013889BB243F04003138023782F68D8
:10B2C00083423ED0FFF7C2FC6E4E6F4AB6F846345A
:10B2D000B2F80080DFF8BCC1002210464FF0050B29
:10B2E0004FF0060A4FF00709F5181CF803402979BA
:10B2F000A14203F1010700F1050112D006EB010E96
:10B3000031182C711D0A81F8E4B181F8E6A181F8A9
:10B31000E73181F8E89181F8E551013206308EF885
:10B32000E441BBB2984502F1010260D9632ADBDD3A
:10B33000A6F8463400285FD14D4A00231370BDE8BB
:10B34000F88F524B4F4E1B78002BBED1D6F83C34B1
:10B35000FB1AB3F57A7FB8D9464B1046198836F0F8
:10B3600015FF454B1B6813B11A689B885383A021B6
:10B370003E4836F0E9FD00213C4836F0E5FD3E4B05
:10B380001B6813B11A689B881383384ADFF8088159
:10B39000138823F040031B041B0C1380138823F035
:10B3A00038031B041B0C138013889BB243F040032B
:10B3B000138098F80030182B00F0B880430700F194
:10B3C000B18000F00500012800F0C18060B9237849
:10B3D000580609D5D6F840242B68002A00F0BC8016
:10B3E0009B1A642B00F2BB80C6F83C746DE7002307
:10B3F000A6F8463400289FD01C491E4B0A881B889B
:10B4000022F040021204120C0A800A8822F038024C
:10B4100012045B084FEA12420BD043F48073002BF6
:10B4200093FAA3F1B1FA81F308BF4FF0FF33013B68
:10B43000DB0013430D4A9BB2138013889BB243F089
:10B44000400313800C4B1E6816B13368B2885A83D0
:10B45000064A0F4F938901384FF47A734FF6FF7401
:10B46000002F5DD03D7801371AE000BF003C00405E
:10B470005F510020D0030020CC920020E800002083
:10B480009C92002094250020E6000020E0920020FD
:10B4900078270020404F0020D5920020A34239D0C9
:10B4A0001189013B89079BB2F8D5ABB293814FF468
:10B4B0007A7302E0ABB2A3422CD01189C90703F121
:10B4C000FF35F7D501389189411CC9D116B13368D0
:10B4D000B2881A832A4A138823F040031B041B0CEA
:10B4E0001380138823F038031B041B0C138013886C
:10B4F0009BB243F040031380224A00231370BDE83F
:10B50000F88F1F480DF0F2FEA0E61D480DF0EEFE8C
:10B51000C0B2B9E61A480DF0E9FE1B4B1E68D5E72C
:10B52000FF25BDE70023C6F840345DE72378174ABE
:10B5300003F04003002B00F007010CBF4FF00D0E8D
:10B540004FF0100E13805180A2F806E036E7237802
:10B550005C067FF53FAF47E7C6F8403444E7FFF7A6
:10B5600075FB98F80030182B7FF43EAFB6F84434E2
:10B57000064A01339BB2A6F84434938034E700BFF7
:10B58000003C00405F510020CC920020D892002067
:10B590002DE9F84FA94F3B7803B1FEE7A84CA94A23
:10B5A00001233B702388128823F040031B041B0CEB
:10B5B0002380238823F038031B0452084FEA1343E7
:10B5C0000BD042F48072002A92FAA2F4B4FA84F208
:10B5D00008BF4FF0FF32013AD2001343984ADFF818
:10B5E00070829BB2138013889BB243F04003138098
:10B5F000D8F8003013B11A689B885383924B01220C
:10B600000D461A7004468E4940F2E93302E0002BE1
:10B6100000F0A3810A89013B12F0020F9BB2F6D021
:10B6200000238B8140F2E933854902E0002B00F0D2
:10B6300094810A89013B12F0010F9BB2F6D08B89ED
:10B640007F4940F2E93302E0002B00F09A810A8939
:10B65000013B12F0020F9BB2F6D000238B8140F227
:10B66000E933774902E0002B00F08B810A89013B26
:10B6700012F0010F9BB2F6D08B89714940F2E93389
:10B6800002E0002B00F079810A89013B12F0020FE1
:10B690009BB2F6D009238B8140F2E933684902E07E
:10B6A000002B00F06A810A89013B12F0010F9BB266
:10B6B000F6D08B89624940F2E93302E0002B00F0BA
:10B6C00058810A89013B12F0020F9BB2F6D0A4B256
:10B6D0008C8140F2E9335A4902E0002B00F04981A5
:10B6E0000A89013B12F0010F9BB2F6D08B89574EAD
:10B6F000534C013D4FF0000A4FF00A0B40F2E93382
:10B7000002E0002B00F010812289013B12F0020FB1
:10B710009BB2F6D0A4F80CB040F2E93302E0002B63
:10B7200000F002812289013B12F0010F9BB2F6D09A
:10B73000A38940F2E93302E0002B00F0F98022896E
:10B74000013B12F0020F9BB2F6D01FFA8AF3A381DD
:10B7500040F2E93302E0002B00F0EA802289013B4D
:10B7600012F0010F9BB2F6D0A38915F8019F40F2A9
:10B77000E93302E0002B00F0DF802289013B12F068
:10B78000020F9BB2F6D00B23A38140F2E93302E013
:10B79000002B00F0D1802289013B12F0010F9BB2F7
:10B7A000F6D0A38940F2E93302E0002B00F0C88014
:10B7B0002289013B12F0020F9BB2F6D01FFA89F9E1
:10B7C000A4F80C9040F2E93302E0002B00F0B880BE
:10B7D0002289013B12F0010F9BB2F6D0A389336896
:10B7E00033B11A689B8851690B4214BF538313838A
:10B7F0000AF1010ABAF1360F80D140F2E93310485C
:10B8000002E0002B00F0B1800289013B12F0020F30
:10B810009BB2F6D008238381094940F2E93302E064
:10B82000002B00F0A2800A89013B12F0010F9BB2AD
:10B83000F6D08B89024840F2E9330EE05F510020D8
:10B84000003C0040D0030020655100206892002099
:10B85000CC920020002B00F084800289013B12F082
:10B86000020F9BB2F6D0A0238381484940F2E9330E
:10B8700001E0002B75D00A89013B12F0010F9BB249
:10B88000F7D08B89414CA02540F2E93301E0002B31
:10B890005AD02289013B12F0020F9BB2F7D0A5814A
:10B8A00040F2E93301E0002B4ED02289013B12F037
:10B8B000010F9BB2F7D0A38940F2E93301E0002BDE
:10B8C00046D02289013B12F0020F9BB2F7D0002331
:10B8D000A38140F2E93301E0002B39D02289013BFA
:10B8E00012F0010F9BB2F7D0A089C0B28306CBD46F
:10B8F000D8F8003013B11A689B881383234A138841
:10B9000023F040031B041B0C1380138823F038031F
:10B910001B041B0C138013889BB243F040030021CF
:10B9200013803970BDE8F88F20460DF0DFFC00E78A
:10B9300020460DF0DBFC18E720460DF0D7FC31E780
:10B9400020460DF0D3FC4AE720460DF0CFFCB3E7CC
:10B9500020460DF0CBFCC0B2C8E70C480DF0C6FC89
:10B960006EE60A480DF0C2FC8CE708480DF0BEFCFC
:10B9700060E706480DF0BAFCB9E604480DF0B6FCE5
:10B9800098E602480DF0B2FC77E600BF003C0040AC
:10B9900030B4147874B11E23074D13FB0101294400
:10B9A000801A83181D2BD8BF0C7012F8014F01317B
:10B9B000002CF6D130BC7047404F0020F8B5434C06
:10B9C000434A2388128823F040031B041B0C238066
:10B9D0002388C1F1030123F0380341EA80071B04E7
:10B9E0005208FFB24FEA13430BD042F48072002A90
:10B9F00092FAA2F1B1FA81F208BF4FF0FF32013A98
:10BA0000D2001343314A334D9BB2138013889BB24B
:10BA100043F0400313802B6813B11A689B8853834B
:10BA20002A4CBFB2102640F2E93301E0002B45D08A
:10BA30002289013B12F0020F9BB2F7D0B3B2A3816F
:10BA400040F2E93301E0002B38D02289013B12F0AB
:10BA5000010F9BB2F7D0A38940F2E93301E0002B3C
:10BA600030D02289013B12F0020F9BB2F7D0A781A0
:10BA700040F2E93300E02BB32289013B12F0010FC1
:10BA80009BB2F8D0A3890136202ECCD12B6813B1FC
:10BA90001A689B8813830D4A138823F040031B0404
:10BAA0001B0C1380138823F038031B041B0C13801A
:10BAB00013889BB243F040031380F8BD20460DF07D
:10BAC00015FCC9E720460DF011FCDCE7003C004006
:10BAD000D0030020CC92002038B5454B1D780028BB
:10BAE0007BD105F0F70543491D700B88424A23F0CE
:10BAF00040031B041B0C12880B800B8823F03803B7
:10BB00001B0452084FEA13430BD042F48072002A00
:10BB100092FAA2F1B1FA81F208BF4FF0FF32013A76
:10BB2000D2001343334A354C9BB2138013889BB227
:10BB300043F040031380236813B11A689B88538332
:10BB400040F2E9332B4901E0002B49D00A89013B3F
:10BB500012F0020F9BB2F7D004238B8140F2E9333D
:10BB6000244901E0002B3BD00A89013B12F0010F70
:10BB70009BB2F7D08B891F4940F2E93301E0002BDB
:10BB800032D00A89013B12F0020F9BB2F7D0ADB25E
:10BB90008D8140F2E933174900E02BB30A89013B5C
:10BBA00012F0010F9BB2F8D08B89236813B11A6889
:10BBB0009B8813830F4A138823F040031B041B0C3C
:10BBC0001380138823F038031B041B0C1380138885
:10BBD0009BB243F04003138038BD45F0080582E76F
:10BBE00004480DF083FBC6E702480DF07FFBDCE75D
:10BBF00094250020003C0040D0030020CC9200207F
:10BC00002DE9F04F9BB0B0F908500D81EDB2442DF5
:10BC100000AF0C46904600F08482064643D9812D41
:10BC200000F0C58200F29980542D00F0CE8040F2E1
:10BC30000F826E2D00F04382802D40F024819F4BB7
:10BC400093F800A00AF1020A1AF0FF0A00F09980A6
:10BC50009B4BDFF8A0829B4EDFF89CB29A4403F125
:10BC600001090A2516E0322D00F00486A5F13C00FA
:10BC7000C0B2132840F2078600232268511C2160BD
:10BC800015702268D14502F101012160137078D04E
:10BC900019F8015B0A2DE6D1BBF80030FF2BA8BFD5
:10BCA000FF23DBB2E9E7052D00F0298220D8022D21
:10BCB00000F0838040F2B981032D00F0F581042D5E
:10BCC00040F0E1802A46804920460EF02BF8002102
:10BCD00020460EF06CF822680221531C01252360D7
:10BCE00028462B466C3711706381BD46BDE8F08F46
:10BCF000242D60D040F24F81282D00F01A82382D7B
:10BD000040F0C1800A68714B0125511C21601570FB
:10BD10002268052150192060117022680A215019EB
:10BD20002060117022680021501920601170226873
:10BD300019785019206011702268597850192060C4
:10BD4000117022689978531923602B461170284688
:10BD50006C376381BD46BDE8F08FA02D19D040F24D
:10BD60003981B82D00F02182FE2D40F08C80584D95
:10BD700005F1080635F8021B20460EF018F8AE4211
:10BD8000F8D101252B4628466C376381BD46BDE8B6
:10BD9000F08F504B084619680DF0F2FF4E4B2046CD
:10BDA00019680DF0EDFF4D4B1968204601250DF087
:10BDB000E7FF2B46E7E74A4BF6E7042249492046CE
:10BDC00001250DF0AFFF2B46C1E70B68464ADFF8AF
:10BDD0002C81581C11212060197023681278591C7D
:10BDE00021601A70236898F85520591C21601A7038
:10BDF000236898F85420591C21601A70B8F8501024
:10BE000020460DF0D4FF23680022591C21601A70CF
:10BE100023682822591C21601A70B8F85210204655
:10BE20000DF0C5FFA8F1020508F14E0635F8021F16
:10BE300020460DF0BCFFB542F8D122682B4B0D21F6
:10BE4000501C20605D181170226813F8011F501CEF
:10BE5000AB4220601170F7D123680222591C216087
:10BE60001A70B8F8561020460DF0A1FFB8F8581017
:10BE700020460DF09CFF0125B8F85A1020460DF021
:10BE800096FF2B4663E7214628460FF04DF8034600
:10BE900000287FF476AF742D00F0F880772D2FD135
:10BEA0003268716891421EBF531C33601178104A8A
:10BEB00008BF1946204631F051FF62E70D530020BC
:10BEC000A84B040818310020027C0020E3BF0020AA
:10BED000D8920020107AFF1F147AFF1F187AFF1FD4
:10BEE00028C1002000870408E4920020B1A60020A9
:10BEF000F1CF0308676666664031002054A6002033
:10BF0000F52D00F0B785762D00F09982472D00F0D1
:10BF1000EB8496E80440A5F12101AEEB020036293E
:10BF200000F2C082DFE811F06C02BE02BE02BE0267
:10BF3000BE02BE02BE02BE020F02BE02BE02BE02B0
:10BF4000BE02BE02BE02BE02BE02BE02BE02BE02F1
:10BF5000BE02BE02BE02BE025C02BE02BE02BE0243
:10BF6000BE02BE02BE02BE02BE02BE02BE02BE02D1
:10BF7000BE02BE02BE02BE02BE02BE02BE02BE02C1
:10BF8000BE02BE02BE02BE02BE02BE022702BE0248
:10BF9000E901BE02D401202D7FF475AF0B68B84DC6
:10BFA000591C6A7821601A7023682A78591C21600C
:10BFB0001A702368AA78591C21601A7029892046B2
:10BFC0000DF0F5FE23686A79591C21601A70226809
:10BFD000A97982E6822D7FF456AF0B68A94AAA4D53
:10BFE0001178A74A581C20601970118920460DF05D
:10BFF000DEFEA64B22681B88FF2B02F10101A8BFC1
:10C00000FF2321601370A96881F3100189B22046D3
:10C010000DF0CDFE296801F30F0189B220460DF025
:10C02000C6FE9B4B2268197857E6012D7FF42BAF93
:10C030000B680022591C21601A7023685A1C226068
:10C040001D7022682521531C23602B4611707EE64B
:10C05000522D7FF418AF0A688E4D531C03212360C4
:10C0600005F10C0E2B461170062601202268511C8A
:10C07000216010702268734502F101012160167081
:10C0800000F0DE809879DE790633EFE73268716878
:10C0900091421EBF531C336011787F4A08BF194676
:10C0A000204631F05BFE6CE60B685A1C0A601D707E
:10C0B0000B685A1C0A601D70226800210DE6734B44
:10C0C0000A681B88704DFF2BA8BFFF23511C2160FD
:10C0D0001370A96881F3100189B220460DF067FE44
:10C0E0006E4B204619880DF062FE296801F30F019E
:10C0F00089B2204601250DF05AFE2B4627E60B2279
:10C10000674920460DF00EFE0822664920460DF0D4
:10C1100009FE01250722644920460DF003FE2B4647
:10C1200015E6002A3FF42DAE604B136001252B4627
:10C130000DE60B68DFF890915D4E591C02222160DC
:10C140001A7023684FF006085A1C226083F800809A
:10C1500023680A22591C21601A70236801255A1984
:10C1600022601D70B9F8001020460DF020FEB9F8CD
:10C17000021020460DF01BFE23685A19226083F836
:10C18000008023685022591921601A702368002208
:10C19000591921601A70318820460DF008FE718807
:10C1A00020460DF004FE2B46D1E5424BFCE5424B08
:10C1B0001E78033616F0FF063FF4E3AD3F4BDFF881
:10C1C0000C811E4403F1010A4FF00A0920E0B9F185
:10C1D000500F00F05683B9F1320F00F06A83A9F1D5
:10C1E0003C00C0B2132840F267830025294623682B
:10C1F0005A1C2260204683F800900DF0D8FD294695
:10C2000020460DF0D4FDB2453FF4BBAD1AF8019BBA
:10C21000B9F10A0FDBD12A4B9D68196805EB85053A
:10C220004FF6FF736D009D42A8BF1D469942A8BFFF
:10C23000194625EAE57521EAE171ADB289B2D6E782
:10C24000204B21681A78481C20600A70002A3FF4AD
:10C2500098AD013AD2B202EB420205EB42025278AB
:10C26000002A3FF48EAD0132D5180133226813F84D
:10C27000011F501CAB4220601170F7D181E500BF57
:10C28000DC55002012540020EC550020FC53002007
:10C29000E0A600209854040855D00308C6A6002044
:10C2A0000887040814870408208704086DAC010877
:10C2B00000310020B84D00200D530020B84B040879
:10C2C000CC300020887000206095002010310020C4
:10C2D000531C336012F8370B07F127010133336029
:10C2E00013F8015C01F8015F9A42F7D107F12801C8
:10C2F0000125FFF74DF92B4629E5531C336092F8D1
:10C300000080B8F1FF0F00F04285B8F1FE0F00F099
:10C31000268530460DF0F6FC33687268D21A002A82
:10C3200007DD5A1C32601B781BB9B8F10C0F40F2C4
:10C330005B85B8F1270F00F28684534B012523F863
:10C3400018002B4603E5531C336013780A2B00F0CA
:10C35000B784502B40F0AC8430460DF0D3FCDFF8AE
:10C360004081A8F8000030460DF0CCFC0125A8F86B
:10C3700002002B46EBE4531C33601178032900F2D2
:10C3800062844B1E414D424ADBB203EB430305EB93
:10C39000430311705D7800293FF4F3AC431EDBB218
:10C3A000AB4240F050840021C2F80610C2F80210DF
:10C3B00091725BB1581C3368104401320133336011
:10C3C00013F8011C02F8011F9042F7D1314B1B7882
:10C3D000002B3FF4D6AC012522F082FE2B46B6E4BA
:10C3E000531C336013780A2B00F09F8430460DF005
:10C3F00094FC30460DF091FC30460DF08EFCC0E40C
:10C400001346511C3160244D13F8021B69703360D0
:10C4100053782B70D31C33609378AB7030460DF09B
:10C4200071FC33682881591C1A46316012F8021BCE
:10C43000697132605B78AB7101252B4687E4326805
:10C44000511C31601278002A00F04184102A00F05B
:10C4500099841D4619462368581C20601A7020468E
:10C460000DF08EFC294620460DF08AFC0B4B204631
:10C4700019680DF085FC204600210DF098FC002184
:10C4800020460DF094FC17E654A6002098540408AA
:10C49000887000206F310020DC550020F02F002034
:10C4A000003100200B3DEF2D00F2CD8301A151F8AA
:10C4B00025F000BF3FDC000847CC000847CC00084F
:10C4C00047CC000847CC000847CC000847CC000800
:10C4D00047CC000847CC000847CC000847CC0008F0
:10C4E00047CC000847CC000847CC000847CC0008E0
:10C4F00047CC000847CC000847CC000847CC0008D0
:10C5000047CC000847CC000847CC000847CC0008BF
:10C5100047CC00089FDB000847CC00087DDB000803
:10C5200047CC000853DB000847CC000847CC000884
:10C5300047CC000827DB000847CC000877DA000862
:10C5400047CC000845DA000847CC00081FDA00088D
:10C5500047CC00080DDA000847CC0008B5D9000820
:10C5600047CC0008F9CB000847CC000847CC0008AE
:10C5700047CC000847CC000883BD000847CC000822
:10C580003FD9000847CC000847CC000825D900084F
:10C5900047CC000867CC000847CC000847CC00080F
:10C5A00047CC000847CC000819D9000847CC000840
:10C5B00047CC000847CC0008D9D8000847CC000871
:10C5C00097D7000847CC000847CC000857D7000889
:10C5D00047CC000847CC000847CC000847CC0008EF
:10C5E00047CC000847CC000847CC0008FDD700081E
:10C5F00047CC0008D5D6000847CC00081BD6000859
:10C6000047CC00086DD5000847CC0008FFD40008CF
:10C61000E1D40008ABD4000847CC000847CC0008A0
:10C6200047CC000847CC000847CC000847CC00089E
:10C6300047CC000847CC000847CC000847CC00088E
:10C6400047CC000847CC000847CC000847CC00087E
:10C6500047CC000847CC000847CC000847CC00086E
:10C6600047CC000847CC000847CC000847CC00085E
:10C6700047CC000847CC000847CC000847CC00084E
:10C6800047CC000847CC000847CC000847CC00083E
:10C6900047CC000847CC000847CC000847CC00082E
:10C6A00047CC000847CC000847CC000847CC00081E
:10C6B00047CC000847CC000847CC000847CC00080E
:10C6C00047CC000847CC000847CC000847CC0008FE
:10C6D00047CC000847CC000847CC000847CC0008EE
:10C6E00047CC000847CC000847CC000847CC0008DE
:10C6F00047CC000847CC000847CC000847CC0008CE
:10C7000047CC000847CC000847CC000847CC0008BD
:10C7100047CC000847CC000847CC000847CC0008AD
:10C7200047CC000847CC000847CC000847CC00089D
:10C7300047CC000847CC000847CC000847CC00088D
:10C7400047CC000847CC000847CC000847CC00087D
:10C7500047CC000847CC000847CC000847CC00086D
:10C7600047CC000885D4000847CC000861D40008F5
:10C770003BD4000847CC000847CC000847CC000851
:10C7800047CC000847CC000847CC000847CC00083D
:10C7900047CC000847CC000847CC000847CC00082D
:10C7A00047CC000847CC0008D3D3000883D3000847
:10C7B0004BD3000847CC0008A9D2000807D20008D4
:10C7C000EBD1000847CC000879D2000853D100080B
:10C7D0002BD1000819D10008B9D0000847CC0008B7
:10C7E00089D0000847CC000847CC00085FD000087B
:10C7F00031D000081DD00008F5CF0008D5CF0008C3
:10C80000ABCF00087FCF000867CF000847CC0008F7
:10C8100047CC000847CC000847CC000847CC0008AC
:10C8200047CC000847CC000847CC000847CC00089C
:10C8300047CC000847CC000847CC000847CC00088C
:10C8400047CC000847CF000847CC000847CC000879
:10C85000EDCE000847CC000847CC000847CC0008C4
:10C8600047CE000847CC000847CC000847CC00085A
:10C870002DCE00083388FF2BA8BFFF23DBB2FFF7C4
:10C88000FCB9BE4BC8E41FF0BBF900283FF4F4A983
:10C8900003780A2B26D8B0F9023088FB0312DB1785
:10C8A000C3EBA2039BB2FF2BA8BFFF23DBB2FFF7B2
:10C8B000E4B998E82200B1E41FF0A2F900283FF49F
:10C8C00094AC03780A2B3FF690ACB0F90430B0F981
:10C8D000061003EB830383F3500521EAE171ADB247
:10C8E00089B284E40023E1E7726835687B623046F0
:10C8F000551B0DF0F0F9052D38627B6A00F26F814F
:10C900008026B346012594E80600521A103AB24236
:10C91000B8BF1FFA82FB9A4A396A92683A61521A82
:10C920009345396A7B622046FA6088BF1FFA82FB12
:10C930000DF026FA7B6A002B00F03081002D40F0CC
:10C94000F6802368C7F800D05D71C0B00533C7F822
:10C9500004D0FB61BBF1000F00F056823B6A3A69DC
:10C96000934280F04E823E6A7D62AA46A846BC6031
:10C970008025FB68A3EB0808814BB8F5807F9B6896
:10C9800028BF4FF4807806EB08029A4288BFA3EBD9
:10C9900006080EF055F87C684246214630460EF0F7
:10C9A000D5F8F969B86104EB000C0B787B6164453C
:10C9B0002ED2DFF8E0910CF1FF3C04F1FF3E1EF8AF
:10C9C000013F09EB830219F823405688ECB100239C
:10C9D0004FF4004204F1FF3816424FEA520202D0EF
:10C9E0000878284308706D0806D10AF1010A4D70D5
:10C9F0001FFA8AFA01318025D34503D8E64533D39F
:10CA0000434531DB01339C42E6D1E645D7D1F9619C
:10CA10007B6ABA6913449BB2D3457B6206D97B6AB1
:10CA20003A6A9846D6183B699E42A2D3BC68802DCC
:10CA30001CBF0AF101031FFA83FA0AF1020189B24D
:10CA400020460DF0B4F92368796A01255A1922604D
:10CA500020461D700DF0ABF92368534423602B462C
:10CA6000D7F800D0FFF773B9FB69BC681A463B7D65
:10CA70001370DCE7336872689A4240F02D81414BB5
:10CA8000FF221A704FF0000A3F4D16F073FB51461B
:10CA900020223E4885F800A037F0FFFF87F828A045
:10CAA00097F82830072B00F2AA81DFF8EC90374E78
:10CAB000524697F8283003EB430309EBC3035B7C32
:10CAC000E3B197F8283003EB430309EBC3032021BC
:10CAD0005B699BB197F8283003EB430309EBC30371
:10CAE000586946F822000CF069F92B7856F82300B3
:10CAF0000CF021FA2A780132D2B22A7097F8283045
:10CB00000133DBB287F8283097F82830072BD0D9CB
:10CB10002368591C21601A70B8F1000F3FF431A945
:10CB20001B4BC8F8003001252B46FFF710B9144BFA
:10CB30003A6A9B68D4F800905A449A4240F288803E
:10CB40003A6AA3EB02080DF07BFF42464946386A79
:10CB50000DF0FCFF236803442360002D3FF411A96E
:10CB6000B042BFF60EA9002100E0236801305A1C34
:10CB7000B04222601970F8D1FFF703B904310020E8
:10CB800054010020E0290020EE4E0020D84B002068
:10CB9000F9700208C84B0408C4570020002DC6D104
:10CBA000594620460DF003F923685A1C22601D7077
:10CBB000BE4B26689D683B6A0BEB03029542C0F0B2
:10CBC00027810DF03DFF5A463146386A0DF0BEFF11
:10CBD00023680125034423602B46FFF7B8B830468D
:10CBE0000DF090F8326871687B6A9142834640F09C
:10CBF000AD8006461D4686E60723B0FBF3F3C3EB84
:10CC0000C301411A1FD1DBB203F1FF3A5FFA8AFA7E
:10CC1000002B3FF4B6A8DFF898B20AF1010A0D46DE
:10CC2000531C336092F90020A14B4FF0000893F998
:10CC30000210914203F1080300F0978608F1010801
:10CC4000B8F1060FF3D14FF0FF352B46FFF77FB851
:10CC50000DF0F6FE5A464946386A0DF077FF236814
:10CC6000034423607CE7531C3360924B1278DFF857
:10CC700074821A700023C8F8003030460DF02BF88B
:10CC80003368D8F800208C498C4D10435A1CC8F8E2
:10CC9000000032601B780B7230460DF033F82860CC
:10CCA00030460DF02FF8686030460DF02BF8A86084
:10CCB00030460DF027F830460DF024F8FFF761B844
:10CCC00030460DF01FF8DFF82082FFF74ABB7C4B9F
:10CCD00093E82200FFF7BFBB5A1C1946326079481F
:10CCE00011F8022B027031605B784370042A03D97B
:10CCF000FF2A7FF4E1A9C5E673490978994205D86E
:10CD0000022A7FF4D9A9FF2B7FF4D6A92368012535
:10CD10005A1922601D70B8F1000F3FF432A86B4B16
:10CD2000C8F800302B46FFF712B8931C3360684BED
:10CD300051781970D11C316091785970111D316092
:10CD4000D2789A7001252B46FFF701B8511C31604B
:10CD500012781D46131C064618BF0123D3E5931C09
:10CD600033605578022D3FF66EAF30460CF0CAFFA7
:10CD7000584B03EB45034FF0FF35A3F856002B4605
:10CD8000FEF7E5BF4F4B59689D68FFF764BB931CE6
:10CD90003360514B51781970D31C3360DFF8348104
:10CDA000937888F85530131D3360D37888F8543061
:10CDB00030460CF0A7FFA8F8500030460CF0A2FF58
:10CDC00030460CF09FFF96E80C009B1A012BA8F848
:10CDD00052007EF7D6AF30460CF094FF0125A8F83C
:10CDE0005A002B46FEF7B3BF3A4B0030984418BFA9
:10CDF0000120012588F85E002B46FEF7A8BF5246A9
:10CE000086E67D62AA4618E6DA46C7F824B014E63C
:10CE10003B6AED1A0DF014FE2A463146386A0DF0D1
:10CE200095FE236803442360FEF7ABBF2B4B1B78B2
:10CE3000DB073FF508AF012503F00AFCFBF710FE06
:10CE40002B46FEF784BF30460CF05CFF3368388514
:10CE50001A46591C316012F8021B326087F82A10FA
:10CE60005A7887F82B20DA1C32609A7887F82C20C1
:10CE70001A1D3260DA7887F82D205A1D32601B792E
:10CE800087F82E3007F1280000233B860CF096FE31
:10CE9000134A0C4B1268801A4FF0010561F1000132
:10CEA000C3E906012B46FEF752BF00BF5401002024
:10CEB00054700020A095002028700020E83F00203A
:10CEC00088870020E02900200D53002079AC01085C
:10CED000E3BF002054A60020E4920020B8520020B6
:10CEE0009C92002028C1002060950020531C3360D4
:10CEF00013780F2B3FF6A7AE911C3160C3EBC30331
:10CF0000C7495078C854D01C30600B449178597090
:10CF1000111D3160D1789970511D31601179D9702E
:10CF2000911D316051791971D11D3160917959711B
:10CF300002F108013160D2799A71012528F048FE8A
:10CF40002B46FEF704BF30460CF0DCFEDFF8E08233
:10CF5000A8F80E0030460CF0D5FE0125A8F80C000C
:10CF60002B46FEF7F4BE30460CF0CCFEAD4A00EB8B
:10CF700080004300012513802B46FEF7E8BE1146D2
:10CF8000531C3360A84B11F8020B187031605178B4
:10CF90005970D11C316091789970111D3160D2782F
:10CFA000DA7001252B46FEF7D2BE30460CF0AAFE01
:10CFB000DFF8B482A8F8100030460CF0A3FEA8F801
:10CFC000120030460CF09EFE0125A8F814002B46F6
:10CFD000FEF7BDBE1346511C316013F8020B3360DF
:10CFE000D31C5178336092782CF0D8FF00287EF45F
:10CFF000C8AE28E61346511C31608C4913F8020B69
:10D00000087033608A4953788B70D31C3360854B2A
:10D0100092789A7001252B46FEF799BE854B86497A
:10D0200018684E22012536F0A5FB2B46FEF78FBE71
:10D030001146531C3360814B11F8020B187031609C
:10D0400051785970D11C316092789A7030460CF04A
:10D0500059FE7B4B0125D8802B46FEF778BE304623
:10D060000CF050FEDFF8D881A8F8000030460CF034
:10D0700049FEA8F8020030460CF044FE0125A8F84D
:10D0800004002B46FEF763BEDFF8E09199F800300C
:10D09000002B3EF476AEDFF8D881002530460CF048
:10D0A00031FE26F001FB99F80030A8EC010A0135A9
:10D0B0009D42F3DBFEF765BE0D287FF4C4AD531C23
:10D0C00033601578072D3FF6BEADDFF8A8913046E6
:10D0D0004FF00C080CF016FE08FB05F809EB0805EC
:10D0E000A88030460CF00EFEE88030460CF00AFEB8
:10D0F000336828811A46591C316012F8021BA97244
:10D1000032605B78EB7230460CF0E5FD012549F8A2
:10D1100008002B46FEF71BBE30460CF0F3FD494BD2
:10D12000012518802B46FEF712BE531C3360107881
:10D13000060600F1AE80444B1B78DD073EF521AEBC
:10D14000032828BF0020012503F00AFA2B46FEF72A
:10D15000FEBD531C3360304692F800A00CF0BBFDBE
:10D16000814630460CF0B7FD054630460CF0B3FD65
:10D17000804630460CF0C6FD30460CF0C3FD30460C
:10D180000CF0CBFDBAF1000F18D0BAF1100F7EF4FD
:10D19000F8AD2E4BC3F804909D60B8F1000F02D09B
:10D1A0002B4BC3F800802B492B4B0222081F012573
:10D1B0001A701CF08FFA2B46FEF7C9BD274B1020C2
:10D1C000C3F800905D600EF057FF254A137843F0D6
:10D1D00001031370B8F1000F3EF4D3AD1C4B0125D1
:10D1E000C3F800802B46FEF7B2BD174B1B78DA0759
:10D1F0003EF5C7AD1A4A1378012543F004031370B6
:10D200002B46FEF7A4BD104B1B78D9073EF5B9ADF0
:10D21000144B4FF4C87201251A802B46FEF797BDB8
:10D22000CC4C00208095002084850020E07C0020EC
:10D230007095002058560020887B040868950020CF
:10D24000008F0020A0880020B8520020E029002094
:10D25000F02F0020E82900209487002088870020F4
:10D260005656002094C40020845800200D530020FE
:10D270007C4000200C4C0020AB4B1B78D8073EF5BF
:10D2800080AD012503F0D8F9FBF7EAFB2B46FEF74A
:10D290005EBD00F07F00032828BF0020012517F0A5
:10D2A000F3F92B46FEF753BD09287FF7CCACDFF826
:10D2B000B4821346511CD8F80050316013F8021B99
:10D2C000297033605378AB70D31C33609378642B30
:10D2D00002F10401A8BF64236B713160D378642B21
:10D2E00002F10501A8BF6423AB7131601379EB71C2
:10D2F000931D33605379642B02F10701A8BF6423A7
:10D300002B7231609379EB7002F108033360D379AB
:10D310002B7130460CF0F6FC726833686881D11AC4
:10D3200000290CDD591CD8F800003160521A002A7F
:10D330001978417203DD9A1C32605B7843700125D5
:10D3400026F0ACFF2B46FEF702BD784B1868D31CC5
:10D35000014621329D1E356013F8035C0D705D1E81
:10D36000356013F8025C4D70336013F8015C8D700A
:10D3700003339A4201F10301ECD126F03FF8FEF7A6
:10D3800000BD531C336013786949002B46D00B78DD
:10D3900043F00203901C0B70664D306053782B7580
:10D3A00030460CF098FC286030460CF094FC686025
:10D3B00030460CF0A7FC288130460CF0A3FC5E4AF6
:10D3C000E8811378012543F0020313702B46FEF722
:10D3D000BEBCC0F34705122D3FF635AC15B307F1BF
:10D3E000680307F1260903EB4508CA46A8F142087D
:10D3F00030460CF087FC2AF8020FD045F8D14F4B8D
:10D4000039F8022F23F8022FD145F9D1112D09D96E
:10D410004B4A01231D461370FEF799BC0B7803F0AD
:10D42000FD03B7E7474A6B00023B13440021223259
:10D4300023F8021F9A42FBD1EAE7531C42483360AB
:10D4400001781378D1B904220270404A9B001380FE
:10D45000FCF78AFC3E4B012518622B46FEF777BC91
:10D46000DFF8048100233046C8F800300CF033FCAC
:10D470000125C8F800002B46FEF769BC04297EF49C
:10D4800080ACE2E71346511C316013F8025B336055
:10D49000D31C5078336091789DB1012D7EF471AC2E
:10D4A00017F0D6F82B46FEF752BC531C33601378A6
:10D4B0006BB14FF4004001250EF00EFE2B46FEF737
:10D4C00046BC012525F01EFE2B46FEF740BC214A36
:10D4D0001368012523F4004313602B46FEF737BC85
:10D4E000114B1B7813F001017FF4ADAB531C33607B
:10D4F0001078012516F0F2FF2B46FEF728BC1346E4
:10D50000511C3160144913F8020BC8703360134981
:10D5100053784B71D31C3360114B9278DA7001252C
:10D520002B46FEF714BC00BFB8520020585600200E
:10D5300056560020545C0020928700204A43002069
:10D54000704300204C430020DC4A0020C6A6002087
:10D55000E0290020505600207095002018A90020D6
:10D56000809500205C560020B84D002030460CF01D
:10D57000C9FB30460CF0C6FB30460CF0C3FB30460E
:10D580000CF0CBFB3368C54D1946581C2A68306037
:10D5900011F8020B82F82C003160597882F83610AD
:10D5A000D91C31609B7882F8373030460CF0B5FBDF
:10D5B00030460CF0B2FB30460CF0AFFB3046D5F8ED
:10D5C00000800CF09FFBA8F83A003046D5F80080A8
:10D5D0000CF098FB33687268A8F83800D11A01295A
:10D5E0000ADD591C2A6831601B7882F82E303046DB
:10D5F0000CF093FB33687268D31A032B0BDD3046B3
:10D60000D5F800800CF07EFBA8F8320030462E687A
:10D610000CF078FBB0862868AFE6531C33609F4D52
:10D62000DFF8A882137888F805303046D5F80090E6
:10D630000CF068FBA9F820003046D5F800900CF0FB
:10D6400061FB72683368A9F81E00D11A072919DD39
:10D6500030460CF057FBA8F80A0030460CF052FB9D
:10D66000A8F80C003046D5F800900CF04BFBA9F858
:10D6700022003046D5F800900CF044FB3368726805
:10D68000A9F82400D11A03290BDD30460CF03AFB2F
:10D69000A8F80E0030460CF035FB33687268A8F825
:10D6A0001000D21A002A05DD591C2A6831601B7847
:10D6B00082F82630FBF72CF921F0F0FF784B286830
:10D6C0001B68002B00F0D080012525F0C7FA2B46FF
:10D6D000FEF73DBB1346511C3160DFF8F08113F8B3
:10D6E000021B88F8021033606E4953780B70D31C0C
:10D6F00033606D4D93782B71131D3360D378092BF4
:10D70000A8BF09233046AB700CF0FCFA336872688E
:10D710002880D11A012905DD30460CF0F3FA336870
:10D720007268E8819A4207D05A1C32601B78003335
:10D7300018BF012388F80730FBF7EAF833687268EE
:10D740009A423EF41EAB5A1C32601B78EB700125E6
:10D750002B46FEF7FCBA554B1B78012B3EF611AB5E
:10D760001146531C3360DFF8688111F8023B88F8DA
:10D7700002303160D31C50783360AEEB0303012BD1
:10D7800091782FDD30460CF0BDFA0125A8F8000095
:10D790002B46FEF7DCBA531C336092F80080B8F1D8
:10D7A000110F3FF650AA931C3360414D537805F892
:10D7B000183030460CF0A6FA40F6CA039842A8BFCB
:10D7C000184640F2EE23984205EB4801B8BF1846D0
:10D7D0000125A0F2EE222B46192092FBF0F24A70AE
:10D7E000FEF7B5BA334B1A88012512FB00F22B461F
:10D7F00092FBF1F2A8F80020FEF7A9BA2E4B1B68A5
:10D80000002B3EF4BEAA1CF05DF8FF283EF4B9AA36
:10D8100030460CF077FA3F2831D9DFF8B880002580
:10D8200088F8005033687268A8F80400D21A012AF8
:10D830007EF7A7AA1A46591C316012F8021B88F815
:10D84000021007F16800326000225D7800F8402D78
:10D850001CF00AF897F82830AB423EF492AA28460A
:10D860001CF026F8FEF78DBA14481549154A164BD8
:10D87000036001250B6013602B46FEF768BAC508EC
:10D8800000F0070301350133EDB2DFF84880284688
:10D89000194688F801301EF037F9C1E758560020C4
:10D8A00098950020649500208458002016C100201F
:10D8B00008460020C6930020BC520020A489002006
:10D8C000F8890020F88D0020EB8B0108E07C002017
:10D8D000C0A60020C05200201346511CC34D316029
:10D8E00013F8021B2971336053786B7130460CF0CA
:10D8F00009FA336828805A1C32601B78AB713046B5
:10D900000CF000FA336868805A1C32601B78EB71A7
:10D9100001252B46FEF71BBA01250DF0F3F82B4627
:10D92000FEF715BAB24B02F108010132326012F86B
:10D93000010C03F8010F9142F7D1FEF722BA13460A
:10D94000511C3160AB4913F8020B8870336050787A
:10D95000487073453EF415AAD31C3360A64B9278E9
:10D960001A7401252B46FEF7F2B90BEBC8093046B5
:10D9700089F802200CF0C6F933682BF838001A46F3
:10D98000591C316012F8021B89F8031032605A7872
:10D9900089F80420DA1C32609A7889F806201A1D6A
:10D9A00032600135DB7889F80530AA457FF438A963
:10D9B000FEF7E7B9531C336013780E2B3FF643A9EB
:10D9C000911C31605578032D3FF63DA98B48062107
:10D9D00001FB03F1431802F1030E5D71C6F800E08C
:10D9E00095784554111D3160D1785970511D3160C1
:10D9F00011799970911D31605179D970D11D3160C3
:10DA000092791A7101252B46FEF7A1B9531C336098
:10DA10007B4B12785A7501252B46FEF798B9531C9B
:10DA2000336015781F2D3FF60EA905287FF40BA94A
:10DA300030460CF050F9734B43F8250023F024F9DD
:10DA4000FEF79FB96F4D05F1400830460CF05AF9CA
:10DA50003368A5F88000591C1A46316012F8021B81
:10DA600085F8821032605B7885F883300435A845EC
:10DA7000EBD1FEF786B9531C614D336013782B72DE
:10DA800030460CF03FF9A88330460CF03BF9288370
:10DA900030460CF037F932686883531C33601278D3
:10DAA000EA747268D31A032B1FDC3368D11A052974
:10DAB0000EDD5A1C32601B78EB7230460CF00BF90D
:10DAC0003368E8605A1C32601B782B7433687268C4
:10DAD000D21A002A7EF755A95A1C32601B7885F8A5
:10DAE000213001252B46FEF732B930460CF00AF9F9
:10DAF000A88430460CF006F933687268E884D11ABD
:10DB00000329D3DD1A46591C316012F8021BA9778C
:10DB100032605B7885F8203030460CF0F3F83368DB
:10DB200072686884C2E7531C336037491078087004
:10DB3000AEEB030EBEF1000F7EF723A9931C3360FA
:10DB40005378003318BF012301254B702B46FEF795
:10DB5000FEB830460CF0D6F8DFF8B480C8F8000004
:10DB600030460CF0CFF8C8F8040030460CF0CAF884
:10DB70000125C8F808002B46FEF7E9B8DFF89480C5
:10DB80000023C8F8003030460CF0A5F8D8F8003073
:10DB900001250343C8F800302B46FEF7D8B8511CC6
:10DBA000316015783B62132D3FF64DA8911C316012
:10DBB00050787A6230F00CF900283FF444A87A6A71
:10DBC0001249007801F82500D01C306001EB850572
:10DBD00090786870101D3060D078A870501D30604B
:10DBE0001279EA703B6A01F1500218E01C8F0020A4
:10DBF0002770002090950020E0290020C44D0020CF
:10DC000028700020E4950020A0950020F04400201A
:10DC1000E83F002028C1002004318A4207D008785C
:10DC20000028F9D18D78C8788542F5D20123114AB0
:10DC300083F00103012513702B46FEF788B80E4BC5
:10DC400010284FF0000228BF10201A605A609A6016
:10DC5000DA601A7400283EF494A83268013B10443C
:10DC60000132326012F8011C03F8011F8242F7D121
:10DC7000FEF787B8A023002072A4002038B50B4C13
:10DC800023688BB15A68821A002A054604DA0CE030
:10DC90005A68AA1A002A07DB9A68226018461A688E
:10DCA00090472368002BF3D138BD38BD8C44002049
:10DCB0002DE9F04F2DED028B9F4BA04A1C7897B0B9
:10DCC00000F59C41203181460B911160002C00F041
:10DCD00039859B4A1268904240F28380994A0892A3
:10DCE00016689949994A0791013C1C70984B059216
:10DCF00006F480560A93002E40F08180954B1B78E5
:10DD0000022B00F0D187042B00F08987012B00F053
:10DD10003D87914B99450A9B9B7800F2E283002B4B
:10DD200040F0E3838D4B0993089B1E6816F48057DF
:10DD300040F0D684DFF85492059BB3F90610079B98
:10DD40005C8BA142B4BF00240124854B1B6813F0F7
:10DD500080535ED0099A127812F001025FD00798C2
:10DD6000408C884241F3AC80002C5ED17D4D95F80B
:10DD70008C10002959D17C487C49006890F82D000E
:10DD800000250D604D608D60794900284ED10870E6
:10DD9000002A4FD0F1064DD5764A1278D20649D4E2
:10DDA000002F47D1002B45D1750243D4724B1B780D
:10DDB000002B01F0BA87714B9B78002C42F04D800C
:10DDC0003BB16F4A6F4B12681B689B1A002BC2F263
:10DDD00085801020634D2FF0DBFD012385F88D3009
:10DDE00028E0584B08931E68584B574A059306F491
:10DDF0008056574B07920A93002E3FF47FAF0021C5
:10DE000057480CF0C6FC00287FF478AF15F0EEF907
:10DE100074E770029ED4099A127802F00102514D03
:10DE2000002185F88C10002CA5D0514901200870E4
:10DE3000002AAFD1544B1A78002A40F0B3800799DA
:10DE4000059D488BB5F90070898BB5F90250874262
:10DE5000CCBF8026002646F040038F42A8BF334641
:10DE60009B0843F080068542C8BF3346059F43F0B8
:10DE700040068D42B8BF33469B08B7F90450B7F946
:10DE8000066043F080078542C8BF3B4643F0400729
:10DE90008D42B8BF3B469B0843F08007314D864218
:10DEA000C8BF3B4643F0400795F88EE08E42B8BFAE
:10DEB0003B469E4501F04D82A5F8902085F89220C2
:10DEC0002D4985F88E300E78002E01F070815F2B81
:10DED00001F0E9816F2B01F02882099B1B78DB0799
:10DEE00060D495F8921000295CD1B5F99030322BAE
:10DEF00058DD95F88E200120572A85F8920001F010
:10DF00008685089B1B685C0741F1BE805A2A41F058
:10DF1000BB8095F89430002B41F0F68695F896304A
:10DF200083F0010385F89630002B41F0AE870C207A
:10DF30002FF02EFD01F0CBB988440020484300208B
:10DF400084440020E084002028700020FCB90020D8
:10DF500098970020DC4A0020404B4C00B85200202B
:10DF6000B4930020102A0020585600201893002057
:10DF7000982F002056560020A023002090950020C6
:10DF80009C9200208C4600200789002040450020FC
:10DF90000F202FF0FDFCB5F8903085F89240FA3B49
:10DFA000A5F89030089BB44A1B680692B34C5F07F3
:10DFB00000F1EE840DF1500ADFF8E8820B940022A4
:10DFC000CAF804204546149240F6330B192740F254
:10DFD0008336059C02E004354D4522D0A978EB78C4
:10DFE000994217FB0160F6D295F801E00EF1040E9C
:10DFF00017FB036134F91E305B45A8BF5B46B3F5E0
:10E00000617FB8BF4FF461739842E4DA9942E2DB72
:10E0100029782729DFD8504604350CF0ABFB4D4555
:10E02000DCD1974A0B9C1378964A9AE8030082E861
:10E030000300002B40F01B81934B1F78002F00F052
:10E04000C38301218F480CF0A4FB002840F04E81CF
:10E050000A9BDB78002B40F0498123881DB225F014
:10E060000105AEB2B342268000F04386874D0227F9
:10E070000E204FF014094FF0FF082F7085F8019023
:10E0800085F802802FF084FC39467E4826880CF003
:10E0900080FB002800F0428126F001039BB2B342CE
:10E0A000238008D00E202F7085F8019085F802801B
:10E0B0002FF06EFC2688B70740F19987DFF8E8B1AA
:10E0C000DFF8E8A19BF80010DAF80400B50708BFF4
:10E0D00081F00201C1F340010AF032FF24216948B6
:10E0E0000CF057FB30B9099A1378590744BF23F055
:10E0F00004031370069B1B6813F00A0F1DD0052143
:10E1000060480CF046FB002800F0B08625886F07B9
:10E1100041F162805B4806210CF03BFB002800F0D7
:10E1200092866E0641F15080072156480CF031FB73
:10E13000002840F0EB85069B1B689D0600F1CB8311
:10E14000268850480C210CF024FB002800F08A811E
:10E1500046F48073B342238009D04C4B022514212E
:10E16000FF220E201D7059709A702FF011FC484B41
:10E170001B78082B00F082810E2B00F07F81089B1A
:10E180001B685E0548D5434B1B79002B00F092803D
:10E1900014213C480CF0FDFA002840F090802DF04E
:10E1A0002BFB01202FF036FB002835D0DFF8008153
:10E1B00000254FF0CC0902E0DDB2022D2CD809FB7E
:10E1C00005F76B1C58F80760002EF5D1032290F973
:10E1D000023002960192C2782F4951F82220009213
:10E1E00018463246334601212EF048FF034605EB20
:10E1F000450000EB0010079353B1314608EB800057
:10E20000CC2236F04AFC079B48F807300135EDB2C6
:10E2100020F0B4FF0028D0D1099B1B78DD0740F126
:10E2200090809BF800101D4D1D4ADAF80000012374
:10E2300001F001012B7013700AF082FE069B1D682D
:10E24000690700F1F280EA0600F12B8117B0BDECFE
:10E25000028BBDE8F08F98F8022098F803309A42BC
:10E26000C0F0BA8608F1040845453FF4E5AE98F8D9
:10E2700000102329F6D1EEE7F8550020545600206F
:10E28000A8580020B49300205E510020F44E0020D6
:10E29000A0950020045400205C800408B95200209E
:10E2A00004300020F0440020649200206892002096
:10E2B000F8640020099B1B78D8077FF570AF4FF4F6
:10E2C0000F701FF079FD0028A6D00EF071FE4FF4FC
:10E2D0000F701FF013FD00289ED00EF069FE4FF462
:10E2E0000F701FF00BFD0028EFD195E7069B1B6810
:10E2F0009A077FF5B2AE2688F3070FD446F00103E4
:10E300009E4223800AD0BB4B1421FF2202250E20FF
:10E310001D7059709A702FF03BFB268826F002037F
:10E320009BB2B34223803FF4C9AEB24B1421FF220B
:10E3300002250E201D7059709A702FF029FB268837
:10E34000BCE6AD4B1E78002E65D1AC4B1B68002B94
:10E3500061D0DFF8F882DFF8F89218F8030C99F82A
:10E3600000704146A8F1030525F0FCFE002800F0EE
:10E37000D285002F40F0238605F10801687925F049
:10E38000F1FE002841F099849D49A87A25F0EAFE23
:10E39000002800F0D385022F41F0A2849949E87B40
:10E3A00025F0E0FE002841F097849749287D25F06C
:10E3B000D9FE002800F0D385042F41F0A1849349B1
:10E3C000687E25F0CFFE002841F096849049A87F12
:10E3D00025F0C8FE002800F0D385062F41F0888480
:10E3E0008C4995F8230025F0BDFE002841F07C847F
:10E3F000894995F8280025F0B5FE002800F0D3855E
:10E40000082F41F04F84854995F82D0025F0AAFE8C
:10E41000002840F0D385824B01221A7032F016FAA0
:10E42000069B1D6869077FF50EAF032025F0D2FE1D
:10E43000002801F01E80238813F008067FF403AF44
:10E4400008200DF031FE7748774B0068186005987A
:10E450007649774A069D774BC0882D6808801660FC
:10E460001E60F0E626F480739BB2B34223807FF4F3
:10E4700074AE714B1B78082B7FF47EAE228822F09D
:10E4800040039BB29A4223803FF479AE594B022558
:10E490001421FF220E201D7059709A702FF078FA07
:10E4A0006DE6162025F096FE002800F06A87238886
:10E4B00013F400747FF4CAAE4FF400700DF0F4FD55
:10E4C000059E5848594D5849594A5A4BF688006894
:10E4D0002E80086014601C6017B0BDEC028BBDE894
:10E4E000F08F13B90A9A01239370544B0A9A1D783E
:10E4F00092F8214009931B2025F06CFE012C05F0B9
:10E500000108814600F0EA8605F002050A9A4C4EA1
:10E5100092F82030DFF83CA14A4F06959346052B30
:10E5200000F23587DFE813F0C100B7000600FF00F6
:10E530000101F400012C04BF05238BF82030B8F151
:10E54000000F12D0079B3088B3F918100022134631
:10E5500061F30F0260F31F4261F30F03059861F34B
:10E560001F430360032342600693374DDBF814100A
:10E570002A68914280F00B8647F230510322CBF893
:10E580001C108BF8202002200DF0A6FD14F02EFEAA
:10E590002968DBF81C200A440421CBF818208BF8EA
:10E5A0002010012C40F06C872A68DBF8181091428B
:10E5B00080F0ED869AF8000020B925F00BFE0028C7
:10E5C00040F0E5863A6822F002023A602A687388D1
:10E5D000642101FB03234FF480600022CBF810304C
:10E5E0008BF820208BF803200DF046FD9BF820309F
:10E5F00095E700BFF44E0020B9520020BC52002025
:10E60000B84E0020BD4E0020C24E0020C74E002054
:10E61000CC4E0020D14E0020D64E0020DB4E0020F4
:10E6200004300020FC550020F02F0020E42F0020B3
:10E63000E82F0020E02F0020A0950020B8520020F5
:10E640001C8F0020505600209C920020AE4E0020CF
:10E6500001000020A023002025F0C2FD012807D1E1
:10E66000B44D72882B68642101FB0233CBF8103063
:10E67000B9F1000F02D0B379002B4BD1012C00F07F
:10E680008686AC4DDBF810102A689142C0F00587F1
:10E6900001238BF82030012C3AD0F379012B46D09E
:10E6A00025F01EFD9BF8203039E7B8F1000FD3D1DB
:10E6B000069D4FF48060B9F1000F00F024830DF047
:10E6C000F3FC0A9A00231361002D3FF42DAB28467A
:10E6D0002FF05EF9089B1E6816F480573FF42AABB2
:10E6E0001D2195480CF055F800287FF423AB934B7F
:10E6F00003F1500903E00433994500F079861A7854
:10E70000262AF8D19978DA789142F4D2FFF714BB2F
:10E71000884D5BE725F0E4FC03224FF47A738BF815
:10E720002020CBF81C30834D2DE7824D39E725F0B2
:10E73000D7FC032240F6B8338BF82020CBF81C30EE
:10E740007C4D20E77E4F3B78002B01F0C3817D4B51
:10E75000DFF82482DFF824B2DFF824A207934546CD
:10E760005E46059099460EE019F804109847032C70
:10E7700028DC88B93B782AF8020F01349C4205F165
:10E78000040580F22A81072CE1B23046DBF8043020
:10E79000EADD984700B2EDE738F824206B88801A4C
:10E7A0004FF47A719B1A01FB00F040F6CA0290FB0D
:10E7B000F3F00844904240F2EE23A8BF104698427E
:10E7C000B8BF184600B2D5E7DFF8B8A1DFF8B881C6
:10E7D0005D4D0AF15A064FF0010951461AF8010C35
:10E7E00025F0C0FCF8B19AF804009AF802309AF8C3
:10E7F00003E000EB400105EB8101013BD1F8A020D3
:10E8000003EB4303434493420DD095F8CC2081F8A9
:10E810009CE009FA00F022EA0000C1F8A030C1F83B
:10E82000A47085F8CC000AF1060A5645D5D14749AF
:10E83000404A474B09681B78D2F80080DFF84C91BA
:10E840000C910B934FF0FF3B4FF0000AD9F80430C6
:10E85000002B37D01E78002E34D0D9F80820A8EB32
:10E860000202002A11DB384D012195F8CC2001FA73
:10E870000AF122EA010285F8CC20364A08F5FA703E
:10E880004FF0FF31C9F8080011600B9AD2B199F826
:10E89000002059780432D2B2002940F0178307993A
:10E8A0000598098B30F9122001F1C800824240F32B
:10E8B000B185254D9A7895F8CC3043FA0AF3D807FC
:10E8C00040F136860AF1010ABAF1040F09F10C0988
:10E8D000BCD1FFF7B6BB204B1B78980704D51F4D62
:10E8E0002B7D042B00F2E485268816F0300F3FF4D0
:10E8F00028AC10200DF0C0FB20200DF0BDFB184B04
:10E90000268800221A70174A1748184F184D002100
:10E910001160184A396000232960416081610360F9
:10E9200083604361C361136051609360536191617F
:10E93000D36106E49C920020B4930020F0440020B0
:10E94000B445002028700020102A00205C560020CA
:10E9500061970020DC03002056560020545C002004
:10E960009487002080880020308800206C2F0020B1
:10E970006030002058880020D4450020C451002079
:10E980000E2A0020C54D0020CC4F0408AC2A0020E0
:10E99000AA4D95F896305BB1099B1B78DE0707D529
:10E9A000059BB3F90620079B5B8B9A4200F3AF856A
:10E9B0001121A3480BF0EDFE002800F06F8295F8BE
:10E9C0009A302BB995F8943013B93223A5F89830C2
:10E9D000012385F89A30FFF7EDBADDF81490994AD3
:10E9E00008929949126842F2010AA1FB091B12EA36
:10E9F0000A0A4FEA9B1B00F04E82944D9448954CB6
:10EA000095492E780078267008701EB192490E78CC
:10EA100086F00106894D0F2185F82410002B00F0A7
:10EA2000F883079C8D4BB4F826C0B4F824E0079C0B
:10EA300010931846248B0078894B129495F8254042
:10EA40000994884C0F9005940446A3FB00035B08CF
:10EA500003EB4303E31ADBB2CDF834C002F4805277
:10EA60000C9397F80080DFF834C27E4C0E910BF5C2
:10EA7000967305F12800CDF844901392DDF82490A8
:10EA80000A930995002106967546069B002B00F017
:10EA90002183099B33F911201FFA82FEAE454FEA0C
:10EAA000410303D30D9EB64540F258835CF8212004
:10EAB000934580F01883E25EBAF1000F40F02D8399
:10EAC00001314145E25200F10600DEDB0E9A099D5C
:10EAD000654B85F824200F2A49460CBF01220022ED
:10EAE000DDF8449085F825101A7000F099835F4B8B
:10EAF0005749594ADFF8A8B10A931C46042001235C
:10EB00000B7013700DF0E8FADBF80030A168626852
:10EB1000E3605B1A934284BF002384F82130089B92
:10EB20003C781E68002C00F0ED87079A504DB2F833
:10EB300024E0178B4B4916F48056284640F0958305
:10EB400032460EE0437803EB830303EB830303F2C7
:10EB5000EE239BB20132A24221F8023B00F10200F7
:10EB60000ED015F81230002B00F0FC82022BE9D0F9
:10EB700001320B8821F8023BA24200F10200F0D1E1
:10EB8000109A137801331370FFF7B5B82B4DD5F8F1
:10EB90008830A9EB0303002BFFF6BBA8354A364BA0
:10EBA000527C079933F812308A7DDFED346A9FED8D
:10EBB000346AC97D9BB207EE102A07EE903AB8EE90
:10EBC000C77AF8EEE77A27EE267A67EE867A0B9A0E
:10EBD000C5F88820C7EE876A40F2FF32FCEEE67A7D
:10EBE000CDED067ABDF81830934228BF134609B11F
:10EBF000D31A9BB22348244D0178244C35F8116078
:10EC0000226825F81130921B13440131204D2360F6
:10EC100001F00F021B0902702B80FFF77AB8FBF797
:10EC2000A3F81C4B1C4A1B68C31A93427FF771A8B8
:10EC3000174B00221A80FFF76CB800BF102A002083
:10EC4000B4930020E0840020D34D621024430020C0
:10EC5000D000002061970020D1000020A5440020B2
:10EC6000ABAAAAAAFCB90020C251002098970020A4
:10EC700008460020A4920020C49200200000C84250
:10EC800000008044DD4A0020E44A0020E04A0020E1
:10EC9000C6A60020002A002060E31600A844002039
:10ECA0009C9200206F12833F079A0599537DD27D75
:10ECB000013B31F913301AB1C3F53B6308331BB282
:10ECC000A3F57A7307EE903A1FED0A7AD14AF8EE6F
:10ECD000E77A40F2FF3167EE877AFCEEE77ACDED16
:10ECE000067ABDF818308B4228BF0B461380FFF719
:10ECF00010B80221C8480BF04CFD00283FF40EABC1
:10ED00002580FFF7D8B90DF0B7F9DAE4C34AB2F9B4
:10ED10000030002BB8BF5B42B3F5E17FBFF60BAA12
:10ED2000B2F90230002BB8BF5B42B3F5E17FBFF60A
:10ED300002AABB4B93ED057AD3ED077AD3ED096AAE
:10ED400093ED030A77EEA67A30EE070AF7EE000A93
:10ED5000B0EE007AE7EEC70A30EE000A0BF066FA72
:10ED6000B6EE008A20EE488A9FEDAE0A38EE000A21
:10ED7000FDEEC07A17EE903A2033402B40F2D58357
:10ED80009FEDA90AA94ADFEDA87A82ED000ABDEE3F
:10ED9000C87AC2ED017A17EE103A2033402BC2ED4B
:10EDA000027A49D8DFEDA27AB4EEE78AF1EE10FAE2
:10EDB00040F3B787DFED9F6A9FED9F7A01E0B0EEE9
:10EDC000678AB4EEC78AF1EE10FA78EE667AF6DC5E
:10EDD0009FED9A7AF4EEC77AF1EE10FA40F19D8732
:10EDE0009FED946ADFED966A01E0F0EE477AF4EE6B
:10EDF000E67AF1EE10FA37EE867AF6D4DFED897A0C
:10EE0000B4EEE77AF1EE10FA40F35786DFED887A38
:10EE100037EEC77A27EE076ADFED8A5ADFED8A6A96
:10EE2000DFED8A7AE6EE256A67EE065AE6EE267A86
:10EE3000A5EEA77AF0EE477A0A20C2ED037A2EF00B
:10EE4000A7FDFFF778B925F040039BB2AB422380C2
:10EE50003FF46AA97E4B02251421FF220E201D706B
:10EE600059709A702EF094FDFFF75EB9238823F055
:10EE70000405ADB2AB4225803FF44CA9744B02258A
:10EE80001421FF220E201D7059709A702EF080FD03
:10EE90002588FFF73FB96F490E78B6E595F89430AD
:10EEA000002B3FF487A8099B1B7813F001037FF424
:10EEB00081A8012285F8943085F89520FFF77AB86B
:10EEC000654D012185F88C10FEF7AFBF012900F0D8
:10EED0005A85BBF1FF3F604D0BD01B780C2B08D03F
:10EEE0005E4B5F4A03EB86065E4BC3F800B0736C63
:10EEF000136095F8CC20012303FA0AF30AF1010A02
:10EF00001343BAF1040F85F8CC3009F10C097FF4F2
:10EF10009DACFFF796B808F10501687925F022F954
:10EF200000283FF431AA012F40F0C78605F10D01FA
:10EF3000A87A25F017F9002840F0D2864A49E87BE4
:10EF400025F010F900283FF430AA032F40F0C486C2
:10EF50004649287D25F006F9002840F0D18644492D
:10EF6000687E25F0FFF800283FF430AA052F40F016
:10EF7000C3864049A87F25F0F5F8002840F0B88600
:10EF80003D4995F8230025F0EDF800283FF430AA1C
:10EF9000072F40F0A986394995F8280025F0E2F8B6
:10EFA000002840F07F86364995F82D0025F0DAF8E4
:10EFB00000283FF430AA092F3FF42DAA0926334632
:10EFC00003EB83031D442F4B6978AA7889F800600E
:10EFD00019705A70FFF71FBA0F480BF0DAFB0028C0
:10EFE0003FF42AA814202EF0D3FCFFF725B846F0F2
:10EFF0000203B34223803FF461A8154B0220142181
:10F00000FF2218700E2059709A702EF0C1FC2688CD
:10F01000FFF754B8C6A60020B49300200456002081
:10F02000D8010020DB0FC93F000000008000002055
:10F03000DB0F4940DB0FC940E4CB1641DB0F49C071
:10F04000E4CB16C192E741B99730083C15A82ABE17
:10F05000F44E002061970020102A0020CC4F0408B5
:10F0600084A40020DC030020BD4E0020C24E0020FE
:10F07000C74E0020CC4E0020D14E0020D64E00209E
:10F08000DB4E0020C05200205D2A00F056825B2A31
:10F0900000F03C855E2A00F07585562A00F0A585B3
:10F0A000972A00F00E86A72A00F07085BB4C2388B3
:10F0B0009B0740F02F85A2F1B703072B00F2678270
:10F0C000DFE813F05F02650265026502590265021E
:10F0D0004B024B02002D3FD05CF8212093454FEAB4
:10F0E0004103FFF4E8ACAE4AAD4ED25C06EB030E32
:10F0F000002A00F0AE80022A47D19EF8012002EBE0
:10F10000820202EB820202F2EE2292B2032933DD86
:10F1100012B2BAF1000F3FF4D3AC0C9E20F81620C7
:10F12000B9F1000F03D10F9E022E7FF6C9ACB0F8E3
:10F1300000904288B0F804E04A449644994A0FFA95
:10F140008EFE82FB0E62984EA2EBEE7226F803E072
:10F1500012B24FF00109B3E42A464B000A9E4CF864
:10F160002160A9E4D3B2022B04D9032B7FF400ADB4
:10F170007346EFE43B46EDE4012606FA01FE0E9EDF
:10F1800026EA0E0612B20E9696E4E25ABEE7874AC7
:10F190001278002A7FF4F0A9B8F1000F3FF4ECA92F
:10F1A000012C40F0F4809BF82030FFF7B8B93146CD
:10F1B0007F480BF0EEFA002800F0938085F893600A
:10F1C00014F048FCFEF789BE45F04003AB422380B3
:10F1D0007FF440AEFEF7A8BF45F004039D422380B4
:10F1E0000AD0744B02251421FF220E201D70597085
:10F1F0009A702EF0CDFB25886F4B704AB3F904301E
:10F200006F4982FB0302DB17C3EBA2030B80FEF7FF
:10F2100081BF6C4B6C4A109201221A706B4B0593A4
:10F220001B2163480BF0B5FA00287FF460AC684BF3
:10F23000DFF8B8B10A931946DBF80030CA688B6072
:10F240009B1AC82B00F24F84089B1E6806F4805658
:10F2500096E4CAB2022A40F29383032A95D1129A05
:10F26000139E002E08BF2A4650E700220FE0437885
:10F2700003EB830303EB830303F2EE239BB2013220
:10F28000A24221F8023B00F102003FF479AC15F8EC
:10F2900012301BB1022BEAD00B88F0E7D3B2032B5C
:10F2A000FAD83B46EBE7B2F5FA7FFEF67BAE95F86F
:10F2B0009230002B7EF476AE099B1B78012213EA74
:10F2C000020485F892203EF463AE13F08FFF414BA9
:10F2D0000693089B314C1B68FEF769BE0025FFF7BB
:10F2E00015B9099B3C4A1B781060D8077EF5F9AD2B
:10F2F0003A4B1B78002B3EF455AE0A9BDB78002B73
:10F300007EF450AE95F893300133DBB2032B85F8D1
:10F3100093307EF647AE324B5B7813B9002C7EF407
:10F3200041AE13F063FFFEF7D8BDB2F5FA7FFEF6EB
:10F3300039AE95F89220002A7EF434AE099B1B78F2
:10F34000012185F89210D90700F1AE8314F082FBF9
:10F35000BDE7244A24491068B5F99020C66981FBAD
:10F3600006018911F617701A00F5FF407F308242BE
:10F370003EF7A6AD891B0A4412B2A5F89020FEF70D
:10F380009FBD4FF400700CF077FEFEF75FBF069D47
:10F39000002D3EF4C9ACFFF79AB900BF54560020C7
:10F3A0000846002056555555802A0020882F0020F9
:10F3B000B4930020F44E0020045600206766666671
:10F3C000A0880020C2510020A5440020FCB90020E4
:10F3D00098970020F8550020904600206197002063
:10F3E0009095002028A90020D34D62109C92002007
:10F3F000BA4A079BD488059A1B8BB2F906101A1BD0
:10F40000914240F3818023449942B4BF00240124F7
:10F41000FEF79BBCC8398A42B14D66DA9A7895F8F6
:10F42000CC3043FA0AF3D9073FF54CAA52420120E7
:10F430000D922EF0D3FB731E0D9A162B00F29A83B9
:10F44000DFE813F056023D0222026F020E02F701BE
:10F45000E001AF019501C6017B0198036F026601CF
:10F46000F701E001AF013201190100018502E70057
:10F47000CF0008200CF000FE069B1D68FEF7E3BEDF
:10F48000AB460A99DBF80020CB69069D13448B61DB
:10F49000002D3EF449ACFFF71AB924F021FE0321F8
:10F4A00040F6B8328BF82010CBF81C20FFF76BB871
:10F4B0000A2024F08FFE26880746002800F0D48218
:10F4C000F10640F1A183864D95F8D470002F7EF4AB
:10F4D00038AE0D202EF05CFA012385F8D430268852
:10F4E000002F7FF410AAFEF72CBE95F8CC30012235
:10F4F00002FA0AF223EA020308F5FA7285F8CC3020
:10F50000C9F80820FFF7DEB90124FEF71EBC002170
:10F5100074480BF03EF900287FF44AAA322385F89C
:10F520009600A5F89830FFF743BA0AF0F5FD29E4F4
:10F53000002A0CBF012002207AE76B4B0022012039
:10F540006A496B4C0B606B4B227006932EF046FBA6
:10F55000089B694C1B68FEF72ABD684A6849644BE2
:10F56000116002225A70634B069324F097FE089BA9
:10F570001B68FEF71CBD614A624911605C4B0022AA
:10F58000F0E75E4A60491160594B0122EAE7792AA7
:10F5900000F03F847A2A00F035849E2A00F02A8405
:10F5A0009D2A00F0F583AE2A00F0EB83AD2A00F02F
:10F5B000E183EF2A00F0DB83FD2A00F0C683FB2AFB
:10F5C00000F05D84FE2A00F05784F72A00F0518491
:10F5D0007B2A00F02584089B464A1B680692FEF7AA
:10F5E000E6BCD5F8D000494F90F836B0BB789344CC
:10F5F000BBF1640FA8BF4FF0640B2BEAEB7B80F8E4
:10F6000036B0002B40F0448423F0F8FED9F80430E3
:10F6100063E4D5F8D0003D4F90F837B0BB78934401
:10F62000BBF1FE0FA8BF4FF0FE0B2BEAEB7B80F87F
:10F6300037B0002BE8D01620594624F015FED5F837
:10F64000D000E1E7D5F8D000304F90F802B09344F5
:10F65000BBF1C80FA8BF4FF0C80B2BEAEB7B80F8BB
:10F6600002B0BB78002BCFD01420594624F0FCFD0B
:10F67000D5F8D000C8E7D5F8D000244F90F801B0F5
:10F680009344BBF1C80FA8BF4FF0C80B2BEAEB7B2C
:10F6900080F801B0BB78002BB6D01320594624F077
:10F6A000E3FDD5F8D000AFE7D5F8D000174F90F8BC
:10F6B00000B09344BBF1C80FA8BF4FF0C80B2BEAB2
:10F6C000EB7B80F800B0BB78002B9DD01220594610
:10F6D00024F0CAFDD5F8D00096E700BF008F0020C7
:10F6E000102A0020B4930020F8BF002058560020B4
:10F6F000FC7B0020F8550020545600205C5600206A
:10F70000845100206C51002078510020C0A60020B8
:10F71000CE4F0C99BB7891F805B09344BBF1640FC0
:10F72000A8BF4FF0640B2BEAEB7B81F805B0002BF0
:10F7300040F0BA83D5F8D00066E7D5F8D000C34FC3
:10F7400090F808B0BB789344BBF1C80FA8BF4FF046
:10F75000C80B2BEAEB7B80F808B0002B3FF454AFCA
:10F760000B20594624F080FDD5F8D0004CE7D5F8A1
:10F77000D000B64F90F806B0BB789344BBF1C80FE9
:10F78000A8BF4FF0C80B2BEAEB7B80F806B0002B2C
:10F790003FF43AAF0920594624F066FDD5F8D00071
:10F7A00032E7D5F8D000A94F90F805B0B978934466
:10F7B000BBF1C80FA8BF4FF0C80B2BEAEB7B80F85A
:10F7C00005B0002940F07883112E7FF43EAF1BE78F
:10F7D000D5F8D0009D4F90F807B0BB789344BBF1AB
:10F7E000C80FA8BF4FF0C80B2BEAEB7B80F807B01F
:10F7F000002B3FF409AF0A20594624F035FDD5F817
:10F80000D00001E7D5F8D000904F90F804B0B97857
:10F810009344BBF1C80FA8BF4FF0C80B2BEAEB7B9A
:10F8200080F804B0002940F00F83102E7FF426AF3B
:10F83000EAE6D5F8D000854F90F803B0B978934444
:10F84000BBF1C80FA8BF4FF0C80B2BEAEB7B80F8C9
:10F8500003B0002940F039830F2E7FF428AFD3E6A0
:10F860000C997A4F91F807B0BB7893448BF3080B4F
:10F8700081F807B0002B3FF45DAF0520594624F016
:10F88000F3FCD5F8D000BFE60C99704F91F804B0A6
:10F890009344BBF1640FA8BF4FF0640B2BEAEB7BE2
:10F8A00081F804B024F0FAFCBB78002B3FF442AF9F
:10F8B0000320594624F0D8FCD5F8D000A4E60C99D2
:10F8C000624F91F802B09344BBF1640FA8BF4FF0B0
:10F8D000640B2BEAEB7B81F802B0BB78002B3FF482
:10F8E00029AF0220594624F0BFFCD5F8D0008BE6A2
:10F8F0000C99564F91F800B09344BBF1FA0FA8BF92
:10F900004FF0FA0B2BEAEB7B81F800B0BB78002BB1
:10F910003FF410AF0120594624F0A6FCD5F8D000E2
:10F9200072E60C98494F90F806B0B9789344BBF151
:10F93000640FA8BF4FF0640B2BEAEB7B80F806B096
:10F94000002940F0AA820D2E7FF4E3AEF2E60C9976
:10F950003E4F91F801B09344BBF5967FA8BF4FF49A
:10F96000967B2BEAEB7B81F801B0BB78002B3FF450
:10F97000E1AE1520594624F077FCD5F8D00043E6D7
:10F98000129AFFF7C3BB059993F802B031F9122020
:10F99000B2F5617F4FF4966191FBFBF17BDB40F6A2
:10F9A000330B9345A8BF93460C2EABF5617B9BFBB5
:10F9B000F1FB5FFA8BFB00F03D81182E40F0908048
:10F9C0005A46C82AA8BFC822214DD5F8D01091F8B0
:10F9D00017E0D0B270453FF480AAB2EB0E021B4F85
:10F9E000C87548BF0732D210B978531CDBB239B999
:10F9F00013B118462EF0F2F8D9F80430FFF76DBABB
:10FA0000594618200D9324F02FFC0D9BF0E7114B65
:10FA100011491A684FF47A73B3FBF2F3C3EB431244
:10FA200003EB8202089B1B68D2001F06A1F8A820E6
:10FA300000F1B880094A0692126855077EF5B6AA09
:10FA4000074A084C0A211180FEF7B1BAC0A600206F
:10FA5000102A0020D0840020F47C0020F8550020DB
:10FA600092C4002054560020F20600F113810B20AE
:10FA700024F0B0FB002840F0DF80B30600F11681CF
:10FA8000C74D95F8D430002B3FF423AD002F7EF402
:10FA90003AAFFEF756BB0C2E00F09380182E1DD106
:10FAA0004FF0000B5A468FE7BE49089B0A60BE4ADA
:10FAB0001B680692BD4CFEF77ABADFEDBD7AB4EE54
:10FAC000E77AF1EE10FA44BFDFEDBA7A37EEC77A83
:10FAD000FFF7A0B9B84A0792FEF781BF4FF0000BBD
:10FAE000AF4DFFF7FAB9B54A089B1E68136823F0BB
:10FAF000040313600A9A012306F4805682F8213029
:10FB0000FFF73EB806F48056FFF73AB8AC4B012237
:10FB1000022015E50023BB2A149300F09281B72A36
:10FB200000F08B81BE2A00F08681BD2A7FF42FADC4
:10FB30004FF6FE71A34A9C48D689069090893344BB
:10FB400001449181D38111F0B3FA09F01FFE11F045
:10FB500097FAF8F785FF01202EF040F8B5F89020CD
:10FB6000089BFA3A00211B68A5F8902085F89210AE
:10FB7000FEF71DBAD5F8D00023F040FC4FF0FF3B54
:10FB8000FFF7B7B9904B02220320D9E48F49089BB5
:10FB90000A7885481B68069042F004020A70834C7C
:10FBA000FEF705BA894A127896077FF543AF884A6F
:10FBB000127D042A7FF63EAF21F000F9089B1B68F6
:10FBC00038E70025AB46834A5278AA4288D0824F54
:10FBD000284614F059FDBB781BB159460C2024F07F
:10FBE00043FB6B1CDBB26E4D02E711F061FA09F0CA
:10FBF000CDFD11F045FAF8F733FF01202DF0EEFFAF
:10FC000095F88E20FFF74CBA10200CF04DFA20200A
:10FC10000CF032FA7149081F19F05CFD704B02229A
:10FC20001A705F4D95F8D430002B00F02B81268898
:10FC3000FEF769BE5D46C6E76A4A6B4B528993ED93
:10FC4000007A07EE902AF8EEE77AB0EEC77AB4EEC3
:10FC5000E77AF1EE10FA7FF510AF93ED017AB0EE8E
:10FC6000C77AF4EEC77AF1EE10FA7FF706AFB30663
:10FC70003FF506AF20200CF017FA95E80C005B4921
:10FC80000A60084641F8043F19F024FD544B012254
:10FC90001A70C6E710200CF0EFF9514B26881F7040
:10FCA0000127E4E608263346FFF78AB920200CF046
:10FCB000E3F94B4B00221A70B3E701263346FFF7F6
:10FCC0007FB939494A4A089B06914FF4C8711B68AD
:10FCD0001180364CFEF76BB903263346FFF770B937
:10FCE00002263346FFF76CB907263346FFF768B99B
:10FCF00006263346FFF764B905263346FFF760B999
:10FD000004263346FFF75CB9274B85F8941085F835
:10FD100095000693254CFEF73CBEB0EE677AFFF7E0
:10FD20006DB8F0EE487AFFF753B8002C3EF451A8B6
:10FD30001B4D95F88D30002B3EF47CA82DF00CFE69
:10FD4000002385F88D30FEF775B80021012014F0EE
:10FD5000C5FBB5F89020089B13491B680691963A9D
:10FD6000A5F89020002285F89220FEF720B9002106
:10FD70000846ECE7FF2100201BF06DF995F88E2076
:10FD800017E4012100201BF066F995F88E200DE4A0
:10FD90000021FF201BF05FF995F88E2003E400BFDF
:10FDA000102A002090460020F855002054560020CC
:10FDB000DB0FC9BFDB0F49C0287000205056002060
:10FDC00046C000207095002094C0002056560020A8
:10FDD000545C0020FC7B0020C0A600208C87002003
:10FDE000948700202488002014540020E429002057
:10FDF00094C40020002101201BF02DF995F88E20DD
:10FE0000FFF7CEBB394A137A43F001031372FFF7B1
:10FE1000E2BB364A137A23F001031372FFF7DBBB10
:10FE20004FF4FA61022014F059FB314B0693089B02
:10FE30001B68FEF7BCB802217CE619464FF6FE733C
:10FE400078E61946022375E6102059460D9224F0F3
:10FE50000BFAD5F8D0000D9AE7E4002B3FF468AF19
:10FE60002449254A09684FF47A7000FB0313136094
:10FE70005EE7002104206AE70021032067E70021F4
:10FE8000022064E70127FFF724BB0B20FEF750B8E0
:10FE90005946172024F0E8F94CE459460D200D92FC
:10FEA00024F0E2F90D9A4EE50E20594624F0DCF9D3
:10FEB000D5F8D000FFF7A8BB112059460D9224F0C9
:10FEC000D3F9D5F8D0000D9A7EE40F2059460D9253
:10FED00024F0CAF9D5F8D0000D9ABDE4074D13F00F
:10FEE00085F9002385F88D30FDF7A4BFAC8800208C
:10FEF000F85500209C9200208C460020102A0020FB
:10FF00002DE9F047C74C636820469847002800F069
:10FF1000C380C54B1B780122042B84F83C2000F0E1
:10FF2000BD80B4F91610B4F91820B4F91A30216361
:10FF30006263A363BD4B1B88002B69D0BC4DD4ED1D
:10FF40000C7AD5ED004A95ED050A95ED015A95ED2F
:10FF5000067AD5ED035A95ED026AF8EEE76AD5ED1B
:10FF6000047AA4EEA60AA5EE267A67EEC07AA5EE7C
:10FF7000C07AE6EE267A85ED057AC5ED067A33F08D
:10FF8000CFFDD4ED0D6AD5ED094A95ED0E0A95ED3C
:10FF90000A5A95ED0F7AD5ED0D7AD5ED0C5A95EDFF
:10FFA0000B6A2063F8EEE66AA4EEA60AA5EE267AAE
:10FFB00067EEC07AA5EEC07AE6EE267A85ED0E7A77
:10FFC000C5ED0F7A33F0ACFDD4ED0E6AD5ED124AD3
:10FFD00095ED170A95ED135A95ED187AD5ED167A29
:10FFE000D5ED155A95ED146A6063F8EEE66AA6EE53
:10FFF000A40AA6EE857A67EEC07AA0EE657AE6EEF0
:020000040801F1
:10000000867A85ED177AC5ED187A33F089FDA063FD
:10001000884FA17F884815F097FE3B88002B40F061
:100020008480864ED6F8D850854B1B685B0743D436
:10003000B5F90070216B636BA06B824A824E92ED22
:10004000026AD2ED006AD2ED015AC91B2163B5F9EB
:100050000270DB1B6363B5F904703568C01B07EEE3
:10006000900AB8EEE75A07EE901AB8EEE77A07EE74
:10007000903AF8EEE77A36EE056A36EE877A77EE52
:10008000A57A0135A06382ED026A82ED007AC2EDA5
:10009000017A3560BDE8F087BDE8F0876B4BB4F9B5
:1000A0001600B4F91810B4F91A201880206359808A
:1000B00061639A80A2633DE7B6F89820322A00F087
:1000C0008880002A66D196F89530002BB0D0604821
:1000D000D6F8F4205F4980FB0273D217C2EB2312DB
:1000E0002A80D6F8F82080FB0273D217C2EB2312C5
:1000F0006A80D6F8FC30A78A80FB0302DB17C3EBCB
:100100002213DB1BAB800023CB6086F8953010F008
:10011000CFFF09F03BFB10F0B3FFF8F7A1FC012083
:100120002DF05CFDD6F8D85082E7444E226BD6F80D
:10013000D850B3F5C87F4FF0000323632B80398874
:1001400018BFD6F8DC00B7F8008008BF0020B1F572
:10015000C87F18BFD6F8E030616B02440B44002022
:10016000B8F5C87F6063C6F8DC20C6F8E030688068
:1001700052D0D4F838E0D6F8E410A0637144B8F156
:10018000010FA880C6F8E41068D008F1FF38A7F87E
:10019000008049E7D6F8F400236B00210344C6F839
:1001A000F43021632980D6F8F800636B616303445F
:1001B000C6F8F8306980A36BD6F8FC00A16303444D
:1001C000012AC6F8FC30A98075D0013AA6F898201B
:1001D00079E72B8820491F48276BA6F8E8300023D1
:1001E000B5F802E0B5F804C0C0684B608B602363CB
:1001F000C6F8F4702B80616BC6F8F81063636B80EF
:10020000A16BC6F8FC10A363A6F8EAE0A6F8ECC060
:10021000C6F8F000AB80D8E7A36BC6F8E430A06363
:10022000A880B2E70C560020D59200204E4700204F
:100230005047002094C400203C560020102A002083
:10024000E08400205889002054890020D8920020A2
:100250001F85EB5170950020042B0020DFF88CC027
:10026000DFF884E0C8328CFB02A9C833D217C2EB96
:10027000E9128CFB03A9DB17C3EBE913C8316B80D0
:100280002A808CFB013CA28ACB17C3EBEC139B1A90
:10029000AB80CEF80C0010F00BFF09F077FA10F0ED
:1002A000EFFEF8F7DDFB40462DF098FCB7F8008034
:1002B000D6F8D85069E70B2086F89A1086F8942073
:1002C0002DF066FBD6F8D850074BB6F8E820B6F804
:1002D000EA70B6F8EC00D6F8F0102A806F80A8809B
:1002E000B6F89820D96070E7709500201F85EB5113
:1002F0002DE9F0478C4B1B78DB07074644D58B4B29
:100300008B4D1C788B4E012C59D01CD3022C07D15D
:1003100089498A4A09881288914201D901241C70AE
:10032000EB7AE3B12B89D3B1854B1B78BBB10CF0D1
:10033000A5FA002800F09B802B7B83422CBF012173
:10034000002131700CE07C497E4A098810886A7B64
:10035000801A8842E2DAEB7A0024002BE2D131786D
:100360002A79632A06D8022C774E00F0BA803378B7
:10037000002B5DD1754AAB7A8C4238BF0C461470A5
:10038000002B4CD1BDE8F0876B4B694D19885B8819
:10039000E878CB1A83EAE3728142A2EBE3721DD3C1
:1003A0002B788B421AD3614B1C78E01E012861D94F
:1003B0006749097802294FD0012C5E4EA5D15F4ACA
:1003C0005D491288687B0988121A914239DD5D4ABD
:1003D00012888A42A4D200241C70A1E7B1EB400F1E
:1003E000E1DC524B1C78E11E012940F29480022A84
:1003F000DEDC57494F4E0878DFF84481DFF844C10E
:10040000DFF838E100210324022834701C7088F8DA
:100410000010ACF80010AEF8001081D11FE0012CE4
:1004200071D0022C0BD10720BDE8F0472DF0B0BAF7
:100430007068381A474B984258DD72709AE7BDE8E9
:10044000F08702241C706BE7022AD2DD404909784C
:1004500002294FF0040464D13949364E09783E48E8
:10046000022ACCBF00220122C28081804BE70221F8
:10047000317075E7022A9BDC95F800C091FBFCFC0B
:100480000CF1010CBCF1080FDFF8B4A0304EA878D5
:1004900095F801E096F800802A4CDFF8A090254EF0
:1004A000A8BF4FF0080C8AF800C01FFA8CFA10FBA6
:1004B0000AF01EFB0AFE80B2DFF88CA02080A9F8AB
:1004C00000E000244FF0640EB8F1020F34701C708D
:1004D000CAF804408AF801E07FF439AF0FFA8CF1D2
:1004E000BDE73078A0B9012377603370C2F16402B0
:1004F0001A4B00FB02F083FB0023C017A0EBA350B4
:100500006430707036E70820BDE8F0472DF040BA3F
:100510007368F81A8EE7032C96D10D4909780229E1
:100520009AD0044EFCE600BFB8520020683100208B
:10053000DC5500206E310020FC5300206C3100207F
:10054000125400206A310020C82F0020E0A60020AD
:10055000D59200207F969800D89200206BCA5F6BDE
:10056000022828BF022010B4084C094B207000EB71
:100570008002C0EBC20207495DF8044B013003EB77
:100580004203C0B20B602DF029BB00BFFC7B0020F2
:10059000F8BF00205856002008B510F089FD09F07A
:1005A000F5F810F06DFDF8F75BFA0120BDE80840A2
:1005B0002DF014BB1C4C08B501210220F9F7D6FE22
:1005C000237803F00502052A29D003F00903092B3B
:1005D00008D000210120F9F7C9FE00210846F9F7EB
:1005E000C5FEFEE7114A124B11681A680B68114CE0
:1005F00023F001030B601388206823F001031B0420
:100600001B0C138018B12A2200238271C3710922A6
:100610004A21F8F73FFE206808F088FCD9E723F06C
:1006200057F92378D1E700BF3C3F00207C31002000
:10063000803100202440002008B5F8F7A9FB10F015
:1006400037FD09F0A3F8BDE8084010F019BD00BF60
:1006500008B510F02DFD09F099F8BDE8084010F03C
:100660000FBD00BF2DE9F04FBC4B1E788BB0002EA4
:1006700040F08180BA4BBB4C1D78BB4FDFF80CB308
:1006800005F00105A4F10A0954F80A0CB8B14FF0BD
:10069000CC0808FB0698F9F751FE80B154F80A0C13
:1006A000F9F744FE14F8023C024683B924283BD0F3
:1006B00075B354F80A0CF9F741FE0028EED1013663
:1006C000032E04F1CC04DFD10BB0BDE8F08F012B79
:1006D0002ED0022B33D0032B40D0042B00F06981A5
:1006E000052B00F05781062BE3D114F801ECBEF185
:1006F000000F00F0DC81BEF1010F00F01F82013617
:100700000023032E04F8023C04F1CC04BCD1DBE747
:10071000232A54F80A0C00F08281944B93F832306B
:100720009342B8D131F040FF012304F8023CC0E706
:100730004D2800F06781002304F8023CB9E700234C
:100740003C2804F8023C00F057813E28B1D1012238
:10075000032304F8012C04F8023CAAE7C028EAD8D5
:100760000021042304F8050C04F8040C04F8061C0A
:1007700004F8023C9DE77E4B18680028A4D008F0DE
:10078000F4FEDFF80CA27B4DDFF8F891DAF80000F8
:10079000F9F7D4FD002897D0DAF80000F9F7C6FD84
:1007A00009281BD03F2819D02B68002B67D10428BB
:1007B00000F0BE810C2800F0CA807F28E6D0A0F1AE
:1007C0002002D2B25E2AE1D80BB92028DED05A1C12
:1007D00009F803002A6023F0EBFFD7E72C68002C10
:1007E0005AD1654FA34607F52078BBF1000F08BF2B
:1007F000BB4610374745F8D1BBF1000F00F05281DE
:10080000103FDBF800003A68065D135D9E4220440D
:1008100002EB040140F04481661E4E4422460BB9AF
:10082000FD2A5CD906F8013F01322A6010F8013F29
:1008300011F801EF9E45F2D00AB15F4512D04F4842
:1008400023F0BEFF5F4508D35BF8100B23F0B8FF21
:10085000092023F0ADFFBB45F6D9494823F0B0FF8E
:100860002A680024944291D2661E4E4416F8010F65
:1008700023F09EFF2B6801349C42F7D386E70C28B7
:1008800065D00A2834D00D2832D07F2800F0BE80F1
:10089000FF2B3FF67BAF92E7374E002706F5207817
:1008A000BB4602E0103646450DD022463168484628
:1008B00009F0B4F90028F5D1B346002FF2D137463C
:1008C00010364645F1D13B465F469B46002B98D1FA
:1008D000002F3FF45BAF294823F072FFB4E7511CAF
:1008E000202009F80200296009F801300A46A4E72F
:1008F00023F0E7FF2321234834F0E6F8002800F036
:100900001581A0EB0900286090B1431E19F803106F
:10091000202940F0308109EB030243B112F8011D98
:10092000202903F1FF304FD10346002BF6D12B6075
:100930004FF480720021484634F0AFF8074B1B7823
:10094000002B3FF4C1AE0E4823F03AFF1EE70E48DD
:1009500023F036FF0A4823F033FF17E75E510020EB
:10096000B852002002650020102A00205470002098
:10097000F04E0020A0410020A06C04082C87040841
:1009800034870408A04000203C8704087450040801
:100990009C40002014F8063C14F8051C994273D8BA
:1009A00014F8043C83427FF4C6AE062304F8023CEC
:1009B0009BE614F8043C04F8030C5A40052304F8A1
:1009C000042C04F8023C74E62B606C4C002204F505
:1009D000207809F8032002E01034444550D0216803
:1009E00048460EF0F5FE0028F6D0444548D2E368AC
:1009F000984700232B609BE7032204F8013C04F88E
:100A0000022C56E6022304F8023C52E6013B002287
:100A10005B482B6009F8032023F0D2FEB6E6594B61
:100A20005949DB78594ADFF890E11060003318BF6C
:100A300001230B70564B574ACEF80030564BC7F87F
:100A400004214FF0400E012187F80CE1C7F80001A6
:100A5000C7F8080187F80D515048197024F08CFA36
:100A60004F4823F0ADFE4FF400600BF035FB4D4BCB
:100A700093F83230232B3FF455AE14F8023C32E6A3
:100A8000494823F09DFEB4E714F8041C08EB03006A
:100A90005140013304F8041C04F8063C827208E655
:100AA0002246C9E64148103F23F08AFECCE69BE887
:100AB0000F000DF1280C0DF1080888E80F004CF824
:100AC00024ED14F8053C14F803AC06946246234464
:100AD0004FF0010C414606A8ADF822E00793ADF8AF
:100AE00020A08DF824C0FBF78BF840B1029A304B60
:100AF00003924146A4F10A0002930CF0CDF8DDF810
:100B00000480002304F8023CB8F1000F3FF4D7AD95
:100B100054F80A0C0CF082F9013654F80A0CC0475C
:100B2000032E04F1CC047FF4AFADCDE52868EBE6ED
:100B300020480DF095FD0BB0BDE8F08F14F8053C92
:100B400014F8032C0694234407936E2A4FF00003F5
:100B500008930993ADF820207FF4D1AD06A809F0E1
:100B6000DCF806A809F0CEF806A809F0CBF806A82C
:100B700009F0C8F8C3E5034627E700BFA06C0408E6
:100B800064870408FC7B0020F43100209C40002096
:100B9000142B0020E98300085E51002068870408B8
:100BA0003487040854700020488704082C87040800
:100BB000BCC40020A0400020F04E00202DE9F04FE2
:100BC0002DED028B95B006462AF016FE9E4B1D7841
:100BD00025B115B0BDEC028BBDE8F08F9B4B1B68B7
:100BE0005805F6D5DFF8B092D9F80020002A00F0B9
:100BF0002781974CD4F8283103F5F43348339E42CB
:100C0000C0F01E81934F94F82C113B68C4F8286102
:100C1000013184F82C11990701F1798713F0140F31
:100C200041F0178713F0080F94F82C3140F0C2817F
:100C300013F0070801F0BA85282B874B029302F0C6
:100C4000B1805E209047854B1B78002B6BD0804C89
:100C5000834AD4F83431F31A934201F24384DFF823
:100C60003CA29AF80080B8F1000F33D1DFF800926F
:100C7000D9F80000F9F762FBC0B201280ED90228AA
:100C8000784F42F04F813B78002B42F02A82D4F813
:100C90003C31F31AB3F57A6F82F0D5827248076857
:100CA000002F40D09AF80030BBB9704BD9F8000043
:100CB0001B689B781E3B012B4FF0020142F26882B9
:100CC00004302AF051FC012200238AF8002084F825
:100CD000483126E0644807682FB3D4F8443140F621
:100CE000B732F31A93421ED994F84031002B02F028
:100CF0000F81013BDBB284F84031002B01F0978774
:100D000017F8011B94F84821076094F849315848B6
:100D10000A440133006884F8482184F84931F9F71E
:100D200011FBC4F84461534A029B12781B68012AE4
:100D300003F101030C9301F0FF824F4B1B787BB151
:100D4000DFF85C91D9F8003053B1414C029BD4F8E4
:100D50005C21D3F800B0ABEB0202632A01F21A82E5
:100D6000DFF8408198F800A0BAF1020F01F03A874D
:100D70003C4F97F87430032B01F0DC843F4B1B7819
:100D800073B13F4D2B685BB1314CF8F7EDFFD4F8F0
:100D90006831039044F61F62C31A934200F26081E7
:100DA000384B1B78002B7FD1374B1B7843B1284C35
:100DB000D4F8B83203F50043E8339E4281F0328321
:100DC000324B1B78002B3FF404AF214E304C314D99
:100DD00006F2C1272068F9F7B1FA00283FF4F9AE0E
:100DE0002068F9F7A3FA2B7880465A1E33B12068A1
:100DF0002A70F9F7A3FA0028F2D1EAE6032239466D
:100E0000781E33F030FE96F8C03296F8C12286F88C
:100E1000C38283F47F4383F0FF039B1A1FFA88F891
:100E20009BB2B8EB132FD5D196F8C222DBB29A420F
:100E3000D0D1781E1AF064FF2B7818442870C9E7C7
:100E4000054B0293FFE600BF5E510020E0840020C6
:100E5000602B0020F85500209C9200208AA70020DB
:100E60003F0D030004000020F0A60020ECA60020A7
:100E7000E8A600208BA7002098A70020A0A70020AC
:100E8000A4A7002010A8002021A80020AAA70020C5
:100E9000B0A70020B4A70020F8A60020F4A60020E8
:100EA000D05500207A440020604C2278002A41F07E
:100EB0003A82DFF8A49199F80040002C40F0AB8012
:100EC0005B4D2878002842F08C805A4C5A4DD4F85B
:100ED000B0222978594B93FBF1F313449E42FFF45F
:100EE00063AF94F8B432564AC4F8B062D75CFB07DB
:100EF00002F17482B80702F1E981790702F12A82CE
:100F00003A074CD54F4BDFF854810D930DF1500942
:100F1000A3F13D0249F8202D0021A3F1400203F87E
:100F2000401C02231121517093704846D8F80010DC
:100F300008F002FF4846D8F8041008F0FDFEB8F8A3
:100F40000E30414903EBC3039B00053381FB0321B2
:100F5000DB17C3EBA10189B2484608F004FFB8F8DB
:100F6000103003EB8303590089B2484608F0FBFEBA
:100F7000364B1B789B0743BFB8F8081001F57A7110
:100F800089B24FF47A71484608F0EDFE0C9B98F850
:100F90001420591C0C9148461A702AF0D3FB94F87F
:100FA000B4322978013393FBF1F201FB123384F858
:100FB000B432F9E613F0030A7FF43AAE5E209047AC
:100FC000D9F8003014209847214B1F4AB3F9043058
:100FD00082FB03124FEAE378C8EBA2080FFA88F805
:100FE0005FFA88F02AF014FBC8F307202AF010FB00
:100FF000D9F800305E209847D9F800301C20984777
:1010000050462AF005FB50462AF002FB94F82C319A
:10101000D9F800200CE60F4D2F6E002F41F09D8671
:10102000044B89F80070C3F8B062BDE67CA70020CD
:1010300018A80020602B002020A80020A086010016
:101040001CA800203CA70020676666665656002054
:101050000456002028A8002019A80020545C002075
:1010600094F86E31002B41F0EA85DF4B1B6803F0EA
:101070000802002A48F603414AF60B404BF60F429D
:1010800049F6074704BF02460F4613F0040F4FF01E
:10109000190118BF17469B0684F86E1103D547F453
:1010A000804747F020070BF0DBFBC7F30909002856
:1010B00042F0D282CD4B9B79002B42F09F82984622
:1010C00064204FF0FF3A4FF0000C0C970D97ADF8ED
:1010D0003CC0CDF842C0CDF846C0CDF84AC0CDF8EE
:1010E0003890ADF83E80ADF840A08DF84E000CAFC2
:1010F0000FCFDFF808E384F805C0AEE80F0097E8EB
:101100000F00AEE807002EF8023B71464FF0010CCD
:101110001B0CFE271F20C82201F81E39A770A271E0
:1011200084F807C0E07094F87E01207180F0F1032C
:1011300083EA0313DAB2130983F0E70343EA0223D5
:1011400083EAC2031BB283EA0312D2B2C3F30723BA
:1011500083EA121343EA022383EAC2031BB283F039
:10116000C80282EA0212D2B2C3F3072383EA12133F
:1011700043EA022383EAC2031BB283EA0C0787EA2D
:101180000717FFB2C3F3072282EA171242EA0722C7
:1011900000EB0C0382EAC7070EEB0C0084F87E31EB
:1011A000278011F8013B7B4083EA0313DBB21A0965
:1011B00082EA172242EA032282EAC3031BB29FB2E9
:1011C00081422780EDD183F07C0383EA0313DBB2F5
:1011D0004FEA131E8EEA172E8EEA032E8EEAC30EF6
:1011E0000FFA8EFE1FFA8EF9DFF814C2A4F80090F1
:1011F0005FFA8EFE4FEA192984F8289084F827E0D8
:101200000CF5D37804F1220ADCF80000DCF80410B5
:10121000DCF80820DCF80C3047460FC70CF1100C46
:10122000D445B846F0D1DCF800003860704F9CF827
:10123000043088F8043007F1270884F8CDE184F8F9
:10124000CE9117F8011F2868F9F77CF8B845F8D156
:1012500094F86F21002A41F05E856649029B087868
:101260001B680A2184F86F11002801F09A86DFF8C4
:1012700094E10128BEF80010059142F2EE820228A6
:10128000BEF8028002F00082BEF804100491032828
:1012900002F0DD820428BEF806A002F0D382052801
:1012A000BEF8087002F0C7820628BEF80AC002F035
:1012B000BF820728BEF80C1001D0BEF80E2094F8AB
:1012C0007EB10C938BF0300383EA0313DBB24FEA59
:1012D000131E494884F804B08EF07A0E4EEA032EAD
:1012E00000888EEAC303DFF820E1C0EB00208EFB0C
:1012F000009E8644C0171BB2C0EB6E200690C3F35D
:10130000072E83EA0310059BC0B24FF0000963F378
:101310000F098EEA101305934FF0000E049B68F33B
:101320001F4967F30F0E4FF00008002763F30F0803
:1013300061F30F07059BCDF834906CF31F4E62F3F9
:101340001F474FF0000C9DF81820CDF83CE06AF3E1
:101350001F48CDF8388010978DF844C08DF845208F
:1013600043EA00230DF1300883EAC007B8E80F0014
:101370003FB287F0C80989EA0919DFF880E084F8EC
:1013800005C05FFA89F9C7F30727AEE80F0087EABF
:10139000191747EA092398E8030083EAC9031BB237
:1013A00083F023074EF8040B87EA0717FFB2C3F355
:1013B000072282EA1712704642EA072282EAC7072A
:1013C00020F814190BF1010B4FF0230CFE2116220B
:1013D000C82384F87EB1278084F807C00EF1020E7E
:1013E000A170E270A37111E0F8550020DC550020D7
:1013F000072D0020C4510020C6A60020682B002025
:10140000622B0020FCB900200308208010F8013B6B
:101410007B4083EA0313DBB21A0982EA172242EA0D
:10142000032282EAC3031BB29FB270452780EDD12D
:1014300083F0F40383EA0313DBB24FEA131E8EEA50
:10144000172E8EEA032E8EEAC30E0FFA8EFE1FFAB7
:101450008EFCD64FA4F800C04FEA1C295FFA8EFE1E
:1014600084F81EE084F81F907968BA683868FB68D1
:1014700007F5D37CACE80F0038697969BA6904F2E2
:10148000C518ACE8070004F2A71784F8C59184F8E2
:10149000C4E117F8011F2868F8F754FFB845F8D1E0
:1014A00094F87231002B41F04684C14F3B681922F9
:1014B000980684F8722140F10E83BE4BDFF800835A
:1014C0001B78990741F1868798F81430042B8CBF5C
:1014D0004FF003094FF00209F8F746FCB8F8103056
:1014E000B8F808200C9003EB83035B00ADF84A309A
:1014F0004FF47A70D8F800308DF84C900E93B8F80D
:101500000E1098F814E0D8F804308DF84DE000FB88
:1015100002F24FF0000A4FF0FF300DF13009CDF824
:1015200034A010920F93ADF848101190CC46BCE84F
:101530000F00DFF890E2AEE80F009CE80F00AEE885
:1015400007007246182122F81C39E17194F87E11C7
:1015500084F805A081F0780383EA0313D8B2030965
:1015600083F0F60343EA002383EAC0031BB283EA55
:101570000310C0B2C3F3072383EA101343EA002326
:1015800083EAC0031BB283F0C80080EA001C5FFA44
:101590008CFCC3F3072080EA1C1040EA0C2080EA90
:1015A000CC0000B280F0180383EA0313DBB2C0F36F
:1015B000072080EA131040EA032080EAC30301F108
:1015C000010CFE204FF01E0A4FF0C80BA0700EF168
:1015D000020E217184F87EC1238084F803A084F870
:1015E00006B0184612F8011B414081EA0111C9B248
:1015F0000B0983EA102343EA012383EAC10109B2FC
:1016000088B272452080EDD181F0180181EA011184
:10161000C9B20A0982EA102383EA012383EAC103DB
:101620001BB29AB261492280DBB2120A049106927F
:10163000059384F8272084F826308E4601F5D37B65
:1016400004F1220ADEF80000DEF80410DEF80820BB
:10165000DEF80C30DC46ACE80F000EF1100ED6457B
:10166000E346EFD1DEF80000CCF800009DF814301E
:10167000DFF854A184F8CC319DF8183084F8CD31CE
:10168000D3461BF8011F2868F8F75CFE4A4B5B4500
:10169000F7D1F8F769FBD8F800103B68B8F80820D4
:1016A0000591D8F80410069113F0140F4FF47A71D5
:1016B00001FB02F141F074850F4694F87EB10C9065
:1016C0008BF06A003D4BDFF804E1B3F9042010977A
:1016D00080EA0010C0B2030983F0D50343EA002377
:1016E00083EAC0031BB283EA0310C0B2C3F307232B
:1016F00083EA101343EA002383EAC0031BB28EFB84
:10170000020E05980D90D2174FF00008C2EBAE0202
:1017100006980E9083F0C80C0F91ADF84A20ADF8F2
:101720004480ADF84680ADF848808CEA0C1CCE466B
:101730005FFA8CFCC3F30727BEE80F0087EA1C178B
:1017400047EA0C2787EACC07DFF878C084F804B0B2
:101750003FB2ACE80F0087F021039EE8070083EA60
:101760000313DBB2C7F3072787EA13170BF1010E48
:1017700047EA03278CE8070087EAC30384F87EE181
:101780004FF0210B4FF0FE0E1C27C8220CF10C0C61
:1017900084F8058084F807B084F802E0ACF11C01FD
:1017A000E7701846A271238012E000BF622B002070
:1017B000F8550020565600202D2D002004560020FC
:1017C000545C0020682B0020072D002067666666A9
:1017D00011F8012B424082EA0212D2B2130983EAC5
:1017E000102343EA022383EAC20212B290B2614597
:1017F0002080EDD182F0680282EA0212D2B24FEA72
:10180000121B8BEA102383EA022B8BEAC20B0FFA1E
:101810008BFB1FFA8BF3DB4F23805FFA8BFB1B0ADA
:10182000059384F8253084F824B007F5D37C04F1BF
:10183000220838687968BA68FB68E646AEE80F00A7
:1018400010374745F446F4D13B88AEF800309DF898
:101850001430CD4F84F8CAB1D04684F8CB3118F893
:10186000011F2868F8F76EFD4745F8D194F87EC14E
:10187000C64A84F804C08CF0EB0383EA0313D9B2A0
:101880000B0983F0C50343EA012383EAC1031BB2BA
:1018900083EA0310C0B2C3F3072181EA101141EAC1
:1018A000002181EAC00109B20CCA81F0C80787EAA9
:1018B0000717FFB24FF0000EC1F307210D93CDF8CB
:1018C00038E081EA17130C9299E8070043EA0723EE
:1018D00083EAC7030FFA83F8AD4B84F805E088F07C
:1018E000310783E8070087EA0717FFB2C8F3072329
:1018F00083EA171343EA072383EAC703277A607A48
:10190000A27AE17A94F80CE094F811801BB25F405F
:1019100087EA0717FFB2C3F3072383EA171343EAE3
:10192000072383EAC7031BB2584080EA0010C0B205
:10193000C3F3072383EA101343EA002383EAC003B7
:101940001BB25A4082EA0210C0B2C3F3072282EAF5
:10195000101242EA002282EAC00212B2514081EA29
:101960000111C9B2C2F3072383EA111343EA012329
:1019700083EAC1031BB28EEA030E8EEA0E1E5FFAE3
:101980008EFEC3F3072383EA1E1343EA0E23677B0D
:10199000A07BE17B227C83EACE031BB25F4087EA17
:1019A0000717FFB2C3F3072383EA171343EA07239A
:1019B00083EAC7031BB2584080EA0010C0B2C3F3E9
:1019C000072383EA101343EA002383EAC0031BB210
:1019D000594081EA0111C9B2C3F3072383EA111305
:1019E00043EA012383EAC1031BB25A4082EA02128E
:1019F000D2B2C3F3072383EA121343EA022383EA32
:101A0000C2031BB288EA030888EA08185FFA88F85C
:101A1000C3F3072383EA181343EA082383EAC803BE
:101A2000A17CE27CDFF874811BB2594081EA01118C
:101A3000C9B2C3F3072383EA111343EA012383EAFC
:101A4000C1031BB25A4082EA0212D2B2C3F3072387
:101A500083EA121343EA022383EAC2031BB283F030
:101A6000270787EA0712D2B2C3F3072787EA1217BC
:101A700047EA022787EAC2073FB20CF10103BAB274
:101A80005FFA87F94FF0310CFE200C2184F87E318B
:101A9000C8234FEA122E228084F807C0A070E1709C
:101AA000A37184F81490049F84F815E07968BA68EB
:101AB000FB683868B7F810C0A8E80F0028F803CB17
:101AC00084F8BBE184F8BA911AF8011F2868F8F786
:101AD00039FCD045F8D194F87671002F41F0268179
:101AE0002C4B94F87E81B3F90010B3F90220B3F9BE
:101AF00004309FED296A677107EE103A029B1B685C
:101B00000C9388F06A0383EA031306EE901AD9B2A5
:101B10000B0983F0D50343EA012383EAC1031BB217
:101B200083EA03115242C9B207EE902AC3F3072396
:101B300083EA111343EA0123F8EEE77AF8EEE66A46
:101B4000B8EEC77A83EAC1031BB267EE867A66EE07
:101B5000866A27EE067A002083F0C80ECDED0E7A55
:101B6000CDED0D6A8DED0F7A1090119012908EEAE6
:101B70000E1C0DF130095FFA8CFCC3F3072EB9E897
:101B80000F000DE0622B00202B2D00208887002005
:101B9000682B00200456002088C3E43A082D00205A
:101BA0008EEA1C1E4EEA0C2E8EEACC0EDFF888C49C
:101BB0000FFA8EFEACE80F008EF01E0799E80700C2
:101BC00087EA071A5FFA8AFACEF3072787EA1A1715
:101BD00047EA0A278CE8070087EACA071C214FF06A
:101BE000050A4FF01E094FF0FE0EC82208F101034E
:101BF000E17084F876A184F8079084F802E0ACF1F3
:101C00001001A2710CF10C0C84F80480278084F878
:101C10007E3111F8013B7B4083EA0313DBB21A09E2
:101C200082EA172242EA032282EAC3031BB29FB26E
:101C300061452780EDD183F0270383EA0313DBB2EC
:101C40001A0982EA172282EA032282EAC3031BB23C
:101C50001FFA83FCDFF8E483A4F800C05FFA83FE78
:101C60004FEA1C2C84F825C084F824E008F5D379C9
:101C700004F1220AD8F80000D8F80410D8F8082097
:101C8000D8F80C304F460FC708F11008D045B946B8
:101C9000F0D1E04FB8F80030A9F8003007F124087F
:101CA00084F8CAE184F8CBC117F8011F2868F8F757
:101CB00049FBB845F8D194F877A1BAF1000F41F08B
:101CC0002F80D54B1B68052284F877219A0641F1B5
:101CD0007281D24ADFEDD27AD18907EE101AB8EEBE
:101CE000C77A13F0140F27EE277A01F0F984CD4B51
:101CF000DFEDCB6AD3ED007AF8EEE77A67EEA67AED
:101D000094F87EC1C84BC94AB3F90410B2F9062051
:101D1000C74FC8488DED0D7A8CF0220383EA031378
:101D20005FFA83FE4FEA1E1383F0590343EA0E2342
:101D3000B2F5FA6F83EACE031BB2A8BF4FF4FA6282
:101D400083EA0318B2F57A7F5FFA88F8C3F3072EA7
:101D5000B8BF4FF47A72A2F57A728EEA181E642325
:101D600003FB02F34EEA082E87FB03278EEAC80E18
:101D7000DA17C2EBA71280FB01300FFA8EF7CB17F0
:101D80004FF0000BC3EBA00387F0C8080DF130093A
:101D9000CDED0E7AADF84220ADF84030CDF830B040
:101DA000CDF83CB0CE4688EA0818BEE80F005FFACE
:101DB00088F8C7F3072787EA181747EA082787EA4A
:101DC000C8089D4FDEF800E084F804C00FC70FFA82
:101DD00088F888F04A0383EA0310C0B2C8F30723E7
:101DE00083EA10133A460CF1010143EA002383EA27
:101DF000C00342F810E900204FF04A084FF0FE0CF3
:101E00004FF0140E84F87E11C821607123800437CE
:101E100084F8078084F802C084F803E0A1711846B2
:101E200012F8011B414081EA0111C9B20B0983EA92
:101E3000102343EA012383EAC10109B288B2BA42FE
:101E40002080EDD181F0140181EA0111C9B24FEA7D
:101E5000111E8EEA102E8EEA012E8EEAC10E774BED
:101E60000FFA8EFE1FFA8EFC1F464FEA1C2B5FFAFC
:101E70008EFE84F81DB084F81CE0596838689A68B2
:101E8000DB68A4F800C007F5D37CACE80F00386924
:101E90007969B7F818800497ACE8030004F2A71733
:101EA000ACF8008084F8C3B1B84684F8C2E104F20B
:101EB000C31B18F8011F2868F8F744FAC345F8D186
:101EC0005F4B604A1B781278013B12F00100DBB2D5
:101ED00014BFC0214021172B03D85B4A134493F849
:101EE00014A05A4B1A8893071ABF002341F010011F
:101EF000012312F4027F18BF022312F0100F18BF43
:101F0000062312F0200F18BF1023002841F0918102
:101F10004FF0030894F87EC10C938CF0460383EADB
:101F20000313DAB2130983F0920343EA022383EA2C
:101F3000C2031BB283EA0310C0B2C3F3072282EAD2
:101F4000101242EA002282EAC00212B282F0C80EE7
:101F50008EEA0E1E00235FFA8EFE0320C2F30722D4
:101F60008DF834A08DF8378082EA1E128DF8353056
:101F70008DF836108DF8380042EA0E2899E80700EF
:101F800088EACE0E0FFA8EF8DFF8ACA0E37188EA8B
:101F90000819AAE803005FFA89F9C8F3072888EA54
:101FA000191848EA092181EAC90994F808808AF8D1
:101FB00000200FFA89F988EA090282EA02185FFA1A
:101FC00088F8C9F3072282EA181242EA0822607AE6
:101FD000A17A94F80B90637182EAC80212B2504061
:101FE00080EA0010C0B2C2F3072282EA101242EA6D
:101FF000002282EAC00212B2514081EA0111C9B244
:10200000C2F3072282EA111242EA012282EAC102E5
:102010001EE000BF072D0020F8550020545C002072
:102020000AD7233CFC55002004560020FCB90020B0
:10203000D34D621067666666682B0020622B002015
:10204000A0950020B8520020845004085456002067
:1020500012B289EA020989EA09195FFA89F9C2F319
:10206000072282EA191242EA092294F80C80607B66
:10207000A17B84F804C082EAC90212B288EA02088D
:1020800088EA08185FFA88F8C2F3072282EA181271
:1020900042EA082282EAC80212B2504080EA0010E6
:1020A000C0B2C2F3072282EA101242EA002282EA98
:1020B000C00212B2514081EA0111C9B2C2F3072233
:1020C00082EA111242EA012282EAC102E17B94F81B
:1020D000109013B281EA030282EA0212D2B2C3F371
:1020E000072383EA121343EA022383EAC2031BB2E3
:1020F00089EA030282EA0212D2B2C3F3072383EA17
:10210000121343EA022383EAC2031BB283F03202B2
:1021100082EA0212D2B2C3F3072383EA121343EA1C
:10212000022383EAC2031BB29AB24FF0FE085FFAA1
:1021300083FE0920C8210CF1010C84F802804FEACB
:102140001228E070A17184F87EC1228084F8128088
:1021500084F811E0049B186859689A68B3F80CB0C9
:102160000AF5CC7CACE807000AF5D47A8CF802902A
:10217000ACF800B084F8B88184F8B7E117F8011F13
:102180002868F8F7DFF8BA45F8D1039BC4F868313E
:10219000FEF706BEDFF83C83BF4FDFF83CA34120CB
:1021A0001AF02EF8B8F9022087FB0230D217C2EBE2
:1021B000A00080B21AF008F8B8F9002087FB0230BE
:1021C000D217C2EBA00080B219F0FEFFB8F90420CC
:1021D00087FB0230D217C2EBA00080B219F0F4FFE7
:1021E0009AF80010D9F80000F8F7ACF894F860817C
:1021F00018F0010700F02885A84F3A68910640F1D1
:102200008180A74ADFF8D4821278920740F1C48710
:1022100098F81420042A8CBF032302230393472039
:1022200019F0EEFFD8F8000019F09AFFD8F8040072
:1022300019F096FFB8F80E209A49D9F80000A1FBD2
:102240000232C2F3471211460492F8F77BF89AF86B
:1022500000003968049A11F0140F82EA00028AF82B
:10226000002040F0BA86B8F80820642000FB02F095
:1022700019F076FF98F81470039BD9F8000043EA30
:102280008707FFB23946F8F75DF89AF80020D9F8C9
:102290000000574039468AF80070F8F753F894F870
:1022A0006081B8F1000F2DD17F4F4F2019F0A8FFAA
:1022B000386819F055FF786819F052FF404619F058
:1022C0004FFF0121D9F80000F8F73CF8744A9AF85A
:1022D00000701278D9F8000002F00108414687F03A
:1022E00001078AF80070F8F72DF89AF80020D9F85D
:1022F000000088EA020211468AF80020F8F722F866
:1023000094F86081694AC4F85CB108F10103DBB25A
:10231000A2FB0312D20802EB8202A3EB420384F871
:102320006031FEF71DBD624B62491868F7F7D2FFB6
:1023300000232370FEF7BDBD5F4F386800283EF4D0
:10234000FCAC4FF0000ADFF898815C4CAB46554678
:10235000F7F7F4FFF8B1F5B94FF00109AA4638686C
:10236000F7F7E4FF83B27E2B00F0518498F8012048
:10237000002A49D194F84C11B1B11B2B84F84C219F
:1023800000F01E840D2B45D0386888F80190F7F7CF
:10239000D5FF0028E3D1AA4650460CAA48495D461D
:1023A00019F048FFFEF7C9BC7D2B00F0F08594F8CA
:1023B000502122B180F02003DBB284F8501194F850
:1023C0004B21062A10D8B4F84E1138681944A4F8E5
:1023D0004E11A118013281F8543184F84B21F7F7DE
:1023E000ADFF0028BBD1D6E7B4F84E2188F80190A4
:1023F00013449BB21A0A52FA83F3FF2BA4F84E310E
:10240000386802D12F4DA3E73868F7F797FF002807
:10241000A5D1C0E73868A4F84E21F7F78FFF002850
:102420009DD1B8E794F8BC32C4F8B862012B40F2F1
:10243000738594F8BD222449981801EB800101327C
:1024400002F00102CF6A84F8BD22BFB11F4D0D9585
:102450000DF15009123DA52349F8205D802284F832
:10246000103115233146484684F8112184F8123181
:10247000B847002840F0D18494F8BC32144A0133A4
:1024800082FB0312A2EBE37202EB42029B1A84F876
:10249000BC32FEF795BC00BF67666666F855002043
:1024A000565600201F85EB5188870020CDCCCCCC20
:1024B00014A800203CA70020E4A60020602B0020E8
:1024C000AA2C0020B42C002084500408852C002065
:1024D0005655555504560020D4550020545C002014
:1024E000040000209E4A9F4B92F80BE0029AD4F819
:1024F000381110681B889C4A401A4FF47A71DFB279
:1025000001FB0EF11B0A9777177588424FF0000701
:10251000D37753759770177180F0EA84934BDFF887
:1025200070C21B689249934F0868DFF86892896807
:102530003F688CFB038EDB17C3EB6E1303F5FA7356
:102540009BB293761B0AD37689FB00A389FB01A972
:10255000C017C917C0EBA300C1EBA90107F5EA43F7
:10256000DFF834E210773033001282F820100912BD
:102570001B12DFF828829EF800E0507782F82110C5
:102580008CFB0790F917C1EB601182F823307A4B6E
:1025900098F814A083F81AA0783130371EF0020F93
:1025A00082F8241082F8227000F09F84D8F800E0AE
:1025B000724AD8F80400DFF8E8B182FB0E714FEAE6
:1025C000EE77C7EBA151039182FB0092C117C1EBDB
:1025D000A25203990BFB01E101EB410149000F46B7
:1025E0000BFB020B0497B9460BEB4B0B644F4FEA06
:1025F0004B01059187FB099B87FB01194FEAA9490C
:10260000CDF81C90B8F80E900399B8F8088002EB4A
:10261000820209EBC90902EB8202089201EB8107F1
:102620004FEA89020599039207EB8707049A0697F8
:10263000CF17C10F0991049852494FEAAB4BD217FB
:102640004FEADE7E83F809E0ABEB020E01FB1E02CF
:102650000798069908F5FA78BAF1050F1FFA88FA73
:10266000A0EB0708059F474883F815A04FFA8EF99D
:1026700009EB8109414600FB18789DF82400987306
:102680000898414FDFF81CE149B201EB80018CFB57
:10269000020B4FEAE2720492039ABEF800E08CFB50
:1026A00008C087FB02C74FEAE27C049AC2EB6B12B8
:1026B0000392364A1FFA89F91288ADF8102083F880
:1026C0000A90039A83F813E089B24FEAE8784FEA58
:1026D000112BC8EB6010CCEBA7174FEA1A284FEA72
:1026E000192C4FEA222A9DF80C2083F810B04FEAEB
:1026F000202983F80BC0D973C7F3072C4FEA1E219A
:1027000034BF4FF0320B4FF0330B1A739DF810208B
:1027100083F80DA0587483F8129083F81680DF7147
:1027200083F808C0197583F81BB01A77C4F83461B0
:10273000FEF795BADFF87090D9F80000F7F7EEFDD4
:1027400000283EF41BABD9F800000121F7F7E2FDA9
:102750000222002387F8742088F80030FEF70EBBB1
:1027600004540020FC530020B8A70020FC55002092
:10277000EC55002000560020E4A700206BCA5F6BD8
:1027800083DE1B4340420F00D34D621070A4002033
:102790001F85EB516766666656560020545C002024
:1027A000806967FF605600208C4500205E209047BE
:1027B000D9F8003002209847FF2019F021FA037859
:1027C000FF2B00F0998490F901304FEAE3785FFA2B
:1027D00088F8D8B228F01CFF404628F019FFD9F835
:1027E00000305E209847D9F8003003209847FF203A
:1027F00019F006FA0378FF2B00F07984B0F908305D
:10280000D8B2C3F3072828F003FF404628F000FFA2
:10281000DA4B1B78042B7DD0DFF88CB3B4F82E1183
:102820009BF80020DFF884A391FBF2F302FB131363
:102830009BB2BAF80010A4F82E314FEA03181FFA21
:1028400088F8642303FB01235200B3FBF2F348EA48
:102850000328C3F303225E20D9F800301FFA88F85A
:1028600048EA02089847D9F80030062098475FFAEE
:1028700088F028F0CDFE4FEA182028F0C9FEC049A4
:10288000B4F82E214B7ABAF800A00132012BA4F83B
:102890002E2100F00C874A7B0AEB8A031FFA83FA89
:1028A000002A40F0C084D9F800305E209847D9F85B
:1028B00000303A209847B34BA3FB0A384FEA581828
:1028C0001FFA88FB5FFA8BF028F0A2FE4FEA1B206C
:1028D00028F09EFED9F800305E209847D9F80030E5
:1028E0003B209847642303FB18A39BB2A6480533FB
:1028F00080FB0320DB17C3EBA000C0B228F088FEEA
:10290000002028F085FEDFF8A88298F80630002B1A
:1029100040F051843B689F0640F11282DFF894A298
:102920009AF80030980700F1EA83DFF88C820027DC
:10293000BB46D9F800305E209847D9F80030012016
:102940009847584628F064FE384628F061FED9F8CA
:1029500000305E209847D9F80030092098470020C1
:1029600028F056FE002028F053FEB8F8123098F8F0
:1029700014B0B3F5967F0AD994F82C2102F00F0217
:10298000072A04D842F20F7B9B4528BF9B46D9F803
:1029900000307B4F5E209847D9F8003005209847DB
:1029A0003B7A002B00F06685ABF1200307EE903AEE
:1029B0009FED767AF8EEE77AF6EE006A67EE877AB0
:1029C000BEEE007AF5EEC07AF1EE10FA58BFB0EE26
:1029D000667A77EE877AFDEEE77ACDED027ABDF979
:1029E00008B05FFA8BF028F013FECBF3072028F035
:1029F0000FFE9AF80020002392070A930B9300F130
:102A0000658394F83031012B00F06083B7F9003012
:102A1000DFED5F6A07EE103AB7F9023007EE903A41
:102A2000B8EEC77AF8EEE77A27EE267A67EEA67A4E
:102A3000BDEEC77AFDEEE77A0CA88DED0C7ACDEDF0
:102A40000D7A28F007FE94F82C31D9F80020FEF713
:102A5000F3B85E209047D9F80030302098474D4BAE
:102A6000D3F800805FFA88F028F0D2FDC8F3072081
:102A700028F0CEFD94F82C3113F003087EF4C8AA98
:102A8000454AD4F82811454B9142186840F28F838B
:102A900080EAE073A3EBE0733A4A1BB282FB0312B5
:102AA0004FEAE37ACAEB621A4FF0640808FB1A385F
:102AB0000FFA88F80FFA8AFA5FFA88FB5FFA8AF24F
:102AC000C8F30728CAF3072AD9F8003002925E201B
:102AD0009847D9F8003010209847029A104628F0FD
:102AE00097FD504628F094FDD9F800305E209847B5
:102AF000D9F8003021209847584628F089FD4046F3
:102B000028F086FD3B68D9F80020FEF78BB8DFF887
:102B1000AC809FED238A4FF0240A5E2090475046F8
:102B2000D9F8003098471F4BF8EC016A9B8A07EEF2
:102B3000103AF8EEE66AB8EEC77A0AF1010AC6EE74
:102B4000877A5FFA8AFA67EE887AFDEEE77ACDED4A
:102B5000027ABDF908B05FFA8BF028F059FDCBF38B
:102B6000072028F055FDBAF1270F02D0D9F8002030
:102B7000D3E73B68D9F80020FEF750B8E0A6002064
:102B8000045400201F85EB5167666666E4380E3FEB
:102B90000050C347005600203F4B4C00FC5500201E
:102BA00000007A440C56002012540020FC530020F0
:102BB000DC55002056560020545C00203C56002076
:102BC0003868F7F7BBFB00287FF4DEAB386884F881
:102BD0004A9188F80190F7F7B1FB00287FF4BFAB6A
:102BE000FFF7D9BBF7F7C0F8D14B1B68A0EB030B7D
:102BF00040F6B8339B4500F2BF81CE4B1A793A2A92
:102C000000F04284002388F80030FEF7B7B8386837
:102C100084F84AA184F84BA184F84C9188F801A06B
:102C2000F7F78CFB00287FF49AABFFF7B4BB94F85E
:102C3000481194F84931C0484A1CFEF76AB8013B74
:102C400084F86E31FEF704BBBC4A1288D30513D456
:102C5000D00600F1E682910600F11D85530600F1D1
:102C60003C85100700F15485D10700F1588512F01A
:102C7000020F0CBF04270C27B149B24A0B78D27857
:102C800003F001030AB143F002035320039319F048
:102C9000B7FAAD4A128802EB820202EB8202900080
:102CA00080B219F091FA002019F08EFAA74AA849CB
:102CB0001288D9F80000C2EBC212520081FB023127
:102CC00011444FEAE278C8EB61285FFA88F8414680
:102CD000F7F738FB9AF80020039BD9F800001F4350
:102CE00088EA020800218AF80080F7F72BFB3946B2
:102CF000D9F80000F7F726FB9AF80020D9F8000071
:102D00007A40D2B211468AF80020F7F71BFB94F8FC
:102D10006081FFF7C6BA013A84F86F21FEF7C0BBA5
:102D20000AF1FF3A84F877A1FFF72FBA013F84F840
:102D30007671FEF7C0BF013B84F87231FEF7CBBE5F
:102D40001B077FF580AE834B93E803000CAB83E851
:102D50000300184628F07EFC75E60024DFF8108298
:102D600027464FF0500A02E0DBB283F3118815F8D2
:102D700004B0601C5946284419F0F0F8002840F0CF
:102D800025810BF101031C44EFF311838AF31288B0
:102D90002A6E9442E8DB0022DBB22A6683F31188B4
:102DA000FEF73EB94FF0000A5E201F6884F82CA1A0
:102DB0009047D9F80030DFF8BC811720984750467B
:102DC00028F026FC644BA3FB07239B0BA8FB0312F4
:102DD0005209C2EB0212A3EB8203D8B228F018FC0E
:102DE000D9F800305E209847D9F80030182098476D
:102DF0005A4BA3FB07239B09A8FB03125209C2EB02
:102E00000212A3EB8203D8B228F002FC504628F04D
:102E1000FFFBD9F80020FDF714BF0C9EAE424FF027
:102E200000014FD941F2210015F8013B81EA03234B
:102E30005A0013F4004F80EA020192B289B208BF2F
:102E400011464A0080EA020311F4004F99B293B28E
:102E500018BF0B46590013F4004F80EA010289B2F3
:102E600092B208BF0A46530012F4004F80EA0301F1
:102E70009BB289B208BF19464A0080EA020311F4E6
:102E8000004F99B293B218BF0B465A0013F4004F8B
:102E900080EA020192B289B208BF11464B0011F4D8
:102EA000004F80EA03029BB292B208BF1A46530059
:102EB00080EA030112F4004F9BB289B208BF1946A1
:102EC000B542B1D1484606F072FF25490C9D254810
:102ED0006D1A152DA8BF15252A4630F04BFC224A45
:102EE00094F8BC321570FFF7C9BA2D22DA761DE4CA
:102EF0001E4B02991B780968C4F83811013B012B5D
:102F00003FF60CAB1021022391701371FFF706BB43
:102F100028F060FBFDF705BF0E4A02EB8302D76A7B
:102F2000FFF793BA28F046FB01233B70FDF7B6BECE
:102F30008044002068440020E8A600205456002069
:102F4000B852002098970020FC530020C6A600200D
:102F5000030820808450040873B2E745D34D621003
:102F6000702C00205442002069420020E0A600207E
:102F700079B7030889888888C44AB2F86231002189
:102F80000133A2F8623188F80010FDF7F7BE386807
:102F900084F85091F7F7D2F900287FF4E0A9FFF701
:102FA000FAB9014684460746824604908046059059
:102FB0000246FEF784B99FEDB67A13F0140F08BFEE
:102FC000F0EE477A7EF493AEFEF79ABE41463A2081
:102FD00018F020FF0743FFB2D3E6AE4A1068FFF7B0
:102FE00047B9AD49AD4B0093A1F13F07AC4BAD4A9A
:102FF0000B9101F8404C0CA8AB490A9706F0AEFFC4
:103000000A9F7B1C0A933C700A9B2922591C0A9137
:103010001A700A9BEA22591C0A911A700A9BC8224C
:10302000591C0A910CA81A702FF045FC00F10108F8
:103030000CA942460A9830F09DFB0A9A02EB08035D
:1030400001330A9302F808400A9B5A1C0A921C702A
:103050000A9B5A1C0A921C700A9B5A1C0A921C70EA
:103060000A9B5A1C0A921C700A9B5A1C0A921C70DA
:103070000A9B5A1C0A921C700A9B5A1C0A921C70CA
:103080000A9B5A1C0A921C700A9B5A1C0A921C70BA
:103090000A9B5A1C0A921C700A9B5A1C0A921C70AA
:1030A0000A9B5A1C0A921C700A9B0122991814A8A8
:1030B0000A911A7050F8283DDB1B3B7028F042FB48
:1030C000724B2C70C3F8B062FDF76EBE98E80C002E
:1030D00001210AA884F830110A920B9328F0BAFA59
:1030E000B1E4C4F83C6187F80080FDF7D7BD4FF02C
:1030F00000084046FFF787BB4046FFF76BBBDFF891
:10310000C081D9F80030694F5E209847D9F8003067
:1031100011209847B8F80E204FF4F36B0BFB02F226
:1031200087FB0237D217C2EB6737F8B228F070FA84
:10313000C7F3072028F06CFAD9F800305E209847D2
:103140001920D9F800309847B8F80E30584A0BFBD0
:1031500003F382FB0301DB17C3EB611382FB032143
:10316000DA17C2EB6112642101FB1233D8B228F0E6
:103170004FFA002028F04CFA9AF80030B8F808709E
:1031800099077FF5D4AB5FFA87FB3F0AFFF7D1BB06
:10319000F7F7C0F8FDF797BD01230393FFF73FB89A
:1031A0003C4B1F6807EB87077F00FEF786BAC346D4
:1031B000C246424688E4D9F80030DFF808B1DFF8AB
:1031C00008A15E209847D9F8003028209847DBF8FE
:1031D00000308AFB032ADB17C3EBAA0A5FFA8AF0E6
:1031E00028F016FACAF3072028F012FAD9F80030AE
:1031F0005E209847D9F8003004209847B8F8083086
:10320000002B40F04B82DBF8083083F310085FFAA4
:1032100088F028F0FDF9C8F3072028F0F9F9FFF746
:1032200079BB342728E59BF800309AFBF3FAFFF7C7
:103230003ABB204AD278002A0CBF4FF004084FF066
:103240000508FEF767BE0123D9F800003B70F7F7C9
:103250006DF80746D9F80000F7F768F87F067DF4A7
:103260001DAD8A2800F043828E287DF417AD9AF8B0
:103270000030002B7DF42EAD0F48104B03602D2342
:1032800084F840310768FDF70DBD00BF602B0020BA
:1032900000000000FC5500203CA70020027C00201C
:1032A000CC880408D4880408E088040889B5F81498
:1032B0001F85EB5198970020F0A60020B8A70020AA
:1032C000545C0020EC55002067666666CF4AD04B00
:1032D0000D920DF15008A2F13D0048F8200D19881B
:1032E000DFF85493A2F1400300204FF00A0E02F8D9
:1032F000400C082283F801E040469A7006F033FD46
:10330000D9F80030C349DA1781FB0313C2EBA303DA
:1033100099B2404606F027FD09F0B0FAD9F80890B6
:103320000C9B4FEA1942591C0C911A700C9B4FEAE6
:103330001922591C0C911A700C9B5A1C0C9283F880
:1033400000900C9B5A1C0C921870404628F0FAF919
:10335000FDF7D3BDAD4B0D93A3F140090022212110
:10336000A3F13D0A03F8402C89F8021089F80120E6
:10337000CDF830A020F020FFA74BA84A1B88A84911
:1033800000280ABF11464FF003084FF004085A0501
:1033900000F19F81D80700F1BE8103F00203A14A2A
:1033A000002B1CBF4FF00308114642469E4830F0E8
:1033B000E1F90AEB080314A89C4A013340F8203DC8
:1033C0009B1A00220AF8082089F8013028F0BAF97F
:1033D000FDF796BD4FF00109FEF77EB8DFF86C925D
:1033E0009FED938AB9F90230884A0D9207EE903A20
:1033F000F8EEE77A0DF1500867EE887AA2F1400303
:10340000FDEEE77AA2F13D0148F8201D02F8400CDC
:103410000822CDED027A5A701E229A70BDF808106B
:10342000404606F0A0FCB9F9003007EE903AF8EEFD
:10343000E77A404667EE887AFDEEE77ACDED027ACC
:10344000BDF8081006F08FFCB9F9043007EE903A89
:10345000F8EEE77A404667EE887AFDEEE77ACDED42
:10346000027ABDF8081006F07EFC404628F06AF9A2
:10347000FDF740BD5FFA8BF028F0CAF84FEA1B2039
:1034800028F0C6F8FFF7B5BA9978039318460EF0FE
:10349000F7FD00287FF4B6AB5D49664F664A0988A0
:1034A0006648674CF961DFF8A89111680368926873
:1034B000F962B4F86211C7F86CB0FB63FA64D9F82A
:1034C0000000F965F4F764FF834600287DF451ACF1
:1034D0005146D9F80000F6F71DFF039B94F86421CC
:1034E000DB780493642A4FF0040387F8743040F0CB
:1034F000198194F86531072B08BF84F865B194F8F9
:103500006521504B079207EB021A0393DAF8041077
:10351000069108462FF0CFF9DAF8083005935FFAE4
:1035200080FA18462FF0C7F95FFA80FB454B079ADF
:1035300006990AEB0B000830D87122F00F00987240
:1035400002F00F020BEBCA005A739873524603F154
:103550000F0030F00FF9059B19463B4B0AF10900AB
:1035600018445A4630F006F93648C37903F1010A87
:10357000CBB1013B5FFA83FC0CF1080CDFF8D4E01F
:1035800084440023073010F8012B5A409300D108DF
:1035900083EA420301F0180153404EFA01F253400E
:1035A0008445DBB2EFD1284A04980AF8023030F0A3
:1035B000BDF894F865310022013384F8653184F850
:1035C0006421039BDDF80CA09B785BB11AF8051011
:1035D000D9F80000F6F7B6FE01359AF80230EDB2E0
:1035E000AB42F3D894F864310322013384F8643198
:1035F00087F8742088F80020FFF79EB80E4B8046AD
:10360000B3F900A06420FDF75EBD00BF3CA7002019
:10361000FC5300206766666654560020B088040894
:10362000B8880408C8880408FFA60020FDA600206A
:1036300058A08B4104000020EC550020FC550020D0
:10364000602B00206C5C0020725C0020045600207F
:103650008C4500200007090E854B864A1B8892790D
:1036600003EB830303EB83034FEA83081FFA88F815
:10367000002A40F0FA804FF0FF330FFA83FA09F086
:10368000FDF840B2FDF71FBD11469446174692461D
:103690000492FDF714BE2427FFF7EEBA09F0EEF806
:1036A00027F0B6FF002027F0B3FFFFF733B9D9F8B2
:1036B00000305E209847D9F80030392098475FFAEB
:1036C0008AF027F0A5FF4FEA1A2027F0A1FFFFF7A5
:1036D0001AB94FF00308684967E61027FFF7CCBA1C
:1036E000138907EE903AF8EE677AFEF709BB634B51
:1036F0001B6898067DF5D2AA9AF80030002B7DF45D
:10370000E9AA5F485F4B03602D2384F84031B9E597
:103710002027FFF7B1BA5C494FF0040845E60827B7
:10372000FFF7AABA97F8753058481A0704BF013353
:10373000DBB2072B28BF01234FEA031B07EB0B0269
:103740005FFA8BFA92F810E0514A039200EB0E01F7
:103750000022087A4E498A7201F10D0207EB0B0133
:103760004AEA0E0E012882F800E0C96802F1010C55
:103770000DD90238C0B200F1020E9644624602F83A
:10378000011B72454FEA1121F9D101308444BB4439
:1037900021F0600201339BF81110DBB20A43082BC1
:1037A0008CF800200CF1010249D04FEA031B07EB13
:1037B0000B00384990F810E034487044511A007AF0
:1037C00001EB000C0AF1100ABCF1130F5FFA8AFA40
:1037D000C4DDC9B28A1DD2B2039842F0400E80F80F
:1037E00007E002F1010ADFF8B8E0CAB105315FFA7B
:1037F00081FB0BF1080B83440EF1010C00221CF835
:10380000010B5040820082EA4002C1084240224837
:1038100001F0180140FA01F14A40E345D2B2EED17D
:1038200004980AF80E2087F875302FF07FFFC8E65D
:103830001146FDF744BD11469446FDF740BD1549BC
:10384000511AC6E7114694461746FDF738BD114692
:10385000944617469246FDF732BD114694461746E8
:10386000924604929046FDF72ABD0C4B1B6804E774
:10387000FC530020DC550020BC880408F8550020CB
:10388000F0A60020E4A70020C088040884500408A3
:103890006C5C0020795C00200007090EEC550020CC
:1038A000725C00202DE9F04F2DED0C8B364C99B059
:1038B0006368069020469847002800F07D82B4F89F
:1038C000A870002284F85120002F67D1B4F9386025
:1038D000206AA16AB4F93A20656AB4F93C30DFF88D
:1038E000B4A0301A5B1A521BE06294F85210636362
:1038F00004F12C00226312F027FADAF80030990064
:1039000042F1A081D4ED0C5ADFF88CB0D4ED0B7AE3
:103910001E4A9BED406ADBED416A9BED427ADBF883
:103920000C311268B8EEE58AD4ED0D5AF8EEE77A5C
:10393000F8EEE58A013377EE867A38EE268A78EE5D
:10394000878A9342CBED407A8BED418ACBED428A58
:10395000CBF80C3101F00C850D4B049393F800C0AB
:10396000BCF1140F03F05D86DBF814210025062A54
:1039700001F2FC85DFE812F06E19DA189B17ED18DA
:1039800008188618DB0D00BFF47C0020C447002017
:10399000D5920020E0840020242E0020D44BD5496D
:1039A000079391F801901B68D348DFF8A083049037
:1039B0004FF47A71B1FBF3F3C3EB431603EB8603C9
:1039C000DE00B6B2B7420578B8F9060003F02E83E0
:1039D000D4F87CE0B4F93820236E0EF1010107EE33
:1039E000902A13440129E1672366F8EEE77A03F091
:1039F0002783D4ED1B5AD4ED1D6A07EE101A37EE5B
:103A0000E56AB8EEC75A012F86EE057A37EE257AB9
:103A100077EEC77A84ED1C7AE7EE866A84ED1B7A2E
:103A2000F0EE667AC4ED1E6AC4ED1D6A03F0558798
:103A3000D4F890E0B4F93A20636E0EF1010107EE7C
:103A4000902A13440129C4F890106366F8EEE77ACF
:103A500003F00E83D4ED205AD4ED226A07EE101A3B
:103A600037EEE56AB8EEC75A012F86EE057A37EED3
:103A7000257A77EEC77A84ED217AE7EE866A84EDBF
:103A8000207AF0EE667AC4ED236AC4ED226A03F070
:103A90004C87D4F8A4E0B4F93C20A36E0EF10101E8
:103AA00007EE902A13440129C4F8A410A366F8EE87
:103AB000E77A03F0F682D4ED255AD4ED276A07EEB3
:103AC000101A37EEE56AB8EEC75A012F86EE057A6E
:103AD00037EE257A77EEC77A84ED267AE6EE276A06
:103AE00084ED257AF0EE667AC4ED286AC4ED276A83
:103AF00003F0E686DFF858B2A8F80600B4F8A8305C
:103B0000049A013B1578A4F8A83007990023072DE3
:103B10004B608B60CB6040F05781F6F725F9049B32
:103B2000DFF828821D78069BC01A9BF82131A8F87F
:103B300000000993002B40F04D816E4B5B79002B08
:103B400001F00B836D4B1B78013BDBB2072D8BF82B
:103B5000213102F06A8400230A93694ADBF82C3190
:103B6000D2ED006A674A9FED686AD2F800A0604A09
:103B70000792069ADBED4AAADFF8D8819BED499AB5
:103B80009FED62AADFED62BA9FED62CA9FED62BA55
:103B9000DFF8C491614FCBF82C21D31A07EE903A8D
:103BA000F8EE677AB7EE007AC6EE279A08F11C03A2
:103BB000002508935A4B05932E4677EE6A8A68EEE5
:103BC000A68AF4EEC78AF1EE10FA88BFF0EE478AB3
:103BD000544B98ED008A2B44D3ED007AF5EE407AF1
:103BE000F1EE10FA17D0504B2B4493ED007A78EE9B
:103BF000476AB0EEE66AF4EEC67AF1EE10FA08D53E
:103C0000F5EEC06AF1EE10FACCBF37EE878A37EED8
:103C1000678A83ED008A454B1A8893073FD0022EAE
:103C20003DD0434B9AF82E1033F9163007EE103A78
:103C3000089B07EE901A2B44F8EEE76AB8EEC77AB5
:103C4000D3ED007A4B42A6EEA77A700007EE903AC9
:103C5000F8EEE77AB4EEE77AF1EE10FA0AD407EE5E
:103C6000901AF8EE677AF4EEC77AF1EE10FA88BF90
:103C7000F0EE477A2F4B30490344085EB3F90C301D
:103C8000C01A07EE100AB8EEC77AD007E7EE4A7AF4
:103C900041F1F981294B93ED008A27EE888A079B31
:103CA0009BF864212B4493ED01DA78EE4DCA002A8B
:103CB00000F0E780224BDBF8682106991B688A1A1E
:103CC0009A4240F3DE809AF84830022B02F0F483E7
:103CD000022E04F0EF841B4B1B68990700F19280C1
:103CE000194B87ED00CA1B689342C0F2C48035E0CF
:103CF000D0840020E07C0020D59200206495002034
:103D00004C8E00205856002000247449CDCCCC3D68
:103D1000AE47813F000000000000C8421893002019
:103D20000C930020408E0020602F0020545600206D
:103D30006C2F00207095002004560020288E002053
:103D4000548E0020F8550020508E0020D89200207C
:103D5000242E0020542F002024930020F7EE007A18
:103D6000F4EEE7AAF1EE10FA40F18B8007991F4BB1
:103D7000D1ED017A93ED007AF0EEE77AF4EEC77AAE
:103D8000F1EE10FA7DD5D1ED027AF0EEE77AB4EEDD
:103D9000E77AF1EE10FA74DDD1ED037AF0EEE77A0E
:103DA000B4EEE77AF1EE10FA6BDD114B1B689A075F
:103DB00061D51049104B45E0104BDFF844B01D7839
:103DC0000493072D3FF4A9AE9BF821310993002BF2
:103DD0003FF4B3AE581E8BF82101012D01F0188479
:103DE00019B0BDEC0C8BBDE8F08F00BF5C8E0020DD
:103DF000F85500200456002070950020D592002030
:103E0000242E0020D74BD849DFF8CCE331F916C077
:103E10009EED008ADFF8C4E387ED00CA03EB46009D
:103E200028EE0A8AB0F90C00A0EB0C0007EE900A0D
:103E3000F8EEE77ADEF8000027EE888A904278EE06
:103E40004DCA8BDAB3F90C20B1F900E0C748AEEBEC
:103E5000020E00688EEAEE72A2EBEE72824210DA77
:103E6000B3F90E30B1F90220D21A82EAE273A3EB61
:103E7000E273984205DD002318468BF86431F6F7AB
:103E8000D1F8BB4B2B4493ED000A059B29EE000AA9
:103E9000022E20EE2C0AA3EC010A059304F05984AB
:103EA000B44BD7ED006A93ED007AB34BD3ED007AB3
:103EB000B24B93ED006AB24B67EE277A2B4427EEA4
:103EC000A87AD3ED007A67EE277AF0EE665AECEE28
:103ED000A75AB1EE467AF4EEC75AF1EE10FA08D4BA
:103EE000F4EEC65AF1EE10FA8CBFB0EE467AB0EEA0
:103EF000657A9BED4A6AF7EE007AB4EEE76AF1EE76
:103F000010FAACBF0123002343B1F0EEE66AF0EEF5
:103F1000C77AF4EEE67AF1EE10FA01D587ED007A71
:103F2000022E04F0B183974A974B52F826001B6883
:103F3000B0EE4D0A9847954A954B52F826001B68FB
:103F400098479AF8373023B1924B1B88002B01F029
:103F50000781B0EE4C8A904B38EE400A2B4493ED2B
:103F6000008A83ED000A9AF8483030EE480A20EEC5
:103F7000298A53B3894B1B78DB0741F17780F7EE31
:103F8000007AF4EEE7AAF1EE10FA9BF86431C1F280
:103F90004887002B01F08981DBF86831069AD31A33
:103FA0007F4A12689A4210DD7E4BD3ED007AF0EE24
:103FB000ECCAF4EEE7CAF1EE10FA42F18682002371
:103FC00018468BF86431F6F72DF8774B9BF874217F
:103FD0002B4493ED000A29EE000A20EE088A89EDB1
:103FE000008A32B9059B87ED00CA03ED01CA89ED4D
:103FF00000CA0136032E08F1040809F1040907F18B
:10400000040705F104057FF4E3AD049B1B78072B3F
:1040100001F00C87012B02F0F581002308939BF837
:104020007C31002B41F00183604BDFF8B4A11E68A6
:10403000DAF8003096F82C70D90401F1AC805C4BB2
:104040005C4A059319465C4B498B5C4D92ED006AC6
:10405000D3ED004A5A4A5B4BD5ED036AD3ED005AC3
:10406000D2ED007A92ED014A92ED025A8BED636A2D
:1040700007EE101AB8EEC77A74EEC63A012336EE90
:10408000C77A8BED616ACBED603ACBED644A8BF871
:104090009431C7EE258A338D5A4206EE102A4A4AD9
:1040A000DFED4A6AD2ED005A494AD2ED004AB7EE36
:1040B000007AF4EEC78A75EEA45AF1EE10FA88BFC2
:1040C000F0EE478A75EEA75AB8EEC66AF4EEE68AB5
:1040D000F1EE10FA07EE903AF4EEC65AB8BFF0EEE1
:1040E000668AF1EE10FACBED678AB8EE677A01F1D5
:1040F0009284F4EEC75AF1EE10FA88BFF0EE475AF8
:10410000314BDFED346AD3ED017A314BD3ED014A07
:1041100077EEA47A65EEA65A77EE847AB4EEE76A73
:10412000F1EE10FA08DCB4EEE77AF1EE10FA8CBF8B
:10413000B0EE676AB0EE476A234A738DD2ED027A19
:104140009FED247A5A4204EE902A75EE277AF8EE13
:10415000E44A26EE076AF4EEE47AF1EE10FA4CD463
:1041600040E000BF7095002004560020588E0020CB
:10417000FC8D00207C000020A0890020708E002093
:10418000088E0020A8890020A4890020FC89002036
:10419000F889002054560020902F0020B8520020AB
:1041A000548E0020608E0020148E0020585600206F
:1041B00028700020CC930020549500201454002037
:1041C00018930020088F00200C93002000000000AE
:1041D000249300206F12833A288E0020508E0020F6
:1041E000E084002007EE103AF8EE474AF4EEE74A82
:1041F000F1EE10FA88BFF0EE674AEB4BDFEDEB7A99
:104200005B7864EEA74A0BB9F1EE644A002F42F0E6
:104210003F80F7EE003AE64F3E78002E03F0DD8156
:10422000E44BDFEDE57A93ED025AD3ED016A93EDAD
:10423000037A26EE055AA5EEA65AA4EE875A23EE77
:10424000855AB4EEE75AF1EE10FAB4BFB0EE674A01
:10425000B0EE454A98BFF0EE457A012E8DED105A2A
:1042600003F0F28193ED067A93ED053AD3ED076AF8
:1042700026EE077AA5EE837AA4EEA67A23EE877A55
:10428000B4EEE77AF1EE10FAB4EEC47A8CBFF0EE39
:10429000676AF0EE476AF1EE10FA88BFF0EE676ADF
:1042A000B4BFF0EE447AF0EE477A022E8DED117A2B
:1042B00000F0DE8093ED0A7A93ED093A93ED0B4A14
:1042C00026EE077AA5EE837AA4EE847A23EE877A27
:1042D000B4EEE67AF1EE10FAB4EEE77A8CBFB0EE07
:1042E000664AB0EE474AF1EE10FA98BFF0EE446A23
:1042F000A8BFF0EE477A032E8DED127A00F0B88059
:1043000093ED0E7A93ED0D3A93ED0F4A26EE077A70
:10431000A5EE837AA4EE847A23EE877AB4EEE67A69
:10432000F1EE10FAB4EEE77A8CBFB0EE664AB0EE6A
:10433000474AF1EE10FA98BFF0EE446AA8BFF0EEDB
:10434000477A042E8DED137A00F0928093ED124A95
:1043500093ED113A93ED137A26EE044AA5EE834AC3
:10436000A4EE874A23EE844AB4EEE64AF1EE10FA50
:10437000B4EEE74A8CBFB0EE667AB0EE447AF1EE66
:1043800010FA98BFF0EE476AA8BFF0EE447A052E07
:104390008DED144A6CD093ED164A93ED153A93EDDA
:1043A000177A26EE044AA5EE834AA4EE874A23EE46
:1043B000844AB4EEE64AF1EE10FAB4EEE74A8CBF56
:1043C000B0EE667AB0EE447AF1EE10FA98BFF0EEF5
:1043D000476AA8BFF0EE447A062E8DED154A47D005
:1043E00093ED1A4A93ED193A93ED1B7A26EE044A9F
:1043F000A5EE834AA4EE874A23EE844AB4EEE64A49
:10440000F1EE10FAB4EEE74A8CBFB0EE667AB0EE89
:10441000447AF1EE10FA98BFF0EE476AA8BFF0EECA
:10442000447A072E8DED164A22D093ED1E7A93ED35
:104430001D3A93ED1F4A26EE077AA5EE837AA4EE85
:10444000247A27EE237AB4EEE67AF1EE10FAB4EE8F
:10445000E77A8CBFB0EE666AB0EE476AF1EE10FA0A
:104460008DED177A98BFF0EE466AA8BFF0EE477A56
:1044700077EEE67AF7EE006AF4EEE67AF1EE10FAFD
:10448000CBED4A7A43F3F78786EEA77A022EDDED6D
:10449000117A25EE075A67EE877A8DED105ACDED29
:1044A000117A2DD0DDED127A67EE877A032ECDEDED
:1044B000127A25D0DDED137A67EE877A042ECDEDE2
:1044C000137A1DD0DDED147A67EE877A052ECDEDD7
:1044D000147A15D0DDED157A67EE877A062ECDEDCC
:1044E000157A0DD0DDED167A67EE877A072ECDEDC1
:1044F000167A05D0DDED177A27EE877A8DED177ADB
:104500002E4B1B68DA0041F11884F6EE008ACBEDE1
:10451000678A002E03F05880294B9BF99421D878A4
:10452000284BDBED647A93F800E0274B9BED63AA00
:10453000079309EE102AB3F90630244A0A93FDEED8
:10454000E77A059BDAF800C02149D2ED00AA5B8B1F
:1045500091F800900B9317EE902AFDEECA7A0CF0BA
:1045600010010CF48053DBED609A9BED618AB8EE8C
:10457000C99A0EF0010C17EE908A002841F0B08025
:10458000002941F05D850B499DED107AD1ED007A4F
:10459000104B68EEA77AE7EE097AB0EE487AA7EEFC
:1045A000A97AFDEEC77A17E0A09500206F12833A32
:1045B0000D530020788E002000000000B4930020EE
:1045C00098970020B8520020FCB90020748E00207B
:1045D000A85800206C93002017EE90EA17EE900A7E
:1045E0009645A8BF1046F045C8BF404607EE900A62
:1045F000F8EEE77A012EC3ED007A00F0DC80D1ED11
:10460000047A9DED117A68EEA77AE7EE097AB0EEAA
:10461000487AA7EEA97AFDEEC77A17EE90EA17EE70
:10462000900A9645A8BF1046F045C8BF404607EE21
:10463000900AF8EEE77A022EC3ED017A00F0BB8013
:10464000D1ED087A9DED127A68EEA77AE7EE097A45
:10465000B0EE487AA7EEA97AFDEEC77A17EE90EA97
:1046600017EE900A9645A8BF1046F045C8BF4046D1
:1046700007EE900AF8EEE77A032EC3ED027A00F017
:104680009A80D1ED0C7A9DED137A68EEA77AE7EE69
:10469000097AB0EE487AA7EEA97AFDEEC77A17EE4E
:1046A00090EA17EE900A9645A8BF1046F045C8BF9D
:1046B000404607EE900AF8EEE77A042EC3ED037A3F
:1046C00079D0D1ED107A9DED147A68EEA77AE7EEF5
:1046D000097AB0EE487AA7EEA97AFDEEC77A17EE0E
:1046E00090EA17EE900A9645A8BF1046F045C8BF5D
:1046F000404607EE900AF8EEE77A052EC3ED047AFD
:1047000059D0D1ED147A9DED157A68EEA77AE7EECF
:10471000097AB0EE487AA7EEA97AFDEEC77A17EECD
:1047200090EA17EE900A9645A8BF1046F045C8BF1C
:10473000404607EE900AF8EEE77A062EC3ED057ABA
:1047400039D0D1ED187A9DED167A68EEA77AE7EEAA
:10475000097AB0EE487AA7EEA97AFDEEC77A17EE8D
:1047600090EA17EE900A9645A8BF1046F045C8BFDC
:10477000404607EE900AF8EEE77A072EC3ED067A78
:1047800019D0D1ED1C7A9DED177A68EEA78AE9EE73
:10479000078AA9EEA88AFDEEC87A17EE901A8A4217
:1047A000A8BF0A468845D8BF904607EE908AF8EE23
:1047B000E77AC3ED077ABCF1000F01F09F80E14B6F
:1047C0001B68002B41F0A780DF4B1B789BB138782A
:1047D00070B1DFF8A083DFF8A0930026F0B2D9F81B
:1047E0000030B8EC010A9847387801368642F5DB8C
:1047F000D64B1B689847049B1B78072B01F02B8333
:1048000000230B93DAF800300A935E0501F17681FC
:10481000CF4B1F683C0701F11381CE4BB3F80090DA
:10482000CD4B0893CD4B079A1C68B2F9068062897C
:10483000904580F261864FF07E53CBF82431059984
:10484000089A0E8B079992F90430B1F9000092F89A
:1048500001E01178002BA0EB060383EAE37CACEBCC
:10486000E37C14BF01224FF0FF32BCF5FA7FA8BFF2
:104870004FF4FA7C614580F23B86ACEB010307EE16
:10488000903AF8EEE77AB042C5ED007A03DAF1EE3D
:10489000677AC5ED007A079BB3F90200831B83EAB0
:1048A000E37CACEBE37CBCF5FA7FA8BF4FF4FA7C69
:1048B000614580F21986ACEB010307EE903AF8EE01
:1048C000E77AB042C5ED017A03DAF1EE677AC5ED19
:1048D000017A079BB3F904108B1B83EAE370A0EB0A
:1048E000E370B0F5FA7FA8BF4FF4FA707045CCBF03
:1048F000A0EB0E0E4FF0000E02FB0EFE07EE90EA4C
:10490000F8EEE77AB1420A9BC5ED027ABCBFF1EE40
:10491000677AC5ED027A13F48053079300F0BF85E0
:10492000B8F5FA6F4246A8BF4FF4FA62B2F57A7F43
:104930009BF8A431B8BF4FF47A72A2F57A72002BBB
:1049400040F0C6858649DFF834E281FB0230D31798
:10495000C3EB6013581C6FF0630C3EF910003EF976
:1049600013E00CFB0323A0EB0E0003FB00F381FB21
:104970000321DB17C3EB61139E440FFA8EFE07EE93
:1049800090EA079BB8EEE78A85ED038A002B41F099
:10499000C28019F040030C9300F0FD80714B724906
:1049A00093ED019A93ED026A91ED020A91ED043ABA
:1049B000D3ED030AD3ED003AD1ED038AD1ED015ACC
:1049C000D5ED011A95ED002A684B30EE435A39EEC9
:1049D000467A73EEA07A25EE077A75EEE84A73EE12
:1049E000E09A35EEA8AA24EEA71AB0EE474AAAEE3E
:1049F000294A19F00302B0EE415A79EE067A70EEB8
:104A0000036AAAEE295AA6EEA74AA6EEE75AF0EEE6
:104A1000474AD6EEA74A34EE014AF6EE006A73EE34
:104A200089AA26EEC44A35EE475A35EE807AF0EE72
:104A3000647AEAEE694AA7EE2A4A77EEC17A36EE40
:104A4000607A73EE68AA25EE265AEAEE297AAAEE73
:104A5000875A74EE814A24EE047A73EEC93A33EE33
:104A6000283A64EEA64A67EEA66AF0EE477AE3EECD
:104A7000234A75EEC05A36EE206AD5EE057AA5EEC9
:104A8000057AE5EE866AF1EE648AB0EE476AB0EE2A
:104A9000677AA8EEA47AF1EE663A26EEA43AA3EE7F
:104AA000A66A64EE260AF0EE665AB1EE450AA6EE54
:104AB000A67AB0EE431AF0EE606AE3EEA57A64EEF1
:104AC000243AE5EE246AA0EE041AA8EEA46AF0EEF9
:104AD000638A71EEA19AE0EE240AE5EE258A27EEBC
:104AE000217A32EE029AA5EE043A61EE211A66EEC0
:104AF000A96AE4EEA47AE0EE253A0CBFD5ED022ACD
:104B0000DFED1B2A83ED005AE2EE066AA9EE207A59
:104B1000E2EE281A33EE033A67EEA27A73EEA33A76
:104B2000B0EE006AA2EE837AE2EEA36AE1EE867A44
:104B30008BED6C7A85ED017ACBED6B6AC5ED006A81
:104B40001EE000BF04910020D05B0020A45800208C
:104B5000F855002054560020689500205C5600202F
:104B60001F85EB51C80100207C00002000020020BE
:104B7000000000006C9300209C580020248F00202F
:104B8000CBED6D7A83ED014AC3ED025AC3ED034AC2
:104B90000AB9C5ED027A17F0140F03D019F4027F99
:104BA00041F05B80DA4B1B789BB1059B5B8B4345E7
:104BB0000FDBD84B1B78012B01F03C84192B01F043
:104BC00039840E2B05D0082B03D00023AB60CBF823
:104BD00038319BF8DA611EB119F0030F41F0998367
:104BE0009BF8E061002E40F0D387059B9B7F002B54
:104BF00000F04D84022B01F08083032B41F0798378
:104C0000059B93F82030C3EB431203EB8202D200E2
:104C100092B2059BDB7F0233DBB2002E00F01D85D4
:104C2000002A00F01A85BC490968B2FBF1F20FFABC
:104C300082F8ABF81082ABB307EE908AF8EEE77A11
:104C4000F7EE006A86EEA77A012BD5ED007ADBED50
:104C5000896A77EEE67A67EE877ACBED857A21D09E
:104C6000D5ED017ADBED8A6A77EEE67A022B67EE04
:104C7000877ACBED867A15D0D5ED027ADBED8B6A9B
:104C800077EEE67A032B67EE877ACBED877A09D049
:104C9000D5ED037ADBED8C6A77EEE67A67EE877AFC
:104CA000CBED887A049A1278092A03F02B83B8F1A5
:104CB000000F40F3F2839BB39BED897ADBED857A9D
:104CC00077EE877A012BCBED897AC5ED007A21D07A
:104CD0009BED8A7ADBED867A77EE877A022BCBED35
:104CE0008A7AC5ED017A15D09BED8B7ADBED877A58
:104CF00077EE877A032BCBED8B7AC5ED027A09D05C
:104D0000DBED8C7A9BED887A77EE877ACBED8C7A27
:104D1000C5ED037A013B022BB8BF0223DBB2099336
:104D2000002E099818BF02202378DFED806AA27850
:104D300007EE903AF8EEE77AB0EE007A67EEA67AE0
:104D4000049BF4EEC77AF1EE10FA197840F34E8620
:104D5000DFED736A37EEC77AB0EE676AA7EE266AB0
:104D6000F0EE466A95ED007A9FED6E6A27EE066AD0
:104D7000F0EEC65A8BED536ACBED565A9AB107EE58
:104D8000102AB8EEC75A9FED697A66EE064A25EEFC
:104D9000075AB7EE007A37EE457A64EEA54AA4EEDC
:104DA000857A26EE076A9FED607A637926EE877A28
:104DB00027EE067ACBB1DFED5D6A9FED5D6A65EEA9
:104DC000A65A06EE903AF8EEE66A66EEA56AF4EEAA
:104DD000C66AF1EE10FA01F33C82F7EE005A75EE66
:104DE000E66A85EEA66A27EE067A0C299FED518ABF
:104DF000DFED516A00F0FA87B4EEC87AF1EE10FAEE
:104E000098BFB0EE478AB4EEE68AF1EE10FAB8BF6A
:104E1000B0EE668A8BED4C8A002800F0F580B0EE8B
:104E2000007AF4EEC77AF1EE10FA05DD37EEC77AB4
:104E3000DFED3B6AE7EE267A95ED017ADFED396A20
:104E400027EE267AF0EEC75A8BED547ACBED575AFF
:104E50009AB106EE902A9FED356AF8EEE66A27EEE3
:104E6000075A66EE866AB7EE006A36EE666A25EE87
:104E7000255AA6EE856A27EE067ADFED2B6AA3791E
:104E800067EEA67A67EE877AABB107EE103AB8EE16
:104E9000C77A9FED266ADFED266A27EE257A27EE90
:104EA000067AB4EEE67AF1EE10FA41F3D681DFED40
:104EB0001B6A67EEA67A0C2900F04E87DFED1D6AAB
:104EC0009FED1D7AF4EEE67AF1EE10FA88BFF0EE6F
:104ED000667AF4EEC77AF1EE10FAB8BFF0EE477AD0
:104EE0000128CBED4D7A40F38F806378DFED0F6AB8
:104EF00007EE903AF8EEE77AB0EE007A67EEA67A1F
:104F0000637AF4EEC77AF1EE10FA1DDD16E000BF09
:104F1000A0230020A0950020989500200000C84202
:104F2000D7A368416F12033B000048430AD7233CD4
:104F3000A4707D3F00C0F94400C0F9C437EEC77AC1
:104F40005FED096AE7EE267A95ED027A5FED0B6A6E
:104F500027EE267AF0EEC75A8BED557ACBED585AEC
:104F60009BB106EE903A1FED0F6AF8EEE66A27EE67
:104F7000075A66EE866AB7EE006A36EE666A25EE76
:104F8000255AA6EE856A27EE067A5FED196AE3795F
:104F900067EEA67A67EE877AFBB107EE103AB8EEB5
:104FA000C77A1FED1E6A5FED1E6A27EE257A27EE8F
:104FB000067AB4EEE67AF1EE10FA01F35C81B5EE12
:104FC000C07AF1EE10FA02F1DC84B7EE006A36EE38
:104FD000477AC6EE076A67EEA67A0C2900F0B48617
:104FE0005FED2C6A1FED2C7AF4EEE67AF1EE10FA02
:104FF00088BFF0EE667AF4EEC77AF1EE10FAB8BF29
:10500000F0EE477ACBED4E7A092900F08886059BB1
:1050100093F82140002C40F03D86B94B1F680023D7
:105020008BF8E031B80607D519F0300F04D0B54B36
:105030001B78D90702F13082B34B1B7823B9B34CEC
:10504000A678002E41F07A81069807F0B3FB049B06
:105050001D78072D7EF4C1AEF4F786FE049AAC4BA2
:1050600015780B9A801AD880FEF7B7BE9BF864318A
:10507000002B3EF4AAAF002318468BF86431F4F7F6
:10508000D1FFFEF7A2BFB1F900209BED567AB1F92E
:105090000200DBED576A9F4982EAE273A3EBE273F9
:1050A000F4EEC76A80EAE072F1EE10FAA2EBE07269
:1050B000B4BFB0EE476AB0EE666A9342B8BF13461B
:1050C00007EE103A0B78B8EEC77A27EE0A7A002B73
:1050D00040F0BC80904BD3ED005AF4EEEB5AF1EE69
:1050E00010FA41F11181B7EE005A75EE654ADFED15
:1050F0008B6A9FED8B5A8B4B36EEC77A24EE855A1E
:10510000D3ED006AE7EE055A65EEA65AF5EEC05AF1
:10511000F1EE10FA40F20D86CBEE256AB7EE007A7A
:10512000F0EE475AE6EE665AF0EE656AF4EEC76AAC
:10513000F1EE10FA88BFF0EE476AF5EEC06AF1EEC4
:1051400010FAB8BFF0EE4C6A774B93ED007A67EE39
:10515000877AA7EEA68AFEF7A2BD0123FEF7F6BC6A
:10516000724B734A2B4493ED007AD2ED007A714B67
:1051700067EE277AF7EE006AF4EEE67AF1EE10FABF
:1051800093ED007A88BFF0EE667A67EE877A27EEB5
:10519000888AFEF7E0BE684B684D1B78D5ED037A30
:1051A00013F0010F664B059304BF1B8BABF88831DE
:1051B000644B1B8807EE103AB8EEC77AF4EEC77A54
:1051C000F1EE10FA42F20C815F4A128807EE102AC3
:1051D000B8EEC77AF4EEC77AF1EE10FAC1F2378171
:1051E0005A4B5B4A93ED006AD2ED006A9BF9943109
:1051F000CBED636A76EE665A012BCBED616ACBED9F
:10520000605A8BED646A01F0E686069BCBF8983114
:10521000002237EEC77AFCEEE77A4E498BED677ACB
:1052200017EE903AABF888310123D1ED005A8BF894
:105230009431494B9A4242F29A80484BD3ED007A1E
:1052400093ED014A93ED025AFEF723BF354B93EDE0
:10525000005AB5EEC05AF1EE10FA40F36A85404BA1
:10526000D3ED006AF5EEC06AF1EE10FA40F3618505
:1052700036EEC77A66EE4B5A87EE266AC5EE856A29
:10528000B7EE007AB4EEC76AF1EE10FA88BFB0EE5E
:10529000476AB5EEC06AF1EE10FA76EE876AB8BFDB
:1052A000B0EE4C6A66EE266A40E72E4AD2ED007AEE
:1052B000B0EEC87AB4EEE77AF1EE10FA7EF785AE7A
:1052C000294AD2ED007AB0EEEC7AB4EEE77AF1EE4C
:1052D00010FA7EF77AAE254AD8ED007A92ED007A80
:1052E000F0EEE77AF4EEC77AF1EE10FA7EF56DAEE5
:1052F00001220699CBF868118BF86421FEF750BEA5
:10530000F8550020565600205E510020C0A600200F
:10531000D8920020348E00203C8E002000003443C0
:10532000610BB63B308E00202C8E00207C2F00209D
:10533000248E0020208E0020B8520020145400201B
:10534000287000200C8F00200E8F00205495002024
:10535000F88E0020148F00208FD0030018930020B7
:10536000388E0020648E0020608E0020688E002021
:10537000C24A049207EE103A1278DFF83883CBF86D
:105380000C71B8EEC77AF7EE006A132A86EE879A98
:10539000B8F90400BBF8105194ED070A01F0A78595
:1053A000B74BB84A93ED001AD3ED053A93ED122AA4
:1053B00093ED173AD3ED091AD3ED0E4A93ED016A36
:1053C00093ED064A93ED0A7AD3ED0F5AD3ED132AE3
:1053D000D3ED186A93ED045AD3ED030A67EE897A88
:1053E00069EE288A29EE088AE1EE273A02EB850663
:1053F0000021A2EE283ACBF80011CBF80411E1EE1F
:10540000884AA6EE274AE7EE085A93ED167A93EDFE
:105410000D6A93ED021AD3ED0C1AC6ED003AE2EED6
:10542000A86A25EE635A27EE437A93ED0B2AD3ED53
:10543000152AC6ED204AA0EEE34A26EE646AD3EDB3
:10544000143A83ED054AA1EE275AF0EE477AE1EED1
:10545000E45AA2EE086AE2EEC36AE3EEA87A83EDAC
:10546000065AC3ED0E5A83ED0F6A86ED403AC3ED3E
:10547000176AC3ED187ACBF808116B1C03F01F03F1
:10548000ABF81031A8F80400049BFEF767BAABF83C
:1054900010329846002E3FF4C5AD022044E4059B2F
:1054A0005A8B9045C0F2D383B8F5FA6FD4BFC2EBE4
:1054B0000803C2F5FA634FF47A7101FB03F19BF81C
:1054C000A401C2F5FA63B1FBF3F200283FF43AAA53
:1054D0009BF8A5316C4902FB03F281FB0213D21742
:1054E000C2EB6312FFF72EBADFED687AFFF7E9B976
:1054F000DFED667AFFF7C7B9B8F5FA6F80F2A983D6
:10550000217AA8EB020303FB01F3C2F5FA6293FBD5
:10551000F2F3C3F1640307EE903A9FED5D7AF8EE83
:10552000E77A67EE877ACBED497AFFF788B9DBF83F
:105530001801BBF81031534FDFF89881554AC3F179
:10554000200603EB4010F6B2334607EB80004146DD
:10555000F5F730F9BBF81031002B42F0B583049B0E
:105560001B78142B02F09086DBF814214A4B013291
:1055700083FB02139918D317C3EBA103C3EBC30337
:10558000D21ACBF814214549DBF81C21069D44486A
:105590000B680078CBF81C51AA1A13440B60002842
:1055A00040F0BD8107EE902A3E4EDFF82C913E4F31
:1055B000B8EEE78A06F2447506F5F668F6EC017A6D
:1055C00094ED070AD4F86C37F8EEE77A284627EE10
:1055D000800A9847A5F1E000D4F88C369847A5F1E9
:1055E0007000D4F8FC369847D6F85006D4F8AC30A2
:1055F0009847D7ED007AA9EC010AE0EE087A243545
:10560000A845E7EC017AD9D1049B1D78FEF7D9BBF8
:10561000264B274A19681288264BC96919805A8077
:1056200019B0BDEC0C8BBDE8F08F234B234F1B78DA
:105630003A78D80700F11F84002A00F02086204B1A
:1056400020492148059392002EF094F81F4BDFF873
:105650008CA01F4D0793FFF7B2B8BBF8108208F17A
:10566000FF380FFA88F8B8F1000FABF810823FF757
:1056700022AB002E7FF411AFD4E400BFD5920020FE
:10568000544A0020E84700201F85EB51000000002D
:105690000AD7233C242E00209324499244890020D9
:1056A000BC470020207D00204889002028A9002038
:1056B00078400020D8920020B85200200D530020DE
:1056C000287000207C4000206C930020FCB9002052
:1056D0001454002068490020D4840020E084002075
:1056E000002900F0D587BCF1000F42F09884CC4926
:1056F0009DED107AD1ED007ACA4B68EEA77AFDEEE7
:10570000EA6AB9F1000F42F01483E7EE097AB0EECD
:10571000487AA7EEA97A16EE900AFDEEC77A17EE40
:1057200090CA17EE90EA9445A8BF96466045C8BF58
:10573000864607EE90EAF8EEE77A012EC3ED007A8E
:1057400000F0DF80D1ED047A9DED117A68EEA77A42
:10575000E7EE097AB0EE487AA7EEA97AFDEEC77AAD
:1057600017EE90CA17EE90EA9445A8BF9646844576
:10577000B8BF864607EE90EAF8EEE77A022EC3ED50
:10578000017A00F0BE80D1ED087A9DED127A68EEC4
:10579000A77AE7EE097AB0EE487AA7EEA97AFDEE8D
:1057A000C77A17EE90CA17EE90EA9445A8BF9646BE
:1057B0008445B8BF864607EE90EAF8EEE77A032EF6
:1057C000C3ED027A00F09D80D1ED0C7A9DED137A45
:1057D00068EEA77AE7EE097AB0EE487AA7EEA97AE2
:1057E000FDEEC77A17EE90CA17EE90EA9445A8BF6F
:1057F00096468445B8BF864607EE90EAF8EEE77A0B
:10580000042EC3ED037A7CD0D1ED107A9DED147A8D
:1058100068EEA77AE7EE097AB0EE487AA7EEA97AA1
:10582000FDEEC77A17EE90CA17EE90EA9445A8BF2E
:1058300096468445B8BF864607EE90EAF8EEE77ACA
:10584000052EC3ED047A5CD0D1ED147A9DED157A66
:1058500068EEA77AE7EE097AB0EE487AA7EEA97A61
:10586000FDEEC77A17EE90CA17EE90EA9445A8BFEE
:1058700096468445B8BF864607EE90EAF8EEE77A8A
:10588000062EC3ED057A3CD0D1ED187A9DED167A3F
:1058900068EEA77AE7EE097AB0EE487AA7EEA97A21
:1058A000FDEEC77A17EE90CA17EE90EA9445A8BFAE
:1058B00096468445B8BF864607EE90EAF8EEE77A4A
:1058C000072EC3ED067A1CD0D1ED1C7A9DED177A18
:1058D00068EEA78AE9EE078AA9EEA88AFDEEC87AE3
:1058E00017EE901A8A42A8BF0A468842D8BF1046CF
:1058F00007EE900AF8EEE77AC3ED077A002E3EF441
:105900005EAFB200484947482DF034FF474B1B6853
:10591000002B3EF459AF1FF08FFDFEF755BF07EE89
:10592000902A434D434BDFF81081DFF81091CDF8FA
:1059300014B0F8EEE78A05F2D46600279B46CDF84E
:105940002080049BD4ED077A1B78172B52D095ED5D
:10595000007AB8EEC78A082B28EE278A07D1B0EE66
:10596000480A07932EF0DCF8079BA8F80000DAF845
:10597000002092000BD5002F02F0D086B0EE480A2E
:10598000D4F86C3706F170009847B0EE408AB0EE5C
:10599000480AD4F88C36A6F170009847D4F8FC3643
:1059A00030469847049B1B78032BB0EE408A2DD0DD
:1059B000D5F85406D4F8AC30B0EE480A9847D9ED83
:1059C000007AABEC010AE0EE287A0137032F06F1EA
:1059D000240608F1020805F10405E9EC017AB0D1CA
:1059E000049BDDF814B01D78FEF7EBB9F0EE676AA2
:1059F000FFF7B8B995ED007A04EB4702B8EEC78A15
:105A0000128FA8F8002028EE278AB0E72EF088F839
:105A1000A8F80000CCE7F0EE465AFEF771BB00BFD5
:105A2000788E00206C9300207C40002004910020A0
:105A3000207D0020D4840020D892002048890020B6
:105A4000D5ED027AD44BB2EE0E7AF0EEE76AF4EEC0
:105A5000C76AF1EE10FAB3F80090D04B40D519F0B8
:105A6000040F3DD0B3F90430CD4ACE4982FB030286
:105A70000988DB17C3EBA2035B1A9BB219B211F1C1
:105A8000B30FBCBF03F5B47319B2B329C4BFA1F5FA
:105A9000B47319B2C44BC54A08931B791278002B12
:105AA0004FF6FF7318BF012310077EF5BBAEC04A47
:105AB000126811FB03F3117EBE4A9BB211FB03F384
:105AC00082FB03121A44DB17C3EB221307EE103AD2
:105AD000B8EEC77A77EEC77AC5ED027AFEF7A2BEB6
:105AE000B3F90430AE49AF4A81FB0301DB17C3EBC6
:105AF000A103AD4908911380FEF794BEA368002B63
:105B00003EF486AEAC49A1F14C009847DAF800307B
:105B10000A93FEF77DBE1D21A84804F03AFE002836
:105B200041F08E8426201EF0F9FA00283EF431AFB1
:105B3000A34BDB78002B7EF42CAF26219F4804F08A
:105B400028FEDFEDA07AA049002802F0708438EE2C
:105B5000678AC6F57A72FDEEC87A12B2CDED0C7A7C
:105B6000BDF930301B0381FB0301DB17C3EBA1132D
:105B700002FB03F343F30F33334407EE903AB8EEDE
:105B8000E78A012385ED038A8BF8A031FEF701BF78
:105B90008E4A8A4BD2F8EC201B6844F620618A4278
:105BA000A8BF0A46B2F57A7FB8BF4FF47A7292B2B4
:105BB000D906ABF8E22140F14484079B002B01F0A9
:105BC000E9867B4BD3F800E0BEF8320040087E49FE
:105BD000DBF8E431D5ED037AA1FB021291096422CE
:105BE00092FBF1F2142ABDEEE77A0BEB430CA8BF4F
:105BF000142201339A42CBF8E43117EE108ADCBF4D
:105C00000023CBF8E4310BEB4303ACF8E881B3F9A4
:105C1000E83107EE103AB8EEC77A77EEC77AFDEEB4
:105C2000E77ACDED077ABDF91C2082EAE273A3EB97
:105C3000E273834202F35480654A4FF07E5313604F
:105C4000FEF7D3BF634B0493DFF89CB19BE4079945
:105C500035E4237AC3F164035DE4544B1B7813F0FD
:105C6000100301F08E849BF8B821DBF8BC3195ED70
:105C7000017A002A0CBF01224FF0FF3203FB02F32E
:105C800007EE903AF8EEE77A77EE877AC5ED017A7B
:105C9000FEF788BF1E21494804F07BFD00283FF431
:105CA000BCA90C9B002B7FF4B8A99BF83432A3420B
:105CB00042F04483464B9BED8E0AD3ED058ADBED23
:105CC0004E5A9FED456ADFED456A20EE657A60EE3B
:105CD000087AA8EE887AE5EEA87AB4EEC67AF1EEF4
:105CE00010FA88BFB0EE467AB4EEE67AF1EE10FA1A
:105CF000F4EEC67AB8BFB0EE667AF1EE10FA88BF5D
:105D0000F0EE467AF4EEE67AF1EE10FAB8BFF0EE75
:105D1000667A8BED4C7ACBED4E7AFFF77EB9FDEECD
:105D2000C87A2F4A17EE903AA2F80480D380FFF782
:105D30006EB9DFED2C6AFFF707BADAF800305B02C4
:105D40003EF5E3ABFEF7E5BBBDEEE77A244B17EE7D
:105D5000102A9A80FFF744B99FED1F7ADFED1F6A82
:105D60001F4AF4EEC77AF1EE10FA98BFB0EE677AE8
:105D7000FDEEE77AB4EEE67AF1EE10FA17EE903A1D
:105D8000B8BFB0EE667A01288BED4D7A53803FF7AD
:105D9000ACA8FFF73CB900BF5456002004560020C1
:105DA00067666666A0880020689500205656002029
:105DB0005856002089888888407D0020B4930020B0
:105DC0009897002000007A44D34D6210E40300202D
:105DD0007C000020D592002000C0F94400C0F9C426
:105DE000D892002000000000242E0020B4EEC87AD3
:105DF000F1EE10FA98BFB0EE478ABDEEC77AB4EE66
:105E0000E68A874EF1EE10FA17EE103AB8BFB0EE00
:105E1000668A8BED4C8A338000287FF400A8FFF758
:105E2000F6B8002B3EF4D1A8FEF7B6B8F3F79CFF06
:105E3000049B0A9A1B78DFF8E881801A012BA8F8E6
:105E4000020000F0E182072B7EF4E7A8F3F78CFF55
:105E50000890FEF7E4B8F3F787FF049B08991B78D6
:105E60006F4A401A072B90807EF4CAACF3F77CFF90
:105E70000B90FEF7C7BC002A00F00182DBED573A19
:105E80009BED566A674BDBED617AD3ED005A9BEDD3
:105E9000607A9BED544ADBED534A6349634BF4EE61
:105EA000C63AF3EE046AF1EE10FA37EEA65A00F1A4
:105EB0001B8391ED026A26EE446AF0EE674AE6EE35
:105EC000074AF4EEC54A34EEE66AF1EE10FA48BF2E
:105ED000B0EE656A012A83ED006A00F0D08191ED91
:105EE000066A26EE446AF0EE674AE6EE074AF4EEEA
:105EF000C54A34EEE66AF1EE10FA48BFB0EE656AC4
:105F0000022A83ED016A00F0BA8191ED0A6A26EE59
:105F1000446AF0EE674AE6EE074AF4EEC54A34EE0C
:105F2000E66AF1EE10FA48BFB0EE656A032A83ED27
:105F3000026A00F0A48191ED0E6A26EE446AF0EE4A
:105F4000674AE6EE074AF4EEC54A34EEE66AF1EE39
:105F500010FA48BFB0EE656A042A83ED036A00F0C8
:105F60008E8191ED126A26EE446AF0EE674AE6EE03
:105F7000074AF4EEC54A34EEE66AF1EE10FA48BF7D
:105F8000B0EE656A052A83ED046A00F0788191ED30
:105F9000166A26EE446AF0EE674AE6EE074AF4EE29
:105FA000C54A74EEE66AF1EE10FA48BFF0EE656A93
:105FB000062AC3ED056A00F06281D1ED1A6A66EE29
:105FC000C46AF0EE674AE6EE874AB3EE046AF4EE7E
:105FD000C54A74EEC66AF1EE10FA48BFF0EE656A83
:105FE000072AC3ED066A00F04A81D1ED1E6A104A05
:105FF000059226EEC44A0F4ADFF840A00E4D0792E4
:10600000E4EE077AF4EEC57A77EEC67AF1EE10FA8E
:1060100048BFF0EE657AC3ED077AFEF7D0BB00BF4C
:10602000D8920020748E0020788E00206C9300207F
:1060300028700020FCB9002014540020E0840020C7
:10604000BCF1000F41F03483C7499DED107AD1EDCA
:10605000007AC64B68EEA77AE7EE097AB0EE487A86
:10606000A7EEA97AFDEEC77A17EE90EA17EE900A2E
:106070009645A8BF1046F045C8BF404607EE900AB7
:10608000F8EEE77A012EC3ED007A3FF43AACD1ED99
:10609000047A9DED117A68EEA77AE7EE097AB0EE00
:1060A000487AA7EEA97AFDEEC77A17EE90EA17EEC6
:1060B000900A9645A8BF1046F045C8BF404607EE77
:1060C000900AF8EEE77A022EC3ED017A3FF419AC9C
:1060D000D1ED087A9DED127A68EEA77AE7EE097A9B
:1060E000B0EE487AA7EEA97AFDEEC77A17EE90EAED
:1060F00017EE900A9645A8BF1046F045C8BF404627
:1061000007EE900AF8EEE77A032EC3ED027A3FF429
:10611000F8ABD1ED0C7A9DED137A68EEA77AE7EE35
:10612000097AB0EE487AA7EEA97AFDEEC77A17EEA3
:1061300090EA17EE900A9645A8BF1046F045C8BFF2
:10614000404607EE900AF8EEE77A042EC3ED037A94
:106150003FF4D7ABD1ED107A9DED147A68EEA77AB3
:10616000E7EE097AB0EE487AA7EEA97AFDEEC77A93
:1061700017EE90EA17EE900A9645A8BF1046F04534
:10618000C8BF404607EE900AF8EEE77A052EC3ED49
:10619000047A3FF4B6ABD1ED147A9DED157A68EE32
:1061A000A77AE7EE097AB0EE487AA7EEA97AFDEE73
:1061B000C77A17EE90EA17EE900A9645A8BF1046E8
:1061C000F045C8BF404607EE900AF8EEE77A062E83
:1061D000C3ED057A3FF495ABD1ED187A9DED167AB3
:1061E00068EEA77AE7EE097AB0EE487AA7EEA97AC8
:1061F000FDEEC77A17EE90EA17EE900A9645A8BF13
:106200001046F045C8BF404607EE900AF8EEE77A20
:10621000072EC3ED067A3FF474ABD1ED1C7A9DEDE9
:10622000177A68EEA78AE9EE078AA8EEA98AFDEE3A
:10623000C87A17EE901A8A42A8BF0A468845C8BF96
:10624000424607EE902AF8EEE77AC3ED077AFFF7A9
:1062500055BB9FED476AFEF7C6BDB5EEC07AF1EEBD
:1062600010FA01F18A83B7EE006A36EE477AC6EE7D
:10627000076AFEF71EBEDFED3E6AFEF7ACBE3D4B81
:1062800005933D4BDFF820A13C4D0793FEF797BAED
:106290003B4A5379002B3DF4BCAF3A4B1B78002BA3
:1062A0003DF4B7AF12789FED385A07EE902A374A7F
:1062B000B8EE677A128807EE903A06EE902AF8EE6A
:1062C000E77AF8EE666A67EE277AB7EE007AC7EEED
:1062D000A63AF4EEC53AF1EE10FA88BFF0EE453A70
:1062E000F4EEC73AF1EE10FAB8BFF0EE473AFDF718
:1062F00092BF274B5A88FEF78CBCBBF8E22102F50F
:106300007A7292B2FEF785BC224BD3ED005AFEF7AB
:10631000FDBE214B9FED217AD3ED087AF4EEC77ACA
:10632000F1EE10FA00F259859FED1D7AD5ED037A52
:1063300077EE877AC5ED037AFEF752BC194D2B78BC
:10634000013B0D2B47D8DFE813F0E10706087B0778
:106350005907C707AC07EF07460716073100F706CE
:10636000EB063B070C0700BF788E00206C930020E3
:106370000000C84228700020FCB9002014540020FE
:10638000DC55002012540020713DAA3FFC53002030
:10639000C4510020308E00201C8900208FC2753C23
:1063A0000000000016C10020E0840020A94B1B78EB
:1063B000002B02F07F801A201DF00CFF002842F015
:1063C0007980A54B1B78002B42F0748009232B7039
:1063D00021F0B6FDA678012E00F04A852379012B25
:1063E00001F0FE85022B7EF42FAE2B78012B7EF47C
:1063F0002BAE994B1B78002B7EF426AE22F046FD87
:10640000FEF722BEDFF88082F3F7AEFC934ADBF89A
:10641000783112680890C31A9A1ACBF87801A8F854
:106420000430A8F80620FDF7FABDF3F79DFC0A90AA
:10643000FDF793BB8A4B9B7B002B3EF4C6ABFEF76C
:10644000C8BB0A9BDB003FF5B8ABFEF7CEBBBBF881
:1064500088219A4200F2228526201DF05FFE002846
:1064600040F01C857F4B804AD3ED007A7F4B92ED44
:10647000007A1B78CBED637A8BED647A002B01F008
:106480001D8477EE676A9BF99431CBED606A013326
:10649000CBED617A01F00387069BCBF8983100229F
:1064A0009FED737A73498BED677AFF23D1ED005A24
:1064B0008BF89431FEF7BDBE0120F3F7B3FDDBF896
:1064C0006821069B9A1AFDF703BC6B4BD8ED007A46
:1064D00093ED007AF0EEE77AF4EEC77AF1EE10FA77
:1064E0007DF773ADFDF76BBD91ED016A26EE646A31
:1064F000B0EE674AA6EE074AB4EEC54A34EE666AC5
:10650000F1EE10FA48BFB0EE656A012A83ED006A29
:106510003FF4B5AE91ED056A26EE646AB0EE674AC7
:10652000A6EE074AB4EEC54A34EE666AF1EE10FAFA
:1065300048BFB0EE656A022A83ED016A3FF49FAE60
:1065400091ED096A26EE646AB0EE674AA6EE074A44
:10655000B4EEC54A34EE666AF1EE10FA48BFB0EE0A
:10656000656A032A83ED026A3FF489AE91ED0D6AF4
:1065700026EE646AB0EE674AA6EE074AB4EEC54A54
:1065800034EE666AF1EE10FA48BFB0EE656A042A8E
:1065900083ED036A3FF473AE91ED116A26EE646AEF
:1065A000B0EE674AA6EE074AB4EEC54A34EE666A14
:1065B000F1EE10FA48BFB0EE656A052A83ED046A71
:1065C0003FF45DAE91ED156A26EE646AB0EE674A5F
:1065D000A6EE074AB4EEC54A74EE666AF1EE10FA0A
:1065E00048BFF0EE656A062AC3ED056A3FF447AE80
:1065F000D1ED196A66EEE46AB0EE674AA6EE874A04
:10660000B3EE046AB4EEC54A74EE466AF1EE10FACF
:1066100048BFF0EE656A072AC3ED066A3FF42FAE65
:10662000D1ED1D6A154A059266EEE44A144ADFF878
:106630005CA0144D0792E4EE877AF4EEC57A77EE0B
:10664000C67AF1EE10FAB8BFF0EE657AC3ED077ABC
:10665000FEF7B5B8A2950020A395002098950020DC
:106660000C7C0020CC930020FC8E0020A858002039
:1066700000000000108F0020688E0020287000208D
:10668000FCB9002014540020D8920020E08400209F
:10669000B8499DED107AD1ED007AB74B68EEA77A34
:1066A000FDEEEA6AE7EE097AB0EE487AA7EEA97A3B
:1066B00016EE900AF0EE477AB9F1000F41F08081B2
:1066C000FDEEC77A17EE908A17EE90EA9045A8BFC4
:1066D00096464045C8BF864607EE90EAF8EEE77A50
:1066E000012EC3ED007A3EF466A8D1ED047A9DED4B
:1066F000117A68EEA77AE7EE097AB0EE487AA7EE4B
:10670000A97AFDEEC77A17EE908A17EE90EA9045C7
:10671000A8BF96468045B8BF864607EE90EAF8EED9
:10672000E77A022EC3ED017A3EF445A8D1ED087A4E
:106730009DED127A68EEA77AE7EE097AB0EE487A14
:10674000A7EEA97AFDEEC77A17EE908A17EE90EAC7
:106750009045A8BF96468045B8BF864607EE90EAAA
:10676000F8EEE77A032EC3ED027A3EF424A8D1EDC9
:106770000C7A9DED137A68EEA77AE7EE097AB0EE0F
:10678000487AA7EEA97AFDEEC77A17EE908A17EE3F
:1067900090EA9045A8BF96468045B8BF864607EE6A
:1067A00090EAF8EEE77A042EC3ED037A3EF403A8EC
:1067B000D1ED107A9DED147A68EEA77AE7EE097AAA
:1067C000B0EE487AA7EEA97AFDEEC77A17EE908A66
:1067D00017EE90EA9045A8BF96468045B8BF86461A
:1067E00007EE90EAF8EEE77A052EC3ED047A3DF461
:1067F000E2AFD1ED147A9DED157A68EEA77AE7EE57
:10680000097AB0EE487AA7EEA97AFDEEC77A17EEBC
:10681000908A17EE90EA9045A8BF96468045B8BF8B
:10682000864607EE90EAF8EEE77A062EC3ED057A83
:106830003DF4C1AFD1ED187A9DED167A68EEA77AD6
:10684000E7EE097AB0EE487AA7EEA97AFDEEC77AAC
:1068500017EE908A17EE90EA9045A8BF96468045BD
:10686000B8BF864607EE90EAF8EEE77A072EC3ED4A
:10687000067A3DF4A0AFD1ED1C7A9DED177A68EE53
:10688000A78AE9EE078AA9EEA88AFDEEC87A17EE74
:10689000901A8A42A8BF0A468842D8BF104607EE1F
:1068A000900AF8EEE77AC3ED077AFDF784BF334E1E
:1068B000DBED017A9BED006A3188736977EEA77A88
:1068C000F0EE006AB0EE677AA6EE267A4E1E0BEB6B
:1068D000C601D6EE267A08391033F6EE003A27EED6
:1068E000237A67EEA37A8BED207ACBED217ADFF85D
:1068F00090B05F460BF1800091ED027A91ED036A52
:10690000D7ED036AD7ED027A53ED014A13ED025A2F
:1069100037EE674A76EEC65A77EE277AE4EE845A67
:10692000013EA1F10801E5EE047A07F1080703F141
:10693000080336EE267A00F10800E4EE877AE5EEE9
:10694000475A67EEA37A25EEA37AC0ED007A80ED70
:10695000017AD1D1BCF1140F7EF408AEF3F704FA3A
:10696000DFF82080DBF81421401BA8F80200FEF7B6
:10697000FDBD00BF788E00206C930020D047002022
:10698000242E0020D8920020A64B1978DBF818019D
:10699000A54F9FEDA67AC600BB1983ED007A0029AA
:1069A00001F0B781A24AB0EE476AF0EE476A0023D1
:1069B000F2EC017A013367EEA77A05EE903AB4EE75
:1069C000E77AF1EE10FAF8EEE55AB8BFB0EE677A62
:1069D0008B4276EEA76AA7EEA56AE9D1F5EEC06A0A
:1069E000BB19F1EE10FA83ED007A41F3928186EE45
:1069F000268A904BDFF85882B8F80020F7EE007A2C
:106A000038EE678AD3ED007A68EE277AFDEEE77AF2
:106A100017EE903A812B40F3C7879342A8BF1346E5
:106A200007EE903AB8EEE70A834B304403EB800060
:106A300002F084F8FDEEC07AB8F8003017EE902A24
:106A4000812A40F3AE879342A8BF134607EE903ADF
:106A5000F8EEE77AFCEEE77ACDED057ABDF8143072
:106A6000DBF81801C600BA199380049B1B7810B993
:106A7000132B01F01185152B01F04181142B7EF4AD
:106A800073AD6BE7DBF818216C4B67496C4E184609
:106A9000D30019441A448B88016800EE103A10EEB6
:106AA000103A643BC82BA8BFC823782BB8BF782303
:106AB00007EE903AB8EEC07AF8EEE77A06EB820677
:106AC00077EE670A77EE876A67EE877A20EEA67A16
:106AD000B8EE400AC7EE870A3046D6F81890D6F8C6
:106AE0001C80376A96ED058A17F05AFF049B86EDE5
:106AF000058A1B78C6F81890142BC6F81C803762DC
:106B000001F0DD84DBF818214E48DBF81411013266
:106B100080FB0230A0EBE27000EB4000101A013164
:106B2000CBF81801CBF81411FEF703BD464E4048D0
:106B3000B268B1892BF05FFE049B93F800C0BCF1F2
:106B4000140F01F0C584DBF814210132CBF81421B5
:106B5000AEE6344F39785FEA910E01F01C853B4E6A
:106B60000EF101094FEA491906EB090806F1200365
:106B7000A6F1700013ED076A53ED056A13ED037A71
:106B800053ED017A53ED025A13ED084A53ED064ACC
:106B900013ED045A26EE066A66EEA66A27EE077A19
:106BA00067EEA77AA4EE046A20339845E4EEA46A5F
:106BB00000F11000A5EE057AE5EEA57AF1EEC65AD1
:106BC000B1EEE66AF1EEC76AB1EEE77A40ED085A37
:106BD00000ED076A40ED066A00ED057ACAD1A9F119
:106BE000200333440BEB0E1611F0030018BF0833DB
:106BF0000FD053ED017A13ED027A67EEA77A0138D0
:106C0000E7EE077A03F10803B1EEE77AA6EC017A22
:106C1000EFD1BCF1140F01F067840132CBF81421DD
:106C2000B4E600BFCA470020C04A002000000000B0
:106C3000242E0020CC470020E8490020D0840020EA
:106C40006484002056555555D0470020A42E0020BE
:106C5000C8470020E34E3288D6F804904FEA520825
:106C60004FEA88015FEAD20C0BEB01030BEB8207C2
:106C700000F0A18001F110020CF1010CDA4803EBE5
:106C80000C1C3A44103309F1100E07F1100151EDBC
:106C9000032A51ED043A10ED043A10ED032A51EDA8
:106CA000026A11ED016A10ED021A50ED010A12EDAF
:106CB000044A12ED035A53ED044A53ED035A13EDFF
:106CC000027A53ED017A52ED021A12ED010A73EEC7
:106CD000238A32EE228A40ED048A00ED038A71EEA7
:106CE000268A30EE868A40ED028A00ED018A74EE33
:106CF000848A35EE858A43ED048A03ED038A77EEB4
:106D0000218A37EE808A43ED028A03ED018A73EE11
:106D1000633A75EE655A1EED035A32EE623A74EE2E
:106D2000644A25EE638A1EED044A23EE052A64EECA
:106D3000652AA3EE048A10339C4524EE843AA3EE20
:106D4000842A00F110000EF1100EA5EE853A01F133
:106D5000100102F11002E4EE852A01ED078A01ED2F
:106D6000082A02ED073A42ED082A5EED055A1EEDAB
:106D7000065A71EE666A30EEC66A31EEC77A70EE78
:106D8000677A26EE253A65EEE63A25EE674A67EE23
:106D9000054AE6EE053AA6EE853AA7EE254AE7EE65
:106DA000A54A01ED063A41ED053A02ED064A42EDEB
:106DB000054A7FF46CAF1FFA88F84A4641468B4873
:106DC00020F06CF841467268384620F067F8049B62
:106DD0001B78142B7EF4C8ABC0E5F0EEE76AB7EE83
:106DE000005A35EE665A9FED824ADFED825A9FEDDA
:106DF000826A9FED827A9BED770AF1EEC54AE6EE54
:106E0000845AF5EEC07AA6EEA56AF1EE10FAA6EE67
:106E1000867A48BFDFED7A7A27EE247A48BF37EECC
:106E2000C77A27EE000A2CF07BFEB0F5617F00F3F5
:106E3000398707EE900AB8EEE70ADFED727A20EEA6
:106E4000270A07EE906AB8EEE78AFDEEC07A17EEE1
:106E5000903A2033402B40F22B879FED730A2CF0A1
:106E60005FFE00B207EE900AB8EEE77AFFF75EBA6F
:106E7000654A664B92681B689A423FF6AFAA2B7828
:106E80000C3B022B7EF6E0A8614B2E701A78002A8C
:106E90003EF4DAA800221A70FEF7D6B89BF8A021BB
:106EA000002A7FF4DFAA5B4B5B4993ED007AD1EDBA
:106EB000007A9BF99431CBED637A77EE676A012B08
:106EC000CBED617ACBED606A8BED647A01F0DE8206
:106ED000069BCBF89831514B9FED537AD3ED005A76
:106EE0008BED677A01238BF89431FEF7A2B94C4EF3
